:020000040800F2
:10000000700C012019050008C1D70008F1C60008CE
:10001000E9D50008893300081D110108000000001F
:10002000000000000000000000000000590400086B
:10003000094A000800000000B50400085BE1000860
:1000400037050008370500083705000837050008A0
:100050003705000837050008370500083705000890
:100060003705000837050008370500087143000808
:100070007D4300088943000895430008A143000818
:10008000AD430008B943000837050008BD4A000821
:10009000D54A0008C94A0008E14A000837050008A7
:1000A0003705000837050008370500083705000840
:1000B0003705000837050008370500083705000830
:1000C0003705000837050008370500083705000820
:1000D000A5DF0008C5F50008DDF50008F5F5000806
:1000E0007F4A0008370500080000000037050008B7
:1000F000370500083705000837050008C543000824
:1001000037050008370500083705000837050008DF
:1001100037050008DDEC0008370500083705000842
:10012000D1430008DD430008E9430008F543000817
:1001300037050008370500083705000837050008AF
:1001400000000000000000000000000000000000AF
:10015000370500083705000837050008370500088F
:10016000370500083705000837050008370500087F
:1001700037050008E9D8000837050008000000002E
:100180003705000837050008F5EC000837050008BA
:10019000370500083705000837050008370500084F
:1001A0003705000837050008370500080000000083
:1001B000370500083705000837050008370500082F
:1001C00037050008370500080000000000000000A7
:1001D00000000000000000003705000800000000DB
:1001E000000000000000000000000000000000000F
:1001F0000000000000000000370500083705000877
:100200003705000837050008000000003705000822
:1002100037050008370500083705000837050008CE
:100220003705000800000000370500080000000046
:1002300037050008370500080000000037050008F2
:10024000370500083705000837050008370500089E
:10025000370500083705000837050008370500088E
:10026000370500083705000837050008370500087E
:1002700037050008370500083705000800000000B2
:10028000370500083705000837050008370500085E
:1002900000000000370500083705000800000000D6
:1002A0000000000037050008370500083705000882
:1002B000ADF500083705000837050008ED4A0008CD
:1002C000F94A0008F5E200083705000800F002F8D6
:1002D00000F0B2F80AA090E8000C82448344AAF12E
:1002E0000107DA4501D100F0A7F8AFF2090EBAE82C
:1002F0000F0013F0010F18BFFB1A43F0010318475A
:10030000CC4E0100FC4E01000A444FF0000C10F8E6
:10031000013B13F0070408BF10F8014B1D1108BF83
:1003200010F8015B641E05D010F8016B641E01F823
:10033000016BF9D113F0080F1EBF10F8014BAD1C73
:100340000C1B09D16D1E58BF01F801CBFAD505E091
:1003500014F8016B01F8016B6D1EF9D59142D6D3EB
:10036000704700000023002400250026103A28BF13
:1003700078C1FBD8520728BF30C148BF0B60704717
:100380006E2900F08983702900F0D384662914F067
:10039000CB82652914F0C882672914F0C5826129CF
:1003A00014F0C48203681B0A28BF41F08001692948
:1003B00000F03683642900F03383752900F0308320
:1003C0006F2900F06084782900F09F84E92900F00B
:1003D000FB83E42900F0F883F52900F0F583EF2989
:1003E00000F05D84F82900F09E840368DB0928BFD3
:1003F00041F08001632901F0A581732901F0AA81F0
:10040000E32901F0B581F32901F0BA81002070479A
:100410001FB514F00AFA01F009FA040000200021C7
:1004200014F072F9401C60600020002114F056F9AD
:10043000E0601FBD10B510BD01F0CAF91146FFF70D
:10044000E7FF11F0C3FF01F0A7FA03B4FFF7F2FFD3
:1004500003BC01F0DFFA00002C4B19680868B0E813
:10046000F04F80F30988BFF36F8F4FF0000080F3E7
:10047000118870470000000008480068006880F399
:1004800008884FF0000080F3148862B661B6BFF3AD
:100490004F8FBFF36F8F00DF00BF00BF08ED00E09C
:1004A000DFF80C00016841F470010160704700BF83
:1004B00088ED00E0EFF30980BFF36F8F134B1A68EC
:1004C0001EF0100F08BF20ED108A20E9F04F1060D9
:1004D00009B44FF0500080F31188BFF34F8FBFF382
:1004E0006F8F13F011FA4FF0000080F3118809BCF0
:1004F00019680868B0E8F04F1EF0100F08BFB0ECA4
:10050000108A80F30988BFF36F8F704720010020A5
:10051000EFF30580704700000A4880470A4880478B
:100520000A480047FEE7FEE7FEE7FEE7FEE7FEE7D4
:10053000FEE7FEE7FEE7FEE705480649064A074BE9
:1005400070470000A14A00081DE20008CD02000823
:1005500070AC0020700C012070CC002070CC00200A
:1005600053EA020C00F069802DE9F04B4FF00006D1
:10057000002B1FBFB3FA83F503FA05F424FA05F63E
:100580005E4012BF1643B2FA82F502FA05F4C5F1D5
:1005900020051EBF22FA05FC44EA0C04203556EA69
:1005A000044C4FEA144418BF641C4FF000084FF08D
:1005B0000009904271EB030C39D3002919BFB1FA3D
:1005C00081F701FA07F6B0FA80F700FA07F6C7F1EB
:1005D00020071EBF20FA07FC46EA0C062037B6FBB0
:1005E000F4FCA7EB0507103F07F01F0BCBF120062B
:1005F0000CFA0BFB2CFA06F644BFB3460026202F5C
:10060000A4BF5E464FF0000B5BEA060C08BF4FF03C
:10061000010B19EB0B09ABFB027C48EB0608C01B76
:1006200006FB02CC0BFB03CC71EB0C01C1E70B46C4
:10063000024641464846BDE8F08B13B54FF0000036
:100640004FF00001AFF30080BDE81C407047000090
:100650007CB51D4616460C00009001D02044401E7B
:10066000074B7B442A4669460190304600F02DFA3C
:1006700005461CB10020694600F03AFA28467CBDC8
:100680009504000010B5431C02E010F8011B71B185
:100690008107FAD14FF0013202C88C1A8C4314EA58
:1006A000C211F9D0C01A0A0603D0C01E10BDC01A6C
:1006B00010BD0A0401D0801E10BD0902FCD0401EEE
:1006C00010BD40EA010370B59B072ED14FF00136F3
:1006D000042A2AD308C810C99D1B9D43121F15EA7E
:1006E000C61517D0D8B2E1B2401A50EA056110D150
:1006F00098B2A1B2401A50EA05410AD123F07F40D6
:1007000024F07F41401A50EA052102D1180EA0EBD7
:10071000146070BDA342DBD018BA21BA884201D957
:10072000012070BD4FF0FF3070BD0AB9002070BDD0
:1007300010F8013B11F8014B63B1A3420AD1521EDC
:1007400008D010F8013B11F8014B1BB1A34201D1B5
:10075000521EEDD1181B70BD032A40F2308010F0FC
:10076000030C00F0158011F8013BBCF1020F62444C
:1007700098BF11F801CB00F8013B38BF11F8013BDD
:10078000A2F1040298BF00F801CB38BF00F8013B8A
:1007900011F0030300F02580083AC0F0088051F8FA
:1007A000043B083A51F804CBA0E80810F5E7121D05
:1007B0005CBF51F8043B40F8043BAFF30080D20724
:1007C00024BF11F8013B11F801CB48BF11F8012BF0
:1007D00024BF00F8013B00F801CB48BF00F8012B13
:1007E000704710B5203AC0F00B80B1E81850203A9D
:1007F000A0E81850B1E81850A0E81850BFF4F5AFC1
:100800005FEA027C24BFB1E81850A0E8185044BF4A
:1008100018C918C0BDE810405FEA827C24BF51F8B7
:10082000043B40F8043B08BF7047D20728BF31F8AB
:10083000023B48BF11F8012B28BF20F8023B48BFFC
:1008400000F8012B704702F0FF0343EA032242EA5B
:10085000024200F002B84FF000020429C0F01280FA
:1008600010F0030C00F01B80CCF1040CBCF1020F63
:1008700018BF00F8012BA8BF20F8022BA1EB0C0138
:1008800000F00DB85FEAC17C24BF00F8012B00F82E
:10089000012B48BF00F8012B70474FF0000200B554
:1008A000134694469646203922BFA0E80C50A0E893
:1008B0000C50B1F12001BFF4F7AF090728BFA0E841
:1008C0000C5048BF0CC05DF804EB890028BF40F80D
:1008D000042B08BF704748BF20F8022B11F0804F4F
:1008E00018BF00F8012B704710B5044610F0030F35
:1008F00008BF11F0030F40F015804FF0013E121FAA
:10090000C0F20E8051F8043BA3EB0E0C2CEA030C52
:100910001CEACE1C08BF40F8043BF0D0A1F1040152
:1009200002F10402521E08DB11F8013B002B00F813
:10093000013BF7D11146FFF78EFF204610BD7047EF
:100940007047704710B500F0C3FA006810BD10B5CD
:10095000044600F0BDFA046010BD70B50446856918
:100960000068C10601D5302600E02026C00707D068
:1009700070BDD4E9012130469047206A401C2062B6
:100980006D1EF6D570BD70B5044685690078C00748
:1009900007D170BDD4E9012120209047206A401C76
:1009A00020626D1EF6D570BD09684A0501D540B2BA
:1009B0007047C905FCD500B2704709684A0501D5E2
:1009C000C0B27047C905FCD580B2704770B50C46FF
:1009D0000546012A05D02878800600D5EA6900235B
:1009E00002E0012305E05B1C934202D2E05C002898
:1009F000F9D1A869E618C01AA861286A18442862C3
:100A00002846FFF7AAFF04E0D5E9012114F8010BFD
:100A10009047B442F8D32846FFF7B5FF70BD0000F9
:100A20002DE9F0410646002410687529314616A5C7
:100A300010D0FFF7B9FF002802DA404213A507E003
:100A400031688A0701D512A502E0490704D511A52E
:100A5000012401E0FFF7B1FF00210A2206F124077B
:100A600009E0B0FBF2FCB0FBF2F302FB1C003030FB
:100A700078541846491C0028F3D123462A463046AC
:100A8000BDE8F04100F06DBA000000002D0000004C
:100A90002B0000002000000011680268006A530566
:100AA00001D508700AE0D30501D5088006E01306D9
:100AB00003D5C217C1E9000200E0086001207047B9
:100AC00001694A1C02610878704700B58FB0CDE912
:100AD00001310021059105497944CDE90310114602
:100AE000684600F031F90FB000BD0000E5FFFFFFE0
:100AF0000A6802F8010B0A607047D1E900239A42A4
:100B000002D2531C0B601070704700002DE9FF5F8C
:100B100015468A460446DFF8AC80F8440027D8E939
:100B200000103E46CDE9001010E03AF816106A4673
:100B300002A800F029FE411C07D02178890603D5C0
:100B4000E269391891420DD80744761C2078800656
:100B500002D5E069B84205DDAE42E6DB3AF81600A0
:100B60000028E2D1A069C01BA0612046FFF7F5FE76
:100B7000D8E90010CDE90010002017E03AF818106D
:100B80006A4602A800F000FEB0F1FF3F81460BD09C
:100B900000250DF1080B05E0D4E901211BF8050043
:100BA00090476D1C4D45F7D308F10100B0428046D7
:100BB000E4DB206A384420622046FFF7E4FEBDE80B
:100BC000FF9F0000864301002DE9F0418046D21DC1
:100BD00022F007020025D2E90002F52915A614D05B
:100BE000011E72F1000106DA0023D0EB030063EB73
:100BF000020211A608E0D8F800108B0701D50FA655
:100C000002E0490701D50EA601251146002408F18E
:100C1000240704E000F060F930323A55641C50EAD1
:100C20000102F7D12B46324621464046BDE8F0414D
:100C300000F097B9000000002D0000002B0000001C
:100C40002000000030B4002100F1240408E002F08C
:100C50000705D208303542EA4372DB086554491C67
:100C600052EA0305F3D10468002310A2250707D533
:100C7000A40600D421B1C46901230DA2641EC4617D
:100C800030BC00F06EB910B5044621461068FFF77D
:100C900094FE02462046BDE810400023D2E7D21D54
:100CA00022F00701D1E90023CCE70000000000009A
:100CB00030000000F0B40D460188090502D5214C32
:100CC0007C4402E01F4C7C440E34002100F12406D9
:100CD00008E002F00F071209E75D42EA03721B0900
:100CE0007754491C52EA0307F3D102780023120714
:100CF00004D5702D06D009B1022311342246F0BC70
:100D000000F02FB901231034F8E770B504460D4602
:100D100021461068FFF751FE024629462046BDE8ED
:100D200070400023C6E7D21D22F00703D3E9002359
:100D3000C0E70368126843F0200303600823C3611F
:100D40000023B7E7E84101002DE9F05F894604463A
:100D50004FF0000ADFF874B1FB44C0F820A0204631
:100D6000E1688847002874D0252806D0D4E90121FD
:100D70009047206A401C2062F1E700265F4620462B
:100D8000E16888472028054607DB312D05D2781910
:100D900010F8200C08B10643F1E7B00701D526F0A2
:100DA0000406C4F81CA00027C4F818A02A2D09D0F6
:100DB000284611F039FA38B304EB8708303DC8F8FB
:100DC000185019E059F8041B204604EB8702916182
:100DD000E1688847012F054618D1E069002820DA2C
:100DE00026F020061DE0D8F8180000EB800005EB87
:100DF00040003038C8F818002046E16888470546AA
:100E000011F012FA0028EED1012F0AD02E2D08D1B0
:100E10002046E16888477F1C0546022F46F02006E1
:100E2000C4DBA069002803DA404246F00106A06155
:100E3000F00701D026F010066C2D0BD0682D09D0DC
:100E40004C2D39D06A2D35D0742D35D07A2D33D034
:100E500016E038E0E1682F4620468847B84205464C
:100E600009D16C2F26D04FF48060E16806432046FC
:100E70008847054604E06C2F1AD04FF48070064373
:100E80000DB3A5F14100192802D8203546F40066BB
:100E90004A462946204626604E46FFF771FA80B141
:100EA00001280BD0F61D26F0070000F1080956E7CF
:100EB0004020E4E78020D8E70020D6E706F10409C7
:100EC0004DE7284652E7206ABDE8F09F78410100CF
:100ED000004870470CAC002030B5B0F10A024FEA70
:100EE000900E71F100034EEA817EB0EB0E0061EBD3
:100EF00091014FEA101E4EEA017E10EB0E0041EB0D
:100F000011114FEA102E4EEA016E10EB0E0041EB6C
:100F100011214FEA104E4EEA014E10EB0E0041EB4C
:100F20001141401841F100014FEAD00040EA417000
:100F30004FEAD10110EB80054FEA810444EA907436
:100F400044EB01046D1944EB0404521BA3414FF020
:100F5000000348BF0A3200D530BD401C41F10001FA
:100F600030BD2DE9F0470D4699469246044600F102
:100F700024080168880604D5E06921F01001216089
:100F800000E00120A84201DD471B00E00027A16925
:100F90007A1902EB0900081AA0612078C00602D471
:100FA0002046FFF7DAFC002608E0D4E901211AF810
:100FB00006009047206A401C761C20624E45F4DBF8
:100FC0002078C0060AD52046FFF7C7FC06E0D4E922
:100FD000012130209047206A401C2062381EA7F172
:100FE0000107F4DC07E0D4E9012118F80500904777
:100FF000206A401C2062281EA5F10105F3DC204672
:10100000FFF7C1FC2078000602D50220BDE8F0877A
:101010000120FBE770472DE9FF4F0C461E464FF0BD
:10102000FF378BB0D2E90001DDF860800A908A4674
:10103000C1F30A5505B93D46002108464FF00000AE
:10104000BAF1000F00F4400005DA00EB80004FF425
:10105000400101EA50004FEA9059B9F1010F00DD5B
:10106000B9460A9850EA4A000ED044F61050A5F24C
:10107000FF3545432F14B8F1000F1ED07542291ECD
:101080001EDDC9F100021CE0B8F1010F4FF00000B5
:1010900001D0302103E0F24305E02154401CB0426E
:1010A000FBDB30460022002121540B99C1F8088057
:1010B000C1E900200FB0BDE8F08FBD1B6D1CDEE75D
:1010C0004A4600DA694206A800F0F4FB06AB93E852
:1010D000070003AB83E8070050460A9900F0A1FC23
:1010E0008DE80700A0F500501F3800900398002DF0
:1010F0000ADD42F21F014A460844002303A9039077
:10110000684600F00AFF09E0A0F500504A461F3883
:10111000002303A90390684600F014FF8DE8070040
:101120000004000C03D04FF0FF30410800E01046EF
:10113000B8F1000F03D00022009215461EE0751E84
:1011400005D4FFF7C9FE303262556D1EF9D5B3469E
:101150000122084302D000227F1C04E020783028BE
:1011600001D100227F1E002A099784D01DE0112D95
:1011700007DAFFF7B1FE303262556D1C50EA01020A
:10118000F5D1084302D00098C8B10EE00021681ED6
:1011900005E0235C625C63542254401E491C81427A
:1011A000F7DBAB46A81B401E0990002004F80B009B
:1011B0000B98099AC0F80880C0E9002B7AE711263D
:1011C0004FF0000857E72DE9F04F88460446D21D3E
:1011D00022F0070191B0D1E90001CDE90A010FF039
:1011E0009EFF02460B98C00F01D02D2007E020681B
:1011F000810701D52B2002E0202101EAC000032A4B
:10120000099001D0072A05DB03464146204600F03D
:1012100011FB0BE12078800601D5E06900E0062093
:10122000B8F1650F814606D0B8F1660F18D0B8F155
:10123000670F70D131E00020B9F1110F009001DB90
:10124000112301E009F101030AAA01A90CA8FFF783
:10125000E2FEDDE90C70002609F10105834647E056
:1012600001204B4600904FF000470AAA01A90CA8A4
:10127000FFF7D1FEDDE90DB00C995D46002610B9EF
:1012800009F101000D18B9EB050003D4C0F1FF36D8
:1012900009F10105A5EB09002BE0B9F1010F01DA15
:1012A0004FF001090020B9F1110F0090484601DD0F
:1012B000112300E003460AAA01A90CA8FFF7ABFE20
:1012C000DDE90C704D4600268346207800070AD4DD
:1012D000AB4500DA5D4601A8012D04DD411911F886
:1012E000011C302907D04F4502DA17F1040F04DA48
:1012F000012082460FE06D1EEEE7002F02DCED1BA1
:101300003E4403E0781CA84200DD7D1CB81B00F1C0
:10131000010A4FF000472078000703D4AA4501DBFB
:101320004FF0FF3A0021B7F1004F0DF143088DF85F
:10133000431024D002202B23002F01DA7F422D23DB
:101340000A21021EA0F1010000DC5FB197FBF1FC55
:1013500097FBF1F201FB1C7C17460CF1300C08F8EE
:1013600001CDEEE7A8F1010003702188090501D540
:10137000452100E06521A0F1010800F8011C099851
:101380000FA9A1EB0807FF1D00B10120411901EBD6
:10139000EA70A1693844081A401EA0612078C0068E
:1013A00002D42046FFF7D9FA099828B1D4E90121DF
:1013B0009047206A401C20622078C00622D5204633
:1013C000FFF7CBFA1EE0002E04DBB34502DD01A8D7
:1013D000805D00E03020D4E901219047206A401C64
:1013E0002062761CAAF101005FEA000A0AD100F02F
:1013F0001DFAC0680168405CD4E901219047206A69
:10140000401C2062281EA5F10105DCDC07E0D4E9C0
:10141000012118F8010B9047206A401C2062381EF9
:10142000A7F10107F3DC2046FFF7ADFA032011B066
:1014300041E600002DE9F04F04460D46D21D22F092
:10144000070089B0D0E90097484639460FF067FE9B
:101450000246F80F01D02D2307E02068810701D54F
:101460002B2302E0202101EAC0038DF820300BB1CC
:10147000012000E00020032A824601D0072A04DB75
:101480002946204600F0D6F93FE12078800601D4B5
:101490000D2500E0E569C7F30A560D2D49DA002154
:1014A0004FEA175B08464FF00000002F00F44000A1
:1014B00007DA00EB80004FF4400100EBD07001EA46
:1014C00060008115012901DD4FF0FF3100224FEA54
:1014D000850CBCF1180F06D31346ACF118004FF081
:1014E0008052C24003E04FF4801323FA0CF30CF156
:1014F0000C0CBCF1200F04D3ACF1200C09FA0CF059
:1015000001E007FA0CF000294FF0004801DD18B99E
:101510000FE00ED140450CD319EB02095F4121B910
:10152000404502D19F4329EA0209BBEB175F00D077
:10153000761C2088000502D57B48784402E07A4872
:101540007844193808AA302302F80A30037C0AF1DB
:101550000101002E0AF1020A53546A4602DC4FF0E0
:10156000300101E04FF031014FF001088DF800101B
:1015700002D0A6F2FF3603E059EA470100D06B4ED5
:10158000002D02DC2178090704D54FF002082E2136
:101590008DF80110C44600210BE0C7F303433F015F
:1015A000C35C491C6D1E02F80830052908F10108CA
:1015B00001DA002DF1DC00210CE000EB1973491C6D
:1015C0001B786D1E082902F808304FEA091908F146
:1015D000010801DA002DF0DC21688B0602D516E047
:1015E000A8F10108E04505DD02EB080313F8013C12
:1015F000302BF5D0B8F1000F09DD02EB080313F82A
:10160000013C2E2B03D1090701D4A8F10108002DBC
:1016100005DD3E2102F808106D1E08F10108407C2E
:10162000002E02F8080008F1010804DA2D207642A5
:1016300002F8080002E02B2002F808000A214FF40B
:101640007A70864208F101080BDB96FBF0F3303329
:1016500002F8083096FBF0F308F1010800FB13666E
:1016600001E0642E0CDB642096FBF0F3303302F8CB
:10167000083096FBF0F308F1010800FB136601E067
:101680000A2E06DB96FBF1F0303002F8080008F174
:10169000010896FBF1F001FB1060303002F8080001
:1016A000A16908F1010808EB050202EB0A00081A1B
:1016B000A0612078C00602D42046FFF74EF9216AC7
:1016C00008AE01EB0A00206204E0D4E9012116F81B
:1016D000010B9047BAF1010AF7D22078C00602D573
:1016E0002046FFF73AF96E4609E016F8010B3E284E
:1016F0000FD0D4E901219047206A401C2062B8F144
:101700000108F2D22046FFF73EF909B00320BDE8F8
:10171000F08F206A2844206203E0D4E901213020C0
:1017200090476D1EEBD3F8E77D3A010002FCFFFF06
:1017300010B5436913B1AFF3008001E0FFF746F93C
:10174000012010BD127800F124010A7000224A70B5
:101750000122EDE711684FF0FF32E9E710B5436968
:1017600013B1AFF3008001E0FFF7D0F9012010BD05
:10177000128800F1240182840022C2840122EDE754
:1017800011684FF0FF32E9E770B516460C46054682
:1017900000F044F8036893F80101012806D0FF2CFB
:1017A0000FD8185D68B101202C7070BDD3F8070107
:1017B0003246214603F2071303442846BDE8704031
:1017C00018474FF0FF3070BD004870470CAC002048
:1017D0007546FFF7F9FFAE4605006946534620F00F
:1017E0000700854618B020B5FEF7A6FEBDE82040EC
:1017F0004FF000064FF000074FF000084FF0000BCD
:1018000021F00701AC46ACE8C009ACE8C009ACE87F
:10181000C009ACE8C0098D467047000010B500F063
:1018200005F8001D10BD00BFE12E01000048704703
:101830002CAC00202DE9F0411F4604460326016828
:10184000072A01F4006004DB08B116A505E016A51F
:1018500003E008B115A500E015A521F010002060F7
:10186000A069C01EA0610FB1401EA0612046FFF715
:1018700074F84FB1D4E9012138469047206A401CE2
:101880002062C01C206206E0206AFAE7D4E9012148
:1018900015F8010B9047761EF8D22046FFF773F833
:1018A000BDE8F0814E414E006E616E00494E46002B
:1018B000696E66002DE9F047814616468AB03548C4
:1018C00078440DC88DE80D0032487844801C03AC84
:1018D0000DC884E80D0041F69B300844372190FB89
:1018E000F1F290FBF1F5A5F1800501FB12041B3C20
:1018F00002D56442012000E00020DFF898A0804675
:101900000027FA44AAF1BE0A0EE0E0070AD03246E8
:10191000684607EB470101230AEB810100F012FB47
:101920008DE8070064107F1C002CEED1194F7F4416
:10193000AE3F19E0E80715D007EB04100DF1180AC7
:1019400090E80E008AE80E00C068F04201D19819B4
:1019500008903246012306A903A800F0F3FA03AB6E
:1019600083E807006D10641C002DE3D14FF00103E4
:1019700032466946B8F1000F03A802D000F0CDFA54
:1019800001E000F0DFFAC9E90001C9F808200AB057
:10199000BDE8F0878837010010B50446AFF300803A
:1019A0002046BDE81040FEF750BD00004FF0013C5E
:1019B00050F8042B51F8043B9A4215D1A2EB0C03CA
:1019C000934313EACC130BD150F8042B51F8043B8A
:1019D0009A4209D1A2EB0C03934313EACC13E7D04C
:1019E0004FF00000704700BFD01A01BAB1FA81F180
:1019F00001F0180122FA01F0CB40C1F12001DBB265
:101A0000C0B2C01A2CFA01F3D11A914311EAC311E2
:101A1000E6D1704701491820ABBEFEE72600020060
:101A200070475FEA400C08BF91F0000F4FEA8C232B
:101A30004FEAC12243EA51514FEA1C5018BF00F54A
:101A4000F0404FEA300018BF41F000415FEA6C5CA3
:101A500000F02980BCF1FF3F08BF40F08040704794
:101A6000130C06BF12044FF0100C4FF0000C130EB5
:101A700004BF12020CF1080C130F04BF12010CF189
:101A8000040C930F04BF92000CF1020CD30F04BF9F
:101A900052000CF1010C11464FF00002A0F11F00A2
:101AA000A0EB0C00704711F0004F08BF704731F0F9
:101AB00000413FF4D5AF0B0C06BF09044FF0100CEA
:101AC0004FF0000C0B0E04BF09020CF1080C0B0FB9
:101AD00004BF09010CF1040C8B0F04BF89000CF149
:101AE000020CCB0F04BF49000CF1010CCCF1200318
:101AF000A0EB0C0022FA03F302FA0CF241EA030114
:101B000000F10100704720F07F4C80EA030023F0D1
:101B10007F47ACEB070303F57C5300F0004003F173
:101B2000FF032DE980494FEA154B09B44FEA1443EE
:101B300025EA0B4E24EA03480FF2042606EB13278E
:101B400049083E785FEA320203FB0667C7F50007E3
:101B500007FB06F64FEA54374FEAD64606F102066F
:101B600007FB066CCCF1005C4FEA1C472CEA074CE3
:101B700007FB06F40CFB06F504EB15464FEA961638
:101B800034BF00204FF000404FEAD13706FB07FC7E
:101B90004FEA1C4C0CFB0BF7D21B03FB0CF761EB61
:101BA00007010CFB0EF7B0EB074072EB17420CFB82
:101BB00008F734BFA2EB0742B2EB074261EB1741D3
:101BC0004FEA0C444FEA910706FB07FC4FEA1C4C16
:101BD0000CFB0BF7B0EBC74072EB573203FB0CF773
:101BE00034BFA2EBC742B2EBC74261EB57310CFBEB
:101BF0000EF7B0EBC70072EB57720CFB08F734BF5F
:101C0000A2EBC702B2EBC70261EB5771039F4FEA29
:101C1000816141EA921104EBCC044FEAD1374FEADB
:101C2000826206FB07FC42EA90124FEA80604FEAAC
:101C30001C4C0CFB0BF7D21B03FB0CF761EB0701F1
:101C40000CFB0EF7B0EB074072EB17420CFB08F7EA
:101C500034BFA2EB0742B2EB074261EB17414FEAF8
:101C60008C554FEA910704EB9C2406FB07FC4FEAD6
:101C70001C4C0CFB0BF7B0EBC74072EB573203FB6D
:101C80000CF734BFA2EBC742B2EBC74261EB57314E
:101C90000CFB0EF7B0EBC70072EB57720CFB08F7AA
:101CA00034BFA2EBC702B2EBC70261EB577115EB71
:101CB0004C254FEA816141EA92114FEA82624FEA74
:101CC000D13742EA901206FB07FC44F100044FEAC8
:101CD00080604FEA1C4C0CFB0BF7D21B03FB0CF78C
:101CE00061EB07010CFB0EF7B0EB074072EB1742FC
:101CF0000CFB08F734BFA2EB0742B2EB074261EBE3
:101D0000174115EB1C154FEA813141EA92414FEA28
:101D1000823242EA90424FEA80304FEA0C7644F138
:101D2000000448EA03434EEA0B484FF0000EB2EBC2
:101D3000080C71EB030724BF624639464EEB0E0ECA
:101D40004FF0000B0018524149414BEB0B0BB2EB2B
:101D5000080C71EB03077BF1000B24BF6246394688
:101D60004EEB0E0E4FF0000B0018524149414BEB69
:101D70000B0BB2EB080C71EB03077BF1000B24BFDC
:101D8000624639464EEB0E0E51EA020718BF46F086
:101D9000010616EB0E7655F1000254F1000103D551
:101DA000BDE88901BDE80088BDE88901BDE80048BB
:101DB000B619524141EB0101A3F101037047808044
:101DC0007F7E7D7C7B7A7978777676757473727195
:101DD00071706F6E6E6D6C6C6B6A6A69686867664D
:101DE00066656464636362616160605F5F5E5E5DDF
:101DF0005D5C5C5B5B5A5A59595858575756565553
:101E000055555454535352525251515050504F4FB4
:101E10004F4E4E4D4D4D4C4C4C4B4B4B4A4A4A4904
:101E20004949484848474747474646464545454447
:101E30004444444343434342424242414141002BD4
:101E40009C4630D477002BD01CB54FEA370703B43B
:101E50004FF010004FF01001BAF1000F06D0BCF1A6
:101E6000000FDCBF40F0080040F008014FF0000018
:101E70000FBCBDE810400BF1010BBBF1010F08BF17
:101E80005FEA170722BF12F1010211F101014FF0C1
:101E9000004143F1000300F0004043EA00007047B6
:101EA000F9D35708D0E746EA064613F1400F4FEA48
:101EB00016461FDD13F1200FDFBF16430A4600212F
:101EC00020335B42BED0C3F1200746EA064602FA41
:101ED00007F74FEA164646EA0706C3F1200722FA3B
:101EE00003F201FA07F721FA03F14FF0000342EA87
:101EF0000702A7E746EA020646EA06464FEA164602
:101F000046EA0106BCBF46EA0646360C4FF000031F
:101F10004FF000024FF0000194E72DE9804C9A4603
:101F2000934670B491E8380007C831EA400C48BFC6
:101F300034EA430C03D5FFF7E6FDFFF780FFF0BC62
:101F4000BDE8008C2DE9804C9A46934670B491E828
:101F5000380007C810F0804F08BF13F0804F03D13E
:101F600000F005F8FFF76BFFF0BCBDE8008C20F037
:101F70007F4780EA030023F07F4C07EB0C03A3F5B7
:101F80007C5300F00040A3F1FE0392F0000F00F03C
:101F9000B38095F0000F00F077802DE901494FEAFA
:101FA00011404FEA144621EA004800FB06FC24EAEF
:101FB000064708FB06F607FB08F800FB07F718EBD7
:101FC00006484CEB164C4FEA124B18EB07484FEA09
:101FD00015464CEB174022EA0B4E0BFB06FC25EA9C
:101FE00006470EFB06F607FB0EFE0BFB07F71EEB84
:101FF000064E4CEB164C4FF000061EEB074E4CEB1A
:10200000174B18EB0B0840F1000018EB0E0B58EBC8
:10201000000840F100008F1A4FF000013CBFC94397
:10202000661B14BFB5EB040C00213CBFC943F61B73
:102030004FEA17444EEA8E0E27EA04454FEA1C4742
:1020400004FB07622CEA074C05FB07F70CFB05F6BF
:1020500004FB0CFC16EB074642EB174216EB0C4652
:1020600042EB1C421BEB060658EB0202414146EADA
:102070009E0601D5BDE80189B619524141EB010127
:10208000A3F10103BDE801894FEA14454FEA114766
:1020900024EA054621EA074C05FB07F406FB07F78F
:1020A0000CFB06F105FB0CFC11EB074144EB17445C
:1020B0004FEA124711EB0C4144EB1C4422EA074C57
:1020C00005FB07F206FB07F70CFB06F605FB0CFC0D
:1020D00016EB074642EB174216EB0C4642EB1C454B
:1020E0006A1854F1000148BF7047B619524141EBDC
:1020F0000101A3F10103704795F0000F37D04FEABB
:1021000011424FEA144721EA024624EA074C02FB37
:1021100007F106FB07F70CFB06F402FB0CFC14EBC3
:10212000074441EB17414FEA154714EB0C4441EBD0
:102130001C4125EA074C02FB07F506FB07F70CFBE1
:1021400006F602FB0CFC16EB074645EB174516EBB3
:102150000C4645EB1C42121951F1000148BF704773
:10216000B619524141EB0101A3F1010370474FEA57
:1021700014454FEA114724EA054621EA074C05FBBE
:1021800007F106FB07F70CFB06F24FF0000605FB14
:102190000CFC12EB074241EB174112EB0C4251EBE6
:1021A0001C4148BF7047921841EB0101A3F10103A4
:1021B0007047000010B5324904460068884202D0DA
:1021C000304A904202D1D1F8080302E02E48D0F8FC
:1021D000080310F4403F10D007F0A8FD6168B1F586
:1021E000803F06D0B1F5003F03D0B1F5403F26D186
:1021F00001E0090C17E0800821E000214FF40020E5
:1022000006F04CFE61688A03920B18D18A140C2ADE
:1022100015D2DFE802F0140606060606060B0D0FBF
:102220001113890C4900B0FBF1F008E0000906E049
:10223000400904E0800902E0C00900E0000A1349F7
:102240004008884204D82068816821F4407108E081
:102250000F49884207D82068816821F4407141F411
:102260008071816010BD0B4988422068816804D864
:1022700021F4407141F40071F3E741F44071F0E75B
:10228000002002400021024000600258105E5F0002
:1022900020BCBE0040787D0170B505000C464FF0B3
:1022A000FF302DED028B5AD0002C58D0D4ED010A0E
:1022B000D4ED001A94ED020A20EEA01A61EEA01AE5
:1022C00094ED032AF7EE008A00EE001A40EE021A9F
:1022D000B0EE008AF0EE680A41EE480A21EE880A64
:1022E0000FF072FA85ED010A94ED000AD4ED021A9E
:1022F000D4ED030A94ED011A20EE210A00EEC10A82
:1023000020EE080AF0EEC00A10EE900AB0F17E5FEF
:1023100006DB10EE101A134860F31E01A96003E0FB
:102320000EF0D2FF85ED020A94ED021AD4ED001AE8
:1023300094ED030A21EE012AD4ED012A61EE801A00
:10234000F0EE680A00EE002A42EE811A42EE480AD8
:1023500021EE880A0FF038FA002085ED000ABDEC66
:10236000028B70BDDB0FC93F70B504000D463ED037
:10237000B7EE001ADFED380AC1EE001A84ED001A3C
:10238000C4ED010AC4ED020AC4ED030AC4ED041A47
:1023900065B3D5ED000A95ED010AB7EEE01AB7EE88
:1023A000C00A0FF02DF9B7EEC00BD5ED002ADFED16
:1023B0002B0A9FED2B1ADFED2B1A9FED2B2AF5EE42
:1023C000C02AB1EE400AF1EE10FA13D1D5ED012A80
:1023D000F5EEC02AF1EE10FA0CD1D5ED022AF5EE99
:1023E000C02AF1EE10FA05D1C4EC040A32E04FF035
:1023F000FF3070BD10EE101A1C48814204DBB5EEB0
:10240000C00AF1EE10FA0ADD9FED190ADFED190A94
:102410009FED191ADFED191A84EC040A1AE010EE88
:10242000102A17498A42DFDB10EE102A8242DBDCD9
:1024300010EE102A13488242D6DB10EE102A8A4290
:10244000D2DC10EE101A8142CEDBB5EEC00AF1EEFE
:1024500010FAC9DC002070BD00000000C5064D3F29
:102460002D4A0D3C56A439BBAD47193FDB0FC93F80
:102470006E597F3F0C53B039AB88BBBB8595973DF8
:10248000DB0F49400000B44230B504004FF0FF308C
:102490002DED108BA1B07CD000297AD0002A78D005
:1024A0009FEDFE0AFE4D85ED000AA3B1D3ED009A23
:1024B000D3ED018A93ED029AF5EEC09AF1EE10FA8F
:1024C00011D1F5EEC08AF1EE10FA0CD1B5EEC09A3A
:1024D000F1EE10FA07D121B02046BDEC108BBDE81B
:1024E000304000F011BA94ED000A92ED001AD2EDDE
:1024F000010AD2ED021A94ED013AD1ED00AA20EEC4
:10250000014A60EE203A60EE214A23EE415AD4EDB2
:10251000022A94ED032A91ED01AA91ED028AF5EECB
:10252000C0AAB6EE000AF1EE10FA02EEE05A02EE90
:10253000A14A43EE613A43EE204A02EE615A02EEAE
:10254000604A42EE013A42EEC14A25EE00FA64EEDC
:1025500000EA23EE80EA64EE80DA09D1B5EEC0AA83
:10256000F1EE10FA04D1B5EEC08AF1EE10FA7CD08B
:102570002AEEAA0A0AEE0A0A08EE080A0AF0D6F8B3
:102580006AEE801ACDED0B1A6AEE001ACDED0A1A2A
:1025900000E0B4E168EE001A29EEA90ACDED091AAF
:1025A00008EEA80A09EE090A0AF0C0F8D4EC021AEB
:1025B000B0EE008AD4ED030A69EE80AA94ED021A07
:1025C00061EEA12A20EE883A21EE88BA62EE08BABE
:1025D000F0EE629A61EE822A8DED163A21EE08AA9B
:1025E000CDED122A61EE812A61EEA01A68EE808A92
:1025F000CDED192A62EE012ACDED1D1A29EE009AC1
:10260000CDED1C2A6BEE2A2A2BEEAA7A2AEE200A9E
:10261000CDED112A8DED1A7A60EEA21A8DED1B0A0E
:102620006BEE282A2AEEA90A48EEA91ACDED182A3F
:1026300062EE02CA02EEE00A6BEE092A62EE20FAAE
:1026400021EE01CA20EEA0DA42EEC21A02EE810AA1
:102650002BEEA82A47EE011A0AEEAC0A48EEEC1A55
:1026600002EE010A48EE8C1A00E005E12BEE892A01
:102670002BEE013A02EE200A2AEE092A42EE201A37
:102680000AEECC0A61EE200ACDED000A48EECD1A22
:102690000AEECD0A8DED043A20EE000A01EEA10A01
:1026A0000AF044F8DDED1C2ADDED1D1ADDED000A0F
:1026B000B7EE002A32EEE11ADDED122A9DED043A62
:1026C000DDED0A1A72EEA04AC2EE000A9DED1B0A69
:1026D0001FEE883A0CEEC82A02EE880A6AEE285AE3
:1026E0000CEE482A70EE612ADDED0B1A73EE611ACA
:1026F000B6EE003A22EEAB0A73EE4C3A33EE6C3A89
:1027000061EEABBA0AEE610A21EE201A33EE4C6A92
:102710009DED163A4AEE22BA73EECD3A22EE837A56
:1027200021EE83AA94ED013A63EEA03A0BEE617AB2
:102730000BEE22AADDED091ADDED192AB1EE00BA81
:1027400072EE617A72EEAF1A7FEEE26A23EE0B2A26
:10275000DDED182A21EEA04A20EE885A63EE221AF7
:1027600002EE67AA94ED022ADDED112A42EEC21AAA
:1027700062EE0B2A49EE291AF0EE479A9DED1A7A7D
:1027800042EEE79AD4ED032A65EE427A47EE221A2A
:1027900094ED007A49EE6C1A45EEA21A62EE205AC8
:1027A000B0EE65BA49EE4C1A49EE0D1A01EEA41AC4
:1027B00063EE214A41EEA63A01EE87BA01EE864A5F
:1027C000B0EE64CA62EE216A05EE62CAB0EE645AE7
:1027D00073EEEA3A22EEA16A00EEE25A41EEC77ABF
:1027E00006EEE30A06EE23AA31EE686A63EE204A9B
:1027F00021EE881A40EEC76AF0EE40AA22EEA08AC7
:1028000045EE06AA27EE207A74EE490AB0EE640A75
:1028100047EEA39A01EEA20A0BEE06AA01EE438A46
:1028200045EEA0AA4CEE23BA01EE427A40EE069A9B
:1028300008EE20AA2AEEAA0A46EE86BA47EE209AA9
:102840000AEE0A0A44EEA0BA09EEA90A0BEEAB0A98
:1028500009F06CFF6AEE800A2AEE001A69EE801A0F
:102860002BEE802A95ED000A00EE60FA40EE41EA78
:1028700000EE61EA40EE42DA94ED040A94ED002A9B
:1028800094ED011AD4ED020A0FEE002A0EEE801A22
:102890004EEE000AD4ED031A04E000009EEF273D3F
:1028A000A80100204DEE801A22EE020A84ED002AD3
:1028B00084ED011AC4ED020A01EE010AC4ED031A07
:1028C00000EEA00A01EEA10A09F030FF94ED001A13
:1028D00094ED012AD4ED021AD4ED030A21EE001A78
:1028E00022EE002A61EE801A20EE800A84ED001AA2
:1028F00084ED012AC4ED021A002084ED030A21B000
:10290000BDEC108B30BD000070B504004FF0FF30FF
:102910002DED0C8B7ED000297CD0002A7AD09FED43
:10292000860A864DF6EE001A85ED000AD2ED000A01
:1029300092ED010A92ED021A91ED00BA94ED022A8D
:10294000D4ED032AD1ED018A91ED028AB5EEC0BA29
:1029500094EC023A23EE204A63EE004A23EE013A59
:1029600023EEE05AF1EE10FA02EE405A02EE014A6E
:1029700043EEC14A03EE803A02EEC15A02EEC04A6B
:1029800042EEA04A02EE603A65EE21AA24EE21AAA8
:1029900064EEA19A23EE219A09D1F5EEC08AF1EEF8
:1029A00010FA04D1B5EEC08AF1EE10FA7ED02BEE0B
:1029B0000B0A08EEA80A08EE080A09F0B7FE94ED23
:1029C000004AF1EE000AD4ED011AF0EE003A94ED5F
:1029D000022A94ED033A2BEE001AB2EE005A68EE8A
:1029E000802A68EE004A24EE047A24EE23BA64EECC
:1029F00020CA21EEA00A63EE035A23EE236A62EE98
:102A0000206A22EE024A61EEA17A62EE23BA21EE3A
:102A100085CA00E08DE021EEA3DA62EE053A27EEEA
:102A2000205A20EE257A27EEA08A64EE20DA65EEA1
:102A3000020A06EE417A28EE038A6CEE848A4BEE97
:102A4000010A0DEE418A05EE217A4BEE818A46EEAF
:102A5000A50A0DEE838A0BEE627A4CEEA78A46EE4B
:102A6000620A0BEEE28A37EE40BA4DEE628A70EEF1
:102A7000E6BA0CEE27BA43EEA7BA0CEE04BA43EE60
:102A800084BA00EE24BA28EEA80A46EEA4BA0BEEE9
:102A90000B0A0BEEAB0A08EE080A09F047FE28EE17
:102AA000801A6BEE000A6BEE801A00E00BE028EE55
:102AB000002A95ED000A40EE41AA00EE60AA40EE21
:102AC000619A00EE429A201D94ED002A94ED040ACA
:102AD000D0EC030A0AEE802A4AEE000A09EE801AB8
:102AE00049EE001A22EE020A84ED002A00EEA00A46
:102AF000C0EC030A01EE010A01EEA10A09F016FE7C
:102B000094ED001A94ED012AD4ED021AD4ED030AD3
:102B100021EE001A22EE002A61EE801A20EE800AD1
:102B200084ED001A84ED012AC4ED021A002084ED20
:102B3000030ABDEC0C8B70BD022B073DA8010020E1
:102B4000B1EE601AB4EEC10AF1EE10FA02D2B0EEA4
:102B5000410A7047B4EEE00AF1EE10FAF9DDB0EE8A
:102B6000600A70470248022140680FF085BE0000ED
:102B7000C8010020044A13231221002010B500F0E0
:102B800097F9002010BD00001200002401214FF031
:102B9000FF3208200FF0AABE9FED010A7047000027
:102BA000000048430248012140680FF065BE000064
:102BB000C8010020044A06230221012010B500F0BC
:102BC00077F9002010BD00001900002401214FF00A
:102BD000FF3204200FF08ABE2DE9F04106000D46B9
:102BE0006FF0010726D02DB3434C207818B16FF059
:102BF0000200BDE8F0810FF0C5FE6060D0B1B622E2
:102C0000F5617E21002000F0BBF9B62214210120DD
:102C100000F0B6F91E2000F08BFA1E21002000F013
:102C200073F90021084600F06FF91E286FF00305C4
:102C300008D101E03846DCE70021012000F064F90A
:102C40000F2801D02846D4E74FF48065284600F0CD
:102C50009DFAAE00304600F099FA284A0121002082
:102C600000F0FAFA2649284600F0B4FA2549304621
:102C700000F0B0FAAA224021002000F081F90122E0
:102C80004121002000F07CF908225321002000F0AF
:102C900077F904225821002000F072F904227D21E6
:102CA000002000F06DF9322000F042FA01220F21DD
:102CB000104600F065F903221021012000F060F9B0
:102CC00000221621012000F05BF901221821104694
:102CD00000F056F980221521012000F051F90A2058
:102CE00000F026FA01202070284600F061FA3046F4
:102CF00000F05EFA00207CE7C8010020552E000895
:102D0000652B0008A52B00081EB5E8B324499FEDEC
:102D1000250AB1F80120ADF80020B1F80320ADF884
:102D20000420B1F80520ADF80820BDF90020BDF958
:102D3000043001EE902A01EE103ABDF90840F8EE99
:102D4000E11AB8EEC11A00EE904A81EE802AF8EE40
:102D5000E00AC1EE001A80ED002A80EE801AC0ED74
:102D6000011A80ED021A4A7C897CD20042EA511194
:102D7000B1F5806F01DBA1F5006100EE101AB4EE31
:102D8000001AF3EE070A00E007E0B8EEC00A40EED2
:102D9000010AC0ED060A00201EBD6FF001001EBD35
:102DA0001200002400A0AA451EB56FF00102E8B38E
:102DB0002549DFED260A9FED260AB1F80730ADF868
:102DC0000030B1F80930ADF80430B1F80B101BB287
:102DD000ADF80810BDF9001001EE903A02EE101A9D
:102DE000BDF90840F8EEE11AF8EEC22A01EE104AE9
:102DF00082EEA02AB8EEC11AC1EEA02AC1EE201AB6
:102E000062EE000A22EE801AC0ED030A80ED041A79
:102E100021EE800A80ED050AC169D1ED001A70EE3D
:102E2000E10AC0ED030AD1ED010A00E009E071EE0C
:102E3000600AC0ED040AD1ED020A30EE600A80EDAE
:102E4000050A10461EBD0000120000246F12034246
:102E500035FA8E3C70B5114D0121284604F090FCE6
:102E60000F4C40B901222846114604F08EFC6068E0
:102E700008210FF001FD0821284604F081FC0028FC
:102E80000AD101222846082104F07FFC6068042151
:102E9000BDE870400FF0F0BC70BD000000080258A3
:102EA000C801002001214FF0FF3203200FF01EBDAA
:102EB00070B514001E460D4621D0114B10B10128EB
:102EC00008D102E00022012101E000220821184679
:102ED00004F05BFC0B4945F080000870002000F016
:102EE000B3F908491423012208F023F8002000F068
:102EF000ABF932462146BDE8704007F01FBF70BDF8
:102F000000080258C901002070B50D460446012092
:102F100000F00EF9184E14B1012C08D102E0002285
:102F2000012101E000220821304604F02EFC45F08A
:102F30008000124D2870002000F086F914232946E5
:102F4000012207F0F6FF002000F07EF91423294645
:102F5000022207F0B9FD44B1012C05D1012230460F
:102F6000082104F012FC287870BD01223046114679
:102F700004F00BFC687870BD00080258C9010020FD
:102F800070B50446154801F07F01017042700120C0
:102F900000F0CEF8124D14B1012C08D102E000224D
:102FA000012101E000220821284604F0EEFB002068
:102FB00000F04AF909491423022207F0BAFF44B18C
:102FC000012C09D1012208212846BDE8704004F0F7
:102FD000DCBB01221146F7E770BD0000C9010020EB
:102FE0000008025810B52DED028BF0EE408AB0EECD
:102FF000608AF5EEC08AF1EE10FA09D9B5EEC08A02
:10300000F1EE10FA04D318EE100AB0F17E5F04DD81
:103010004FF0FF30BDEC028B10BD06F0A9FE134946
:1030200000EE100AD1E90030F8EE400A401C00EE34
:10303000100AB8EE400A20EE280A80EE801ABCEE94
:10304000C10A10EE100A0246401ED86200EE102A95
:10305000C8600968B8EE400A28EE000ABCEEC00A53
:1030600010EE100A88630020D4E7000090090020C9
:1030700010B504002DED028BB0EE408A04D0B5EE01
:10308000C08AF1EE10FA04D24FF0FF30BDEC028B93
:1030900010BD06F06DFE184900EE100AF6EE000AAB
:1030A000D1E90030B8EE401A401C604300EE100A2F
:1030B000B8EE400AC1EE001ABCEEE10A10EE100AAA
:1030C0000246401ED86200EE102AC8600968B8EEB9
:1030D000400A20EE200ABCEEC00A10EE100A8863F7
:1030E0009FED060A28EE000ABCEEC00A10EE100A98
:1030F00000F01EF80020C9E79009002000007A4483
:103100000448042110B508F0A9FB002801D04FF0B5
:10311000FF3010BD900900200448042110B508F0CC
:103120002FFC002801D04FF0FF3010BD9009002087
:1031300070B505460FF097FA4FF47A71B1FBF0F0D5
:10314000B5FBF0F40FF078FA02284FF0FF3110D001
:1031500005DC88420BD090B1012813D10FE0032881
:1031600005D0042803D06FF0004290420AD10846EF
:1031700070BD04B9012420460FF038FA02E0284659
:1031800003F012FE002070BD10F0D8B9B0F5806FCA
:1031900010B508D0B0F5805F05D0B0F5004F02D073
:1031A0004FF0FF3010BD282004F084FB002010BD3C
:1031B000B0F5806F10B508D0B0F5805F05D0B0F5E0
:1031C000004F02D04FF0FF3010BD282004F083FBE9
:1031D000002010BD10B549B10124002204FA02F309
:1031E000034206D0064840F8221006E06FF00100C6
:1031F00010BD521CD2B2102AF0D3002010BD000026
:10320000409B00200A460E4910B530B1012808D075
:1032100002280AD04FF0FF3010BD08464FF480411D
:1032200006E008464FF4005102E008464FF4004122
:10323000012A00D0002204F0A8FA002010BD0000EE
:10324000000802580FF0E4BF08B1002070470148A1
:10325000704700003407002032B1054B03EB4010EB
:1032600040F82120002070476FF0010070470000F7
:10327000809B002005280ED2DFE800F00305070B35
:1032800009000648704706487047064870470648D8
:10329000704706487047002070470000DC09002096
:1032A000980B00202C0C0020700A0020C00C00207D
:1032B00070B504460068C169C90617D510210162BE
:1032C00020460BF0C1FE0A4D00EBC00005EB80006C
:1032D000006A00280AD020460BF0B6FE00EBC000C2
:1032E00005EB8000006ABDE87040004770BD00003B
:1032F0008C9A002042B1064B00EBC00003EB80002B
:1033000040F82120002070476FF001007047000056
:103310008C9A00200FB4104840F2FF3170B505AB15
:10332000049AFDF795F905042D0C11D00A4E0024DE
:103330002946304600F04CF830B1641C0A20E4B253
:10334000FFF7F6FE032CF3D3002070BC5DF814FBEE
:103350006FF00100F9E70000209C002008490020E0
:1033600070B5084E0A88B35C002B08D000251846BB
:10337000541CA3B2B554802B0B8000D30D8070BDBC
:10338000A0010020A09B0020FEE700207047002045
:103390007047000005490022054810B50CF000FBFD
:1033A000044903480CF0EFFA002010BDB41E0020C1
:1033B000D8110020B41600200348012110B5006880
:1033C0000FF05AFA002010BDA40100200020704721
:1033D000094A10B5D2F8BC22D2F814220AB1012051
:1033E00010BD0A46014604480CF0DAFABDE8104068
:1033F00001480CF04BBB0000D811002008B10020A0
:1034000070474FF0FF3070474FF0FF3210B540B1BA
:1034100039B1427C3AB1027C2AB100F007F80020B1
:1034200010BD104610BD00200871F8E710B5447CAF
:103430000022B4B3012C35D00123022C0ED0032C72
:103440001AD106E0012B16D0022B14D0032B13D176
:1034500011E00B71037C002BF4D10CE004240C71FF
:10346000047C44B1012C06D0022C03D0032C03D1E0
:103470004B7101E003224A7190ED030A81ED030ACA
:1034800090ED020A81ED040A90ED000A81ED050A33
:1034900090ED050A81ED020A90ED010A81ED070A1F
:1034A00010BDFFE70A71D5E72DE9F04F04000D4686
:1034B0006FF001002DED0E8BDBB07CD0002D7AD0AB
:1034C0009FEDFE1A2068D4ED020A101A226000EE69
:1034D000100A2046F8EE401A81EE810A84ED010AB6
:1034E00070EE800AC4ED020A00F08CFE94F884129B
:1034F0004FF000099FEDF28AD1B101292ED00426A8
:1035000004F52F709FEDEF9AF2EE04BADFEDEE9A1C
:1035100004294FF0DC0AF1EE04DAB9EE04EAF6EE23
:10352000008AB0EE00AA00907DD0052915D12CE0CC
:10353000F02101A8FDF7B1F9E449F02201A8FDF757
:1035400050F9F02201A904F1A000FDF74AF984ED39
:10355000028A84F8849284F88592AFE25FF00005D5
:10356000DB49142205EB850004EB8000A030FDF759
:1035700038F96D1CEDB20C2DF2D3012184F88412C0
:1035800084F8859284ED028A98E20027D0491422BB
:1035900007EB8700143104EB8000A030FDF721F920
:1035A0007F1CFFB20C2FF1D3D4ED011AD4EDA30A86
:1035B000B0EE480A00E0FDE30098B0EE401A0AF0D1
:1035C00051FAD4EDA90A84EDA60AC24930EE800A68
:1035D00010EE100A84EDA90A884202DD9FEDBE0AB2
:1035E00006E010EE100ABD49884203D99FEDBC0ADF
:1035F00084EDA90A94F8850220B101281BD0032884
:1036000018D13CE100EB400200EB800104EB8202A8
:10361000401C92ED060A04EB8101C0B20C2881ED3A
:103620002A0AEFD300E04AE284F8846284F88592A3
:1036300084ED028A26E2D5ED010A94ED640AD4ED08
:10364000011A00EEA10A84ED640AB0EE480A00985F
:10365000D4EDA30AB0EE401A0AF004FA002604F1F1
:10366000B40B04F1780804F13C0700BF94EDA90AFB
:10367000B5EEC00AF1EE10FA50DD36B1012E27D0BA
:10368000022E28D0032E28D0DFE090483FABF03048
:1036900007C883E80700D4ED640A94EDA90A43AA99
:1036A000F1EE600A3FA830EEC00A8DED410AE168F4
:1036B00001F1DC03C43109F057F89DED430A84EDB4
:1036C0002A0A9DED440A84ED2F0A9DED450A4FE03C
:1036D0007E48FC3051E0834874E0824843AB0C30B4
:1036E00007C883E8070094EDA90AD4ED640A3FAA4D
:1036F00043A830EE600A8DED450AE16801F580735C
:10370000C43109F031F89DED3F0A84ED570A9DED73
:10371000400A8BED2F0A9DED410A94E036B1012E4F
:1037200029D0022E4CD0032E6DD08EE06D4843ABD5
:10373000183007C883E80700D4ED640A94EDA90A9D
:103740003FAAF1EE600A43A830EEC00A8DED450AAB
:10375000E16801F1DC03C43109F006F89DED3F0A90
:1037600084ED2A0A9DED400A84ED2F0A9DED410A61
:1037700084ED340A69E05B48243043AB07C883E832
:103780000700D4ED640A94EDA90A3FAAF1EE600A9D
:1037900043A830EEC00A8DED450AE16801F1E80367
:1037A000C43108F0E1FF9DED3F0A84ED390A9DED3B
:1037B000400A87ED2F0A9DED410A87ED340A44E067
:1037C000484830303FAB07C883E8070094EDA90AAA
:1037D000D4ED640A43AA3FA830EE600A8DED410A99
:1037E000E16801F1F403C43108F0BEFF9DED430A26
:1037F00084ED480A9DED440A88ED2F0A9DED450AA7
:1038000088ED340A21E037483FAB3C3007C883E8F5
:10381000070094EDA90AD4ED640A43AA3FA830EE4C
:10382000600A8DED410AE16801F58073C43108F04A
:103830009BFF9DED430A84ED570A9DED440A8BEDF5
:103840002F0A9DED450A8BED340A761CF6B2042E44
:10385000FFF40CAF95ED020AB5EEC00AF1EE10FAD6
:103860000DD195ED030AB5EEC00AF1EE10FA06D1BE
:1038700095ED040AB5EEC00AF1EE10FA7ED0D5ED52
:10388000010A94ED640A94ED011A00EE810A84EDB8
:10389000640A94ED020AB4EEC90AF1EE10FA03DDEF
:1038A00030EE490A84ED020A95ED020AD5ED030ACD
:1038B0004E4680EE2BBAC0EEABAA15E000007A446B
:1038C000000000009A99193F8FC2F53D004A010897
:1038D000E8010020CDCC4C3DCDCC4C3DCDCC4CBDF9
:1038E000CDCC4CBD084B01089FEDF90BDFEDFACABA
:1038F0009FEDFADAB7EECB1AB1EE4B2A4FF07C58B7
:103900005746B7EEC22A31EE401B32EE400BF7EEBF
:10391000C1BBB7EEC0CB1AE0CEB1032E17D029EE53
:10392000280A00BFD4ED020A30EE200AF0EE490A60
:103930000EF070F9C0EE090AF00700280CFE8D3A6F
:1039400095ED041A022E05D281EE2D0A04E0B0EEA8
:10395000480AE7E781EE0E0A10EE900A40454CDA7D
:1039600033EE6A2A8DED4ECA9FEDDD1B73EE2A2AD7
:1039700055A832EE402A32EE804A00E082E02BEE7B
:10398000280A60EE8A3A8DED4F2A94ED642AB7EE4C
:10399000C00AF1EE424ACDED504A51AB3FAA49A9C7
:1039A00031EE402B30EE010BB7EEC21BB7EEC00B71
:1039B0008DED491A8DED4A3AD4ED640A79EEE00AAC
:1039C000CDED4B0A8DED3F0A8DED403A94ED640A42
:1039D00039EEC00A8DED410ACDED51BA8DED524A56
:1039E00094ED640AB1EE400A8DED530AB0EE630A1D
:1039F00000904EA80AF040F924E033EE2A1A33EE84
:103A00006A2ACDED3FBA55AA71EE001A32EE401A7D
:103A100030EEE80ACDED401AD4ED640A49A920EE53
:103A20000A0AF1EE600ACDED410A8DED49CA8DED2D
:103A30004A1AD4ED640A3FA8F1EE600ACDED4B0AB4
:103A40000AF070F906EB4600E16843AA07EB800034
:103A50000B18C43155A808F087FEC6EB06109DED83
:103A6000430A04EB8000761C80ED2A0A9DED440A8F
:103A7000F6B280ED2F0A9DED450A042E80ED340A42
:103A8000FFF44AAF5FF00005D4ED011A05EB4500E5
:103A900005EB850104EB800004EB8106D0ED060AFE
:103AA000D4F8B80296ED2A0AB0EE481A09F0DAFF07
:103AB0006D1CEDB20C2D86ED280AE5D3D6E2002769
:103AC0008949142207EB870004EB8000A030FCF743
:103AD00088FE7F1CFFB20C2FF2D3844994ED640A58
:103AE000D5ED011A9FED821AD4ED010A01EEA00A6C
:103AF00084ED640A94EDA90AD5ED061A01EEA00A38
:103B000084EDA90A84EDAA8A95ED052AD4EDA81AB8
:103B100010EE100A42EE201A8842C4EDA81A02DD07
:103B200084EDA91A08E010EE100A7249884203D900
:103B30009FED710A84EDA90A94F8850240B1DFF87F
:103B4000A8B10128ABF11C0B19D0032816D159E1FB
:103B500000EB400200EB800104EB8202401C92ED7E
:103B6000060A04EB8101C0B20C2881ED2A0AEFD3CA
:103B700084F8846284F8859284ED028A5AE29BF884
:103B8000001021B1012961D002295ED1B8E084ED95
:103B9000028A8BED011AD846DFED58AA5FF00007C4
:103BA00007EBC70007EB470204EB800004EB82063B
:103BB00090ED060AF90786ED710A90ED090A86ED87
:103BC000720A90ED0C0A86ED730AC6ED95AAE068BC
:103BD00090ED310A01D1B1EE400A86ED960A94EDDE
:103BE000640A0AEB820206F51570B1EE400A86ED12
:103BF000970AE1688B18C4313DAA08F0B5FD9DED28
:103C00003D0AF80786ED950A9DED3E0A86ED960A77
:103C10009DED3F0A86ED970AC6ED65AAE06890ED36
:103C2000310A01D1B1EE400A86ED660A94ED640ACC
:103C30007F1CFFB2B1EE400A042F86ED670AAFD3B6
:103C400098F80010491C88F80010C6E05FF00006E4
:103C500094ED020ADBED010A06EB4600C0EE20AA55
:103C600004EB8007D7ED950A97ED710AB0EE6A1A5A
:103C70000AF053F8C6EB0610B0EE6A1A04EB80089F
:103C800088ED2A0AD7ED960A97ED720A0AF045F8F0
:103C900088ED2F0AD7ED970A97ED730AB0EE6A1AEE
:103CA0000AF03BF8761CF6B2042E88ED340ACFD326
:103CB00094ED020ADBED010A5846B4EEE00AF1EE9B
:103CC00010FA03DB0178491C8BF8001085E0000036
:103CD000B81E85EB51B88E3F3255B0BD3255B03D60
:103CE000B81E85EB51B88EBFFC010020CDCC4C3EF8
:103CF000CDCC4C3ECDCC4CBECDCC4CBE8FC275BCD9
:103D0000F0EE601A0098D4EDA30A94EDA90AB0EE83
:103D1000481A09F0A7FEB0EE401A0098F0EE41AA4A
:103D2000D4ED011AD4EDA40A94EDAA0AB0EE481A13
:103D300009F098FE94ED641AD4EDA60A00265746C1
:103D40007AEEC11AB1EE412A32EE6A1A31EEC02A79
:103D500071EE802A71EE401A31EE000A32EE602ACE
:103D600072EEE02A31EEA01A30EE200A84ED6D2AC0
:103D7000C4ED702A84ED671A84ED6A0A06EB4601E9
:103D800042AA04EB810090ED650A8DED3F0A90EDAB
:103D9000660A8DED400A90ED670A07EB81008DED14
:103DA000410AE1680B18C4313FA808F0DDFCC6EBFE
:103DB000061000E087E19DED420A04EB8000761CCE
:103DC00080ED2A0A9DED430AF6B280ED2F0A9DEDA3
:103DD000440A042E80ED340AD0D395ED020AB5EEE4
:103DE000C00AF1EE10FA0DD195ED030AB5EEC00A46
:103DF000F1EE10FA06D195ED040AB5EEC00AF1EE27
:103E000010FA7DD094F88502032831D10098D4EDC2
:103E1000011AD4EDA30A94EDA90AB0EE481A09F0EC
:103E200021FEF0EE400A0098F0EE60AAD4ED011AEF
:103E3000D4EDA40A94EDAA0AB0EE481A09F012FED5
:103E400094ED641A3AEEC12AF1EE411A71EEEA0AD3
:103E500032EE401A72EE001A30EEC02A30EE800ABE
:103E600084ED6D1AC4ED701A84ED672A84ED6A0A38
:103E70008BED019A94ED020A5F46B4EEC90AF1EEA9
:103E800010FA03DD30EE490A84ED020A95ED020ACC
:103E9000D5ED030A4E46D04680EE2B9A4FF07C5962
:103EA000C0EEABAA19E0C6B1032E16D097ED010AF9
:103EB00060EE280A94ED020A30EE800AD7ED010A7E
:103EC0000DF0A8FED7ED010A022E80EE201A95ED26
:103ED000040A05D2C0EE2D0A04E0F0EE480AE9E734
:103EE000C0EE0E0A11EE100A484506EB460052DA03
:103EF00004EB800053A990ED650A70EE491A00E0CA
:103F000098E021EE0A0ACDED3F1A90ED661A50AB0B
:103F10004DAA31EE6A1A31EE601A8DED401A90ED1D
:103F2000671A8DED411A90ED651A09EE681A8DED4C
:103F30004A1A90ED661A8DED4B1A90ED671A31EE24
:103F4000291A8DED4C1A90ED651A09EE281A8DED9F
:103F50004D1A90ED661A8DED4E1A90ED671A31EEFE
:103F6000291A8DED4F1A90ED651A31EE091A8DED73
:103F7000501A90ED661A31EE2A1A71EE200ACDED34
:103F8000510AD0ED670A3FA8CDED520A00914AA927
:103F900009F072FE2EE004EB800031EE680A90ED2D
:103FA000651A53AA4AA931EE091A20EE0A0A8DEDC4
:103FB0003D1A90ED661A31EE2A1A31EE201A8DED77
:103FC0003E1A90ED671A8DED3F1A90ED651A31EEAD
:103FD000491A8DED4A1A90ED661A31EE6A1A71EEA1
:103FE000600ACDED4B0AD0ED670A3DA8CDED4C0A35
:103FF00009F098FE06EB4600E16843AA08EB800052
:104000000B18C43153A808F0AFFBC6EB06109DEDAA
:10401000430A04EB8000761C80ED2A0A9DED440AD9
:10402000F6B280ED2F0A9DED450A042E80ED340A8C
:10403000FFF439AF5FF00005D4ED011A05EB450040
:1040400005EB850104EB800004EB8106D0ED060A48
:10405000D4F8B80296ED2A0AB0EE481A09F002FD2B
:104060006D1CEDB20C2D86ED280AE5D334264FF0F9
:10407000940864279FED168A002500BFE06806EBD0
:10408000850C07EB85038444034408EB850105EBAD
:104090004502084404EB820105EB85029CED002AF1
:1040A00090ED001A91ED060A04EB820000F1A001E8
:1040B000A830D3ED001A62EE080A08F02DFC6D1C42
:1040C000EDB20C2DDAD35BB0BDEC0E8BBDE8F08FFA
:1040D0000AD7A33C2DE9F04105000E461ED0002E64
:1040E0001CD004274FF034085FF00004E86807EBA9
:1040F000840308EB840204EB84010344024405EBCF
:104100008100A030D3ED000A92ED000A06EB810198
:1041100008F0C8FB641CE4B20C2CE7D3BDE8F081C6
:1041200070B504006FF001052DED028BB0EE408AF2
:1041300056D00020E160DFED320A84F884024FF4AB
:104140003470C4ED640AFFF77DF8C4F8B802E8B330
:104150004FF4C0763046FFF775F8C4F8F802A8B3FC
:104160003046FFF76FF8C4F8FC0278B35FF0000543
:10417000D4F8B802E268C5EB0511B0EE480A00EBCE
:104180008100002102F5867209F020FDE168D4F873
:10419000F802B0EE480AD1ED530A00EB451008F0E2
:1041A00029FCE168D4F8FC02B0EE480AD1ED540ACB
:1041B00000EB451008F01EFC6D1CEDB20C2DD7D3A2
:1041C0000021B0EE480A04F52F7000E00AE0E26832
:1041D00002F5967209F0FAFC0020BDEC028B70BD6E
:1041E0002846FAE7D4F8B80204F52E74FEF7CCFF9F
:1041F000206CFEF7C9FF606CFEF7C6FFF0E7000019
:10420000AE47613E70B504006FF001002DED028BEA
:104210000CD000290AD094F884220878824208D170
:1042200094F885224B789A4203D10020BDEC028B92
:1042300070BD1F4B002204289FED1C8A1A7084F861
:104240008402487884F8850284ED028A84EDA98A84
:1042500084EDAA8A94EDA20A84EDA80A03D09FED0A
:10426000150A84ED640A0025D4F8B802C5EB0511DF
:1042700000EB810009F0EAFCD4F8F802B0EE480A3D
:1042800000EB451008F01CFCD4F8FC02B0EE480A24
:1042900000EB451008F014FC6D1CEDB20C2DE3D3BF
:1042A00004F52F7009F0D2FCBFE700000000000009
:1042B000E0010020AE47613E2DE9F04104270E46A3
:1042C000002405464FF0340807EB8403E86808EB48
:1042D000840204EB44010344024405EB81001030E6
:1042E000D3ED000A92ED000A06EB810108F0C4FA52
:1042F000641CE4B20C2CE7D3BDE8F0816FF001023E
:1043000068B161B191ED000A80EDA20A91ED010A58
:1043100080EDA30A91ED020A80EDA40A70471046D1
:104320007047B5EEC01AF1EE10FA30EE600A0ADD01
:10433000F6EE000A61EE200AB4EEE00AF1EE10FAA1
:1043400002DD30EE410A7047F1EE600AB4EEE00A99
:10435000F1EE10FAF7D230EE010A7047002804D0CF
:1043600002494FF4B472FCF73CBA704710020020C7
:10437000014801F079BE0000F8030020014801F077
:1043800073BE0000540D0020014801F06DBE000016
:10439000BC070020014801F067BE0000340800207F
:1043A000014801F061BE0000AC0F0020014801F09F
:1043B0005BBE000024100020014801F055BE000043
:1043C000BC0E0020014801F04FBE0000340F002059
:1043D000014801F049BE00009C100020014801F096
:1043E00043BE0000CC0D0020014801F03DBE00009E
:1043F000440E0020014801F037BE000014110020D7
:10440000294A016891423AD0274A1832914236D05F
:10441000254A3032914232D0234A483291422ED03E
:10442000214A603291422AD01F4A7832914226D0E6
:104430001D4A9032914222D01B4AA83291421ED08E
:104440001A4A91421BD0194A1832914217D0174A82
:104450003032914213D0154A483291420FD0134A5C
:10446000603291420BD0114A7832914207D00F4A04
:104470009032914203D00D4AA832914211D1CAB272
:104480001823103AB2FBF3F26FF30901032A02F08A
:104490000703074AD25CC26500D9091D8165084639
:1044A000704721F0FF01F9E71000024010040240BC
:1044B0005449010830B5224A012301689142CAB229
:1044C0001BD01F4C1434A14217D01D4C2834A142DC
:1044D00013D01B4C3C34A1420FD0194C5034A14294
:1044E0000BD0174C6434A14207D0154C7834A1424C
:1044F00003D0134C8C34A1420CD11421114C083A36
:10450000B2FBF1F10F4A803201F01F0504EB81018B
:10451000AB4010E00C4D1824103A0D44B2FBF4F1FE
:10452000A82D00D80831094A01F01F0402EB8101CF
:10453000064AA3408032603080E80E0030BD0000A3
:104540000854025800580258F0FBFDBF0008024012
:1045500010B50279531E072B2DD8174C0168A142C4
:104560001BD0154C1434A14217D0134C2834A1424F
:1045700013D0114C3C34A1420FD00F4C5034A14207
:104580000BD00D4C6434A14207D00B4C7834A142BF
:1045900003D0094C8C34A14203D10849074C443163
:1045A00002E00749064C443104EB8202C0E91B21BA
:1045B00001219940416710BD08540258FC58025827
:1045C000FC08024010B583694FF0C074826A01464E
:1045D000002053B1B3F5005F15D072B1012A0CD0A1
:1045E000022A0AD0032A09D104E01AB1012A06D00E
:1045F000022A03D1C96AC90100D5012010BDC96AC8
:10460000A142FAD010BD002AF7D0012AF2D0022A26
:10461000F3D0032AF3D010BD2DE9F04F804E804F28
:10462000DFF8FC911836DFF8F8A148370468856D8B
:104630000AF1300ADFF8ECB14C45DFF8ECC1DFF8E5
:10464000ECE16DD0B4426BD0544569D0BC4267D028
:10465000DFF8D081A8F11808444561D05C455FD0EF
:1046600064455DD074455BD0DFF8C481444557D0C4
:10467000DFF8BC8108F11808444551D0DFF8B0815B
:1046800008F1300844454BD0DFF8A48108F1480810
:10469000444545D0DFF8988108F1600844453FD093
:1046A000DFF88C8108F17808444539D0DFF8808143
:1046B00008F19008444533D0DFF8748108F1A80868
:1046C00044452DD0DFF86C81444529D0DFF8648162
:1046D00008F11408444523D0DFF8588108F1280870
:1046E00044451DD0DFF84C8108F13C08444517D003
:1046F000DFF8408108F15008444511D0DFF83481DB
:1047000008F1640844450BD0DFF8288108F17808E7
:10471000444505D0DFF81C8108F18C08444509D1D7
:10472000D0E91948C4F80480C46E1CB1D0E91C4813
:10473000C4F8048004684C452ED0B4422CD05445B3
:104740002AD0BC4228D0374E183EB44224D05C4513
:1047500022D0644520D074451ED0354EB4421BD0C3
:10476000334E1836B44217D0314E3036B44213D0DF
:104770002F4E4836B4420FD02D4E6036B4420BD087
:104780002B4E7836B44207D0294E9036B44203D02F
:10479000274EA836B44215D190F85C603F2406F04D
:1047A0001F06B440AC600468256825F480252560A8
:1047B0002EE09A600068C160BDE8F08F99600068E3
:1047C000C260F9E71B4EB4421BD01A4E1436B442F5
:1047D00017D0184E2836B44213D0164E3C36B44289
:1047E0000FD0144E5036B4420BD0124E6436B44241
:1047F00007D0104E7836B44203D00E4E8C36B442F9
:10480000DAD190F85C60012406F01F06B4406C60B9
:10481000046863608368402B0368CFD1C9E7000058
:104820001000024088000240A0000240B800024090
:10483000100402400854025800F0AEB810B520B180
:104840001621FCF708F8002010BD6FF0010010BD24
:1048500070B56FF00105B8B10C4C207810B16FF055
:10486000020070BD0EF08EF8606068B1084A032146
:104870000020FEF73FFD074A04210020FEF73AFD25
:1048800001202070002070BD284670BDC0010020AE
:10489000C14900083948000810B504001ED012496B
:1048A00000F0B3F821884FF4A560A1F5B6718142FC
:1048B00017D86188A1F5B671814212D8A188A1F5F7
:1048C000B67181420DD8E188A1F5B671814208D850
:1048D000207A30B1607A20B1002010BD6FF0010065
:1048E00010BD4FF0FF3010BD00000024F0B3E9B35D
:1048F0000288DFED270A01EE902AB0EE001A9FED44
:10490000250AF8EE611A71EEE01A61EE811A81EE65
:10491000802A81ED002A428801EE902AF8EE611A81
:1049200071EEE01A61EE811A81EE802A81ED012A92
:10493000828801EE902AF8EE611A71EEE01A61EEBB
:10494000811A81EE802A81ED022AC28801EE902A26
:10495000F8EE611A71EEE01A21EE811AC1EE001A2A
:10496000C1ED031A427A0A74027A00E00DE04A743B
:10497000808A01EE100A0020B8EE411A71EE600A3A
:1049800080EE801A81ED051A70476FF001007047C4
:10499000000080440000A544002010B5FEF76AFC2A
:1049A0000068016821F0010101600020FEF762FC4F
:1049B0000068016841F001010160002010BD0000A5
:1049C0000248202140680DF057BF0000C0010020C0
:1049D000002010B5FEF74EFC0449122207F0D0FD6E
:1049E000002801D04FF0FF3010BD0000000000246F
:1049F00001210246202010B50DF078FF202801D0BB
:104A0000002010BD012010BD7047002810B535D022
:104A1000002933D00A88C2F30A0202804A788B78D0
:104A2000D20842EA4312C2F30A0242808A78CB7863
:104A30000C79920942EA830242EA8422C2F30A0212
:104A400082800A794B79520842EAC312C2F30A0201
:104A5000C2804A79C2F3011242724A799209027203
:104A6000CA8842810A8982814A89C2810A7B02748A
:104A70004A7B4274CA894282098A818210BD4FF4FE
:104A8000806010B502F062FD4FF4805002F05EFDD0
:104A9000BDE810404FF4004002F058BD72B6FEE78A
:104AA000054805490839026842F0020202600868B8
:104AB0008004FCD5704700000C480258014802F001
:104AC00089B9000070040020014802F083B9000099
:104AD00070040020014802F07DB90000100500209C
:104AE000014802F077B9000010050020014802F0EB
:104AF00071B90000B0050020014802F06BB9000058
:104B0000B0050020F0B503684FF6FC716D4C426BA8
:104B1000D3F884508D4345EA8205C3F88450036876
:104B200053F8845F068F25F47F0545EA06451D602E
:104B3000836B654D9F180268D2F888308B4343EA37
:104B40008703C2F88830026852F8883F868F23F4C2
:104B5000FE0343EA06431360066856F8A03FC26BA3
:104B60008B4307EB420243EA82033360076857F83E
:104B7000A03FB0F8406023F4FE0343EA06433B60E5
:104B8000D0E9103603FB06220368D3F8B0608E43E9
:104B900046EA8206C3F8B0600368B0F84860D3F80C
:104BA000B07027F4FE0747EA0646C3F8B060D0E9C4
:104BB0001267036806FB0722D3F8AC608E4346EA0F
:104BC0008206C3F8AC60D0E91467036806FB0722CD
:104BD000D3F8F0608E4346EA8206C3F8F0600368BB
:104BE000B0F85860D3F8F07027F47C1747EA06460F
:104BF000C3F8F0600368876D53F8C06F02EB47029B
:104C00008E4346EA820119600168B0F85C20D1F851
:104C1000C03023F47C1343EA0242C1F8C02001688B
:104C200090F86020D1F8C03023F07C5343EA026250
:104C3000C1F8C020416B04EB8101C166826B01EBBE
:104C400082020267C36B02EBC3024267D0E91034F1
:104C5000634302EB83028267D0E91234634302EBC1
:104C60008302C267D0E91434634302EB8302C0F8C5
:104C70008020836D02EBC303C0F88430C46D826E64
:104C8000544303EB8403C0F88830046E544303EBB1
:104C90008402C0F89020AA420AD9D0F89C200321AF
:104CA00042F02002C0F89C2080F898100120F0BD4E
:104CB000002200E004C1D0F890308B42FAD80020E6
:104CC000F0BD000000AC0040FCD30040004870473D
:104CD00020A000202DE9F0472F4C054601269146E3
:104CE0008A464FF000086068A0BB04F10C0010E099
:104CF000006807683846FBF7C5FC0246A85C202818
:104D000000D020B939462846FBF7DBFC28B16068A3
:104D1000406860600028EBD134E0D4F804C0DCF8CF
:104D2000000090F90C70002F10DB0020294602468D
:104D300003E0202B18D00022491C0B78002BF8D15F
:104D40000AB1401E40B2B84200D00026BCF1000FAC
:104D500018D07EB160682A4649460068836850468C
:104D6000984706000BD013E0002AE5D10122401C31
:104D700040B2E1E709494A465046FBF7B5FDC4F8A1
:104D8000048005E006494A465046FBF7ADFD002683
:104D90003046BDE8F0870000AC010020A8500108B3
:104DA0000051010870B5050011D008200EF030FA4E
:104DB000040014D00EF08EFB0D480021C4E9005110
:104DC00001684C6004600EF0A5FB012070BD50200E
:104DD00080F31188BFF34F8FBFF36F8FFEE7502032
:104DE00080F31188BFF34F8FBFF36F8FFEE7000092
:104DF000AC01002070B504006FF0010006D000295E
:104E000004D00B4D287810B16FF0020070BD204621
:104E1000C4F8E0144FF40471FBF73FFD4FF4347114
:104E200004F50470FBF739FD01202870002070BDE7
:104E3000D00100202DE9F041060025D02A48007855
:104E400030B301275FF0000404EB440000EBC40022
:104E500006EB800526F8204028466F800DF0E8FA22
:104E6000032C02D3A01F032815D2D6F8E004007843
:104E7000FEF700FA0123112205F1180107F0CCFB1F
:104E8000D6F8E004007814E06FF00100BDE8F0818E
:104E90006FF00200FAE7D6F8E0044078FEF7EAF98E
:104EA0000123112205F1180107F0B6FBD6F8E00442
:104EB0004078FEF7DFF9C4EB0411012306EB810112
:104EC000102201F50F7107F0E7FAC4EB041006EBAE
:104ED000800000F504700DF005FA641CE4B20C2C9F
:104EE000B2D30020D2E70000D001002030B56FF02F
:104EF000010228B321B30022551C02EB820302EB0E
:104F0000420401EB830304EBC20293ED030A00EBBE
:104F10008204EAB284ED040A93ED040A0C2A84EDBB
:104F2000050A93ED020A84ED030A93ED010A84ED6C
:104F3000020A93ED000A84ED010ADDD3002030BDA2
:104F4000104630BD6FF0010210B5D8B1D1B10022CA
:104F5000C2EB021402EB420300EB840401EB830377
:104F600094ED890A521C83ED020A94ED880AD2B2AC
:104F700083ED010A94ED870A0C2A83ED000AE7D33A
:104F8000002010BD104610BD2DE9F0470F4690F8E7
:104F90005C109CB0044601294FF0000915D0002692
:104FA000DFF8F880012084F85C00189619962168D3
:104FB00041450ED13A4D0095284607F09DFC8246AA
:104FC000206807F099FC60B10EE002201CB0BDE83B
:104FD000F087206E84F85C6040F02000206601209D
:104FE000F4E7BAF1000F09D0216E4FF0010941F04A
:104FF00020002066484684F85C60E7E72068414668
:10500000884201D0A84201D1264800E0264840F657
:105010001F72D7F800C0254BBCF1000F23D0D0F889
:1050200008C0D7F804802CF4404C4CEA080CC0F8B7
:1050300008C0D4F800C08C4501D0AC4507D18968C0
:10504000AB6801F0010103F00103194302E0996824
:1050500001F001010029CDD1BD6839688368294379
:105060009343194317E0876827F440478760276810
:105070008F4201D0AF4207D18968AB6801F00101CE
:1050800003F00103194302E0996801F001010029CE
:10509000B0D1816891438160ACE7000000200240FC
:1050A00000210240002302400063025800600258C1
:1050B0002DE9F84F0446DFF8ECB30020FA4E0090DB
:1050C000814694F85C000D46F84F012808D04FF057
:1050D000010A84F85CA0206807F00AFC18B18FE28E
:1050E0000220BDE8F88F286800280FDB2168B14254
:1050F0000CD0CA69030327D090FAA0F0B0FA80F070
:1051000000F01F030AFA03F00243CA61D5E9001256
:105110004FF00C0C20681F23C1F384610CEA921C31
:1051200002F01F02604493409140026B9A430A438D
:105130000263206807F0DCFB8046206807F0D4FBA0
:1051400058EA000003D054E1C0F38460D8E729682E
:105150004FF0040C20680723AA680CEAD15CC1F365
:10516000045160448B408A40416999431143416135
:105170002068B04204D1C2686969C2F3C1020BE081
:10518000CB4A1268BAEB127F02D0C168C90605D4B7
:10519000C2686969C2F38202520004E0C2686969A8
:1051A00002F01002520891402A69042A5AD02B6852
:1051B00000EB8202B04202F1600207D103F0F84036
:1051C0001368084340F00040106008E0D2F800C0C7
:1051D00003F0F84008430CF00041014311602068DF
:1051E000B0421CD12969EA6900EB8100016E21F00F
:1051F00080711143016695F8201020682A69012901
:105200000AD00021B0429ED100EB8200026E22F053
:1052100000720A430266ECE04FF00071F2E795F885
:1052200021102A69012917D05FF0000100EB8200EC
:10523000026E22F000420A430266297E20682A6933
:1052400001290CD00021036902F01F02914023F4D0
:10525000F0420A430261CCE04FF00041E6E74FF430
:105260000061F0E7B04273D1002107F037FB000383
:1052700020684FF000016DD007F030FB90FAA0F0ED
:10528000B0FA80F12868020369D090FAA0F0B0FA71
:1052900080F0814204D100222068114607F030FBE3
:1052A0002068012107F01AFB000320684FF001017C
:1052B00058D007F013FB90FAA0F0B0FA80F12868FC
:1052C000020354D090FAA0F0B0FA80F0814204D1E9
:1052D00020680022012107F013FB2068022107F05B
:1052E000FDFA000320684FF0020143D007F0F6FA00
:1052F00090FAA0F0B0FA80F1286802033FD090FA4B
:10530000A0F0B0FA80F0814204D12068002202218E
:1053100007F0F6FA2068032107F0E0FA000320689E
:105320004FF003012ED007F0D9FA90FAA0F0B0FAAE
:1053300080F1286802032AD090FAA0F0B0FA80F039
:10534000814256D120680022032107F0D9FA50E0AB
:1053500020E0FFE707F0C2FAC0F3846192E7C0F3F0
:10536000846096E707F0BAFAC0F38461A7E7C0F358
:105370008460ABE707F0B2FAC0F38461BCE7C0F326
:105380008460C0E707F0AAFAC0F38461D1E7C0F3F4
:105390008460D5E7016E2A7801F0F841B1EB826FA5
:1053A00003D1016E21F00041016620682978426E28
:1053B00002F0F842B2EB816F03D1416E21F000415F
:1053C000416620682978826E02F0F842B2EB816F64
:1053D00003D1816E21F00041816620682978C26E78
:1053E00002F0F842B2EB816F03D1C16E21F00041AF
:1053F000C1662068816811F0010F52D12D4AB04278
:10540000EB6829680FD1D0F8B0C003F01808C1F3D9
:10541000130322FA08F20A402CEA030C4CEA020CAD
:10542000C0F8B0C00EE0D0F8C0C003F01808C1F357
:10543000130322FA08F20A402CEA030C4CEA020C8D
:10544000C0F8C0C0E968594570D11B482268DFF830
:105450006CC0DFF86CB08242DFF868E01A481B4B82
:10546000DFF86C8043D12968614565D0B1EB4C0C05
:105470006DD0714569D0A1F1865CBCF1100C75D07E
:10548000DFF850C061456DD0DFF84CC061457FD07A
:10549000814273D0994247D01048814222D11048AE
:1054A00076E0B3E00000FF470060025800210240B0
:1054B0000010005CFFFF0F000020024002003004DB
:1054C000400020190800900C0008302E00106032B7
:1054D000002090362000F0140004002A0000214330
:1054E000000052476E48814251D16E4850E0BA42A6
:1054F0001DD1296861451FD0A1F1066CBCF1040CD7
:1055000025D0714521D0A1F1865CBCF1100C2DD0C5
:10551000DFF894C1614525D0DFF890C1614537D0EF
:1055200081422BD09942DDD1404631E040E0B24289
:105530002DD12968614501D1012029E0A1F1066C36
:10554000BCF1040C03D0714503D1594820E0584602
:105550001EE0A1F1865CBCF1100C07D0DFF848C159
:10556000614505D1534813E000E007E052480FE0E1
:10557000DFF838C161450BD0814201D1184607E000
:105580004E48414504D0814201D14D4800E0002001
:10559000B2420DD0D16903031AD090FAA0F0B0FA4C
:1055A00080F000BF00F01F030AFA03F00143D1614D
:1055B000D5F800C0BCF1000F28DA424B2068424900
:1055C000DFF808A1984201D0B84203D10A4602E0B0
:1055D000800EE7E752469268984202F0E07201D0EE
:1055E000B84209D19D68D7F8088005F0010508F098
:1055F000010845EA080502E0B56805F0010555B166
:10560000216E4FF0010941F020002066002084F84F
:105610005C00484665E52E4DAC451CD115021AD4F8
:10562000B042F3D1984202D0B84200D051468B68C4
:1056300042F4000023F0E07202438A6026492548C4
:105640000968B1FBF0F04000801C00E0401E0090B3
:105650000028FBD1DAE7214DAC450CD1D5010AD4A5
:10566000B042D3D1984202D0B84200D051468B68A4
:1056700042F080700EE01A4DAC45C7D15502C5D43A
:10568000B042C3D1984202D0B84200D051468B6894
:1056900042F4800023F0E07202438A60B6E7000023
:1056A0000000844B0000B84F2000F0140004002AD2
:1056B0008000501D0002B025000180210040C03A4A
:1056C0000080F03E002002400023024000630258A8
:1056D000000052C7400D030088000020000021C3D5
:1056E000000084CB2DE9F8434FF0000504002E465E
:1056F000009502D0206E18B108E00120BDE8F883C3
:10570000204600F043F9656684F85C5020688168A3
:10571000C1F3407119B181688E4A114081602068DF
:105720008168C1F3007181B981688B4A114041F0F1
:10573000805181608A4989480968B1FBF0F0401CBA
:1057400000E0401E00900028FBD120688168C1F372
:10575000007141B9216E012641F010012166616E90
:1057600041F00101616607F0C3F8216EC90600D45B
:1057700020B1206E012640F01000E0E0206E20F401
:10578000807040F00200206620688168754D11F03D
:10579000010F1ED1744B754A984201D0904207D137
:1057A0009968976801F0010107F00107394302E0A9
:1057B000A96801F0010161B9984201D0904201D17C
:1057C0006B4800E06B488268616822F47C120A43EF
:1057D00082602168A9421FD1637ED4E90207E26B8F
:1057E0005B033A43082805D00C280FD01C280FD0A3
:1057F00018280FD05FF0000000F00C0794F820008C
:1058000043EA47031A4342EA00400FE00420F3E76B
:105810000820F1E71C20EFE7627E94F82030A768AB
:10582000E06B520342EA03423843104394F82020CD
:10583000012A04D1A28C504B03EB42421043A26ACE
:105840002AB1E36A02F47872024343EA0200CA68AA
:10585000A9420BD1494B1A400243CA602068626BCF
:10586000016921F040611143016103E0444B1A409A
:105870000243CA60206807F03BF80746206807F03B
:1058800033F807434ED12068A946484506D1217E0A
:1058900094F83820890341EA420103E0227E216B1B
:1058A00041EA8231C26844F203039A430A43C26068
:1058B00094F844000128206803D0016921F0010117
:1058C00022E048450ED1D4E9121CD4E9143502690E
:1058D0002C4F41EA0C012B433A401943114341F04C
:1058E000010111E0D4E91317B4F848C0DFF898803B
:1058F000636D026908EB0C4C224D394343EA0C03FB
:105900006D1E2A401943114301612068236C02690E
:1059100022F070421A4302612068484502D02046B6
:10592000FCF748FC2069012820680BD0016B21F0AE
:105930000F010163206E20F0020040F0010020669C
:105940003046DBE6E269016B521E21F00F01114384
:10595000EFE70000C0FFFF5FC0FFFF7F400D0300C7
:105960008800002000600258002002400021024010
:1059700000230240006302580000FEFF0740F0FFD2
:1059800003C0F0FF1FF800FC0100FFFFF0B5B5B049
:10599000064614212EA8FAF780FFB8216846FAF7C8
:1059A0007CFF3149306888425BD1022000224FF4ED
:1059B00000210091CDE901201024154606AACDE969
:1059C0000340C023059082E8290068460995289580
:1059D00003F0B2FB08B1FFF761F82448016841F019
:1059E00020010160006800F0200033901F4808305B
:1059F000016841F001010160016801F0010133918A
:105A0000016841F004010160006803272EA9309568
:105A100000F0040033902020CDE92E07144801F057
:105A2000A1FD14482EA9CDE92E47309501F09AFD2D
:105A3000114C092111484FF4807C021584E82300A1
:105A4000D700C4E90352C3142046C4E907C5656200
:105A5000C4E9053700F07CFE08B1FFF71FF8B46514
:105A6000A66335B0F0BD000000200240D8440258C3
:105A70000000025800080258F803002010000240FD
:105A80002DE9F84F044601F085FE00903CB194F8F2
:105A90003500022806D0802161650020E4E0012065
:105AA000BDE8F88FC74DC74EC64918352068303657
:105AB000DFF81483DFF814938842DFF814A3DFF8CB
:105AC00014B32ED0A8422CD0B0422AD0404528D0C2
:105AD000484526D0504524D0584522D0BD4A1832DA
:105AE00090421ED0BC4A90421BD0BB4A1832904212
:105AF00017D0B94A3032904213D0B74A4832904258
:105B00000FD0B54A603290420BD0B34A78329042FF
:105B100007D0B14A9032904203D0AF4AA8329042A7
:105B200009D1026822F01E0202602068426922F058
:105B30008002426103E0026822F00E0202602768E0
:105B40008F4238464DD0A8424BD0B04249D0404554
:105B500047D0484545D0504543D0584541D09D4A4F
:105B6000183290423DD09C4A90423AD09A4A18321C
:105B7000904236D0984A3032904232D0964A4832DB
:105B800090422ED0944A603290422AD0924A783283
:105B9000904226D0904A9032904222D08E4AA8322B
:105BA00090421ED08D4A90421BD08C4A14329042B3
:105BB00017D08A4A2832904213D0884A3C32904209
:105BC0000FD0864A503290420BD0844A64329042C1
:105BD00007D0824A7832904203D0804A8C32974272
:105BE00004D1206E026822F4807202607549206838
:105BF000884228D0A84226D0B04224D0404522D0A6
:105C0000484520D050451ED058451CD07149183108
:105C1000884218D07049884215D06F49183188429F
:105C200011D06D49303188420DD06B4948318842DE
:105C300009D069496031884205D067497831884286
:105C400001D065499031016821F0010101600EE049
:105C500001F0A0FD0099401A052808D920226265AC
:105C60000321002084F8351084F8340017E73868E1
:105C7000C007EDD1534A0121206890422ED0A8429E
:105C80002CD0B0422AD0404528D0484526D0504597
:105C900024D0584522D04F4B183398421ED04E4B3B
:105CA00098421BD04C4B1833984217D04A4B303394
:105CB000984213D0484B483398420FD0464B60333C
:105CC00098420BD0444B7833984207D0424B9033E4
:105CD000984203D0404BA833984208D194F85C70A6
:105CE0003F23A06D07F01F07BB40836007E094F8D7
:105CF0005C30A06D03F01F0301FA03F343602068DA
:105D000090424DD0A8424BD0B04249D0404547D0F8
:105D1000484545D0504543D0584541D02D4A1832CA
:105D200090423DD02C4A90423AD02B4A18329042B1
:105D300036D0294A3032904232D0274A48329042F7
:105D40002ED0254A603290422AD0234A783290429F
:105D500026D0214A9032904222D01F4AA832904247
:105D60001ED01E4A90421BD01C4A1432904217D0BB
:105D70001A4A2832904213D0184A3C3290420FD02F
:105D8000164A503290420BD0144A6432904207D0E7
:105D9000124A7832904203D0104A8C3290420BD192
:105DA000D4E919024260E06E30B1026822F48072D8
:105DB0000260D4E91C024260002084F8351084F8A7
:105DC00034006DE6100002405800024070000240AE
:105DD00088000240A000024010040240085402580B
:105DE0002DE9F05F28B190F83510022904D0802108
:105DF00041650120BDE8F09F904C904B0168183C34
:105E000018338E4ADFF83C92A1428D4CDFF838E21D
:105E10008E4FDFF83CB2DFF83CA28F4D8F4E31D071
:105E200091422FD099422DD0A1422BD0494529D063
:105E3000714527D0B94225D0DFF810C20CF1180CFB
:105E400061451FD0DFF808C2ACF1600C614519D084
:105E5000DFF8FCC1ACF1480C614513D0DFF8F0C1AC
:105E6000ACF1300C61450DD0DFF8E4C1ACF1180C99
:105E7000614507D0594505D0514503D0A94201D00D
:105E8000B1422CD1DFF8B4C14FF0040880F835805E
:105E9000ACF1180C61451DD091421BD0994219D02C
:105EA000A14217D0494515D0714513D0B94211D040
:105EB0006648183081420DD065486038814209D06B
:105EC00063484838814205D061483038814201D06A
:105ED0005F481838086820F001000860ABE0D1F88E
:105EE00000C02CF00E08DFF854C1C1F80080ACF1FE
:105EF000180C0168614527D0914225D0994223D0E2
:105F0000A14221D049451FD071451DD0B9421BD0B7
:105F1000DFF838C10CF1180C614515D0DFF830C13D
:105F2000ACF1600C61450FD0DFF824C1ACF1480C36
:105F3000614509D0DFF818C1ACF1300C614503D0E0
:105F4000DFF80CC1ACF1180CD1F800C02CF0010C3A
:105F5000C1F800C0DFF8E4804FF0010C0168A8F13F
:105F60001808414546D0914244D0994242D0A142BE
:105F700040D049453ED071453CD0B9423AD0334A31
:105F80001832914236D0324A603A914232D0304A89
:105F9000483A91422ED02E4A303A91422AD02C4A89
:105FA000183A914226D0594524D0514522D0A942D1
:105FB00020D0B1421ED02A4A91421BD0284A143226
:105FC000914217D0264A2832914213D0244A3C32BB
:105FD00091420FD0224A503291420BD0204A643273
:105FE000914207D01E4A7832914203D01C4A8C322B
:105FF000914218D1016E0A6822F480720A6090F80A
:106000005C20816D02F01F020CFA02F24A60D0E9B6
:1060100019124A60C16E31B10A6822F480720A60B6
:10602000D0E91C124A600022016D80F835C080F86A
:10603000342001B188470020DCE60000280002403F
:10604000580002407000024088000240A000024058
:106050007004024088040240A0040240B8040240D8
:1060600008540258406D70472DE9FC5F0446F74E16
:106070000020DFF8D88300904FF41652F44808F15E
:106080001808A56DDFF8C493DFF8C0A3016809F113
:10609000300920680AF1480AB1FBF2F1B0420191DF
:1060A0002F68D5F800C0DFF8ACB335D04146884240
:1060B00032D0484530D050452ED058452CD0E549F7
:1060C0001831884228D0E3493031884224D0E14950
:1060D0004831884220D0E04988421DD0DE4918313D
:1060E000884219D0DC493031884215D0DA4948312C
:1060F000884211D0DFF860E30EF1600E70450BD0DE
:10610000D54A7832904207D0D34B9033984203D08F
:10611000D149A83188427DD194F85C20082102F051
:106120001F0201FA02F23A424AD0B04232D0404550
:1061300030D048452ED050452CD058452AD0C54A9D
:106140001832904226D0C34A3032904222D0C14AFF
:10615000483290421ED0C04A90421BD0BE4A1832EC
:10616000904217D0BC4A3032904213D0BA4A4832DB
:1061700090420FD0B84A603290420BD0B64A783283
:10618000904207D0B44A9032904203D0B24AA8322B
:10619000904203D1026802F0040202E0026802F0B9
:1061A00008026AB1026822F00402026094F85C00FE
:1061B00000F01F008140A960606D40F00100606543
:1061C00094F85C00012100F01F008140394240D06A
:1061D0002068B04234D0404532D0484530D0504598
:1061E0002ED058452CD09B4A1832904228D0994A3C
:1061F0003032904224D0974A4832904220D0964A7A
:1062000090421DD0944A1832904219D0924A3032AE
:10621000904200E0AFE113D08F4A483290420FD055
:106220008D4A603290420BD08B4A7832904207D030
:10623000894A9032904203D0874AA83290427DD159
:10624000406910F0800F04D0A960606D40F002003A
:10625000606594F85C00042100F01F008140394221
:106260003ED02068B04232D0404530D048452ED094
:1062700050452CD058452AD0764A1832904226D024
:10628000744A3032904222D0724A483290421ED034
:10629000714A90421BD0704A1832904217D06E4A11
:1062A0003032904213D06C4A483290420FD06A4A42
:1062B000603290420BD0684A7832904207D0664AEA
:1062C0009032904203D0644AA83290424ED1006886
:1062D00010F0020F04D0A960606D40F0040060650A
:1062E00094F85C00102100F01F008140394258D022
:1062F0002068B04234D0404532D0484530D0504577
:106300002ED058452CD0534A1832904228D0514AAA
:106310003032904224D04F4A4832904220D04E4AE8
:1063200090421DD04C4A1832904219D04A4A30321D
:10633000904215D0484A4832904200E014E00FD015
:10634000454A603290420BD0434A7832904207D09F
:10635000414A9032904203D03F4AA832904207D13E
:10636000006800F0080006E0006872E70068B7E720
:10637000006800F00400A0B1A9602068016849032A
:1063800004D50068000308D5A16C07E00168C905C1
:1063900003D4016821F008010160216C09B1204695
:1063A000884794F85C00202100F01F0081403942AA
:1063B00079D02068B04232D0404530D048452ED008
:1063C00050452CD058452AD0224A1832904226D027
:1063D000204A3032904222D01E4A483290421ED08B
:1063E0001D4A90421BD01C4A1832904217D01A4ABC
:1063F0003032904213D0184A483290420FD0164A99
:10640000603290420BD0144A7832904207D0124A40
:106410009032904203D0104AA832904203D10068D3
:1064200000F0100002E0006800F00200B0B3A960C4
:1064300094F835000428206801680FD049037ED500
:10644000006800032BD4616C2AE0000010000240B9
:1064500088000020700002401004024021F0160164
:1064600001602068416921F080014161206C08B918
:10647000A06C20B12068016821F00801016094F847
:106480005C303F21012003F01F0300229940A960E6
:1064900084F8350084F83420216D65E003E0E16B79
:1064A00009B120468847606D00287DD0606DC00727
:1064B00059D02068042184F83510B0422BD04045D3
:1064C00029D0484527D0504525D0584523D09D494F
:1064D000884220D09B49183188421CD099493031DC
:1064E000884218D09849884215D097491831884277
:1064F00011D09549303188420DD0934948318842B6
:1065000009D091496031884205D08F49783188425D
:1065100001D08D499031016821F0010101602068AE
:106520000099019A491C0091914202D80168C9075B
:10653000F6D10068C00710D003200FE0FFE7016824
:10654000C905ACD403680121002223F010030360C5
:1065500084F8351084F83420A1E7012084F8350050
:10656000002084F83400E16C00291DD002B02046E0
:10657000BDE8F05F0847754988421DD07349143162
:10658000884219D071492831884215D06F493C3171
:10659000884211D06D49503188420DD06B49643129
:1065A000884209D0694900E084E07831884203D00C
:1065B00066498C3188427DD194F85C80042701685B
:1065C00008F01F0807FA08F717EA0C0F009746D0E3
:1065D0004F0744D500980F04686003D5C8033CD426
:1065E000A16CC1E7880638D42068B0422DD0554947
:1065F0006039884229D0484527D0504525D0584594
:1066000023D05049884220D04E49183188421CD0AE
:106610004C493031884218D04B49884215D04A49FC
:106620001831884211D04849303188420DD046494E
:106630004831884209D0704507D0904205D0984231
:1066400003D04149A831884203D1016821F00801F3
:1066500002E0016821F004010160216C84E7022757
:1066600007FA08F717EA0C0F00974ED08F074CD5A2
:1066700000980F04686003D5C80344D4616C73E7C5
:10668000880640D42068B0422FD02E496039884215
:106690002BD0484529D0504527D0584525D02949E9
:1066A000884222D02749183188421ED025493031EE
:1066B000884200E044E018D02349884215D022499E
:1066C0001831884211D02049303188420DD01E49FE
:1066D0004831884209D0704507D0904205D0984291
:1066E00003D01949A831884203D1016821F014016F
:1066F00002E0016821F00A010160012184F83510EF
:10670000002084F83400E16B2EE7082202FA08F238
:1067100012EA0C0F14D0090712D5016821F00E01FE
:10672000016094F85C100120002201F01F0100FAC2
:1067300001F16960606584F8350084F8342012E75F
:10674000BDE8FC9F88000240100402400854025833
:106750002DE9F05F044601F01DF8002C07467DD0BE
:10676000E24E022120684FF00308DFF884934FF0D7
:106770000005DFF880A3B042DFF87CB334D0DB4AF9
:106780001832904230D048452ED050452CD0584534
:106790002AD0D94A1832904226D0D74A3032904275
:1067A00022D0D54A483290421ED0D44A90421BD0C3
:1067B000D24A1832904217D0D04A3032904213D089
:1067C000CE4A483290420FD0CC4A603290420BD031
:1067D000CA4A7832904207D0C84A9032904203D0D9
:1067E000C64AA83290427DD184F83510B04284F870
:1067F00034502ED0BD49183188422AD0484528D07F
:10680000504526D0584524D0BB491831884220D065
:10681000B949303188421CD0B7494831884218D034
:10682000B649884215D0B5491831884211D0B349CC
:10683000303188420DD0B1494831884209D0AF4942
:106840006031884205D0AD497831884201D0AB49EA
:106850009031016821F00101016008E025E100BFED
:1068600000F098FFC01B052801D920211AE12068FB
:106870000068C007F4D1D4E902032168103418433A
:106880008E4694E88410D4E9033809683A431043EB
:106890009B4A40EA0C00676918431140103C40EAEB
:1068A0000800042F40EA010003D1D4E90B12114380
:1068B00008436168A1F12902052A0BD9163A032A77
:1068C00008D9083A012A05D9083A032A02D97439A5
:1068D000032901D840F48010CEF800002068676AD0
:1068E000406900E020E0042F20F0070047EA00079D
:1068F0000DD1D4E90A01074349B12046FDF762FEF4
:1069000028B140206065012184F83510CDE0206871
:1069100047612046FDF774FD94F85C203F2102F0AA
:106920001F029140816055E0764A90421BD0754B22
:106930001433984217D0734B2833984213D0714BBD
:106940003C3398420FD06F4B503398420BD06D4B75
:106950006433984207D06B4B7833984203D0694B2D
:106960008C3398427ED184F8351084F83450664BCD
:106970000168A26801EA030E402A74D0802A73D00D
:106980005FF00002D4E90378D4E9053142EAD70286
:1069900042EAD8085B4AD4E9077C48EAD30848EAC7
:1069A000D10141EAD701524241EA1C11142341EAC4
:1069B0000E01016020681044B0FBF3F08000E06538
:1069C0002046FDF71DFD94F85C20012102F01F0216
:1069D000914041602068B04257D044491831884204
:1069E00053D0484551D050454FD058454DD04249DD
:1069F0001831884249D040493031884245D03E491B
:106A00004831884241D03D4988423ED03B49183107
:106A100088423AD039493031884236D037494831F6
:106A2000884232D03549603188422ED0334978319E
:106A300088422AD031499031884226D02F49A83146
:106A4000884222D02F4988421FD02E4914318842D3
:106A50001BD02C492831884217D02A493C31884222
:106A600013D002E01DE017E018E0264950318842BB
:106A70000BD024496431884207D0224978318842BA
:106A800003D020498C31884229D12046FDF712FDE0
:106A9000A06880280CD00CE0102273E74FF48042ED
:106AA00070E74021616584F835800120BDE8F09FE2
:106AB0006560216E20790860D4E919014160606841
:106AC000401E072808D82046FDF742FDE06E05600D
:106AD000D4E91C01416002E0E56625676567012095
:106AE000656584F835000020E0E7000010000240F2
:106AF0004000024058000240700002401004024072
:106B00003F8010FE085402580F00FEFF2DE9F84F99
:106B100004008C464FF00000009014D094F834002C
:106B2000012812D094F835500120002184F8340057
:106B3000012D0CD0C00260650120009084F8341053
:106B40000098BDE8F88F0120FBE70220F9E78C4DA3
:106B50000226206884F83560A8428A4D61658A4E15
:106B60008A4FDFF82C82DFF82C92DFF82CA2DFF8B6
:106B70002CB226D0A84224D0B04222D0B84220D095
:106B800040451ED048451CD050451AD0584518D015
:106B90008349884215D082491831884211D08049F2
:106BA000303188420DD07E494831884209D07C4935
:106BB0006031884205D07A497831884201D07849DD
:106BC0009031016821F00101016061462046FDF726
:106BD00023FD6B49206888422CD0A8422AD0B042BD
:106BE00028D0B84226D0404524D0484522D0504530
:106BF00020D058451ED06A4A90421BD0684A1832AD
:106C0000904217D0664A3032904213D0644A4832DC
:106C100090420FD0624A603290420BD0604A783284
:106C2000904207D05E4A9032904203D05C4AA8322C
:106C300090420CD1026822F01E0242F0160202605D
:106C4000206C88B12068026842F008020BE00268FC
:106C500022F00E0242F00A020260206C20B120688D
:106C6000026842F004020260206888424BD0A842C9
:106C700049D0B04247D0B84245D0404543D04845BE
:106C800041D050453FD058453DD0454A90423AD03A
:106C9000434A1832904236D0414A3032904232D084
:106CA0003F4A483290422ED03D4A603290422AD02C
:106CB0003B4A7832904226D0394A9032904222D0D4
:106CC000374AA83290421ED0364A90421BD0354AED
:106CD0001432904217D0334A2832904213D0314AAE
:106CE0003C3290420FD02F4A503290420BD02D4A66
:106CF0006432904207D02B4A7832904203D0294A1E
:106D00008C3290420DD1206E0268D20303D5026806
:106D100042F480720260E06E18B1026842F4807240
:106D200002602068884226D0A84224D0B04222D0F7
:106D3000B84220D040451ED048451CD050451AD0FE
:106D4000584518D01649884215D01549183188423F
:106D500011D01349303188420DD011494831884251
:106D600009D00F496031884205D00D4978318842F9
:106D700001D00B499031016841F001010160DFE66B
:106D8000100002402800024040000240580002402B
:106D90007000024088000240A0000240B80002409B
:106DA000100402400854025870B5044600F0F2FC8A
:106DB0000546601C02D004480078044400F0EAFC58
:106DC000401BA042FAD370BD7C0000207047704782
:106DD000704770472DE9FF5FDFF80CB304460BF1F5
:106DE0000401DBF8000025680F68AA468007D5F883
:106DF0005090696DD5F850806E6D2A6DD5F854C0ED
:106E00002B6D00EA8770009009F470496F6D286D52
:106E100001EA09010191DAF85410DAF85490DAF82D
:106E2000505008F00F0806EA0806029602F0F00239
:106E300003F071536FEA09061F4000F060700CEA1E
:106E4000020CCDF80CC0F20501EA00090CD4E843AD
:106E5000C00509D400214FF48073CAF85030CBF834
:106E600000102046FFF7B5FF700512D4E843400537
:106E70000FD4206800234FF48068D0F8DC20D0F8CD
:106E8000E410C0F85080CBF800301140204600F0EC
:106E900042FBDFF858A2009850B12268830F00EA45
:106EA0000A001065CBF8003020460099FFF78EFFEE
:106EB000019850B12268830F00EA0A001065CBF8F0
:106EC00000302046019900F028FB029850B122685A
:106ED000830F00EA0A001065CBF8003020460299C3
:106EE00000F011FB039850B12268830F00EA0A00FA
:106EF0001065CBF800302046039900F005FB300503
:106F00000CD4E843000509D4236800204FF4006244
:106F10001A65CBF80000204600F000FBB00512D443
:106F2000E84380050FD4206800234FF40078D0F8A0
:106F3000D820D0F8E010C0F85080CBF800301140D5
:106F4000204600F0E9FA30030CD4E843000309D4EA
:106F5000236800204FF400221A65CBF80000204679
:106F600000F0D0FAF0030CD4E843C00309D423683E
:106F700000204FF480321A65CBF80000204600F064
:106F8000C9FA70030CD4E843400309D422680020F6
:106F90004FF480231365CBF80000204600F0B9FAC7
:106FA000B0030FD4E84380030CD4236800204FF4CF
:106FB00000321A65CBF80000D4F89C0040F0800045
:106FC000C4F89C00B9F1000F0BD022684FEA997306
:106FD00009EA0A001065CBF8003049462046FFF761
:106FE000F7FE5FB12268BB0F07EA0A001065CBF815
:106FF0000030D4F89C003843C4F89C003C49206819
:10700000884268D1606881468068800763D0D9F87B
:107010002060D9F82410D9F82080D9F82400D9F8B4
:1070200020C0D9F82470D9F82030D9F82450D9F8E4
:10703000202003F4FC4306F00F0AD9F824601D4019
:10704000D9F824B008F030080CF4C07C02F4F02227
:1070500011EA0A0100EA080807EA0C0706EA020634
:10706000D9F820A004D0C9F82010204600F04EFA2C
:10707000B8F1000005D0616808624146204600F082
:1070800047FA6FEA0B0040060ED46FEA0A0040068A
:107090000AD460684021C36BC26B01622046190CA0
:1070A00002F03F0200F033FA2FB160680762394600
:1070B000204600F02AFA35B160680562D4F89C00D9
:1070C0002843C4F89C0036B160680662D4F89C007E
:1070D0003043C4F89C00D4F89C00002802D020461D
:1070E000FFF775FEBDE8FF9F10A80040FFFFCF3FF0
:1070F00000A000402DE9F04194B08D494C22044697
:107100006846F9F76EFB64B18A4D2068A84202D147
:1071100000F58070606094F898004FF0000820B18E
:1071200008E0012014B0BDE8F081204684F8998081
:1071300000F002F92068816921F01001816100F0FE
:1071400029FB0327064604E000F024FB801B0A28E5
:1071500011D8206880690007F6D42068816941F061
:107160000101816100F016FB06460DE000F012FB04
:10717000801B0A2808D9D4F89C0040F00100C4F80C
:107180009C0084F89870CCE720688069C007EDD037
:107190002068816941F002018161207C012820681A
:1071A000816937D041F040018161607C012820680D
:1071B000816932D021F480418161A07C012820685E
:1071C00081692DD041F4805181612068A268816974
:1071D00021F44071114381612068816921F0A4018B
:1071E00081612068016921F010010161E0680128D6
:1071F00019D010B302281BD02068816941F08001AA
:1072000081612068016941F010010161E068032893
:107210000ED012E021F04001C6E741F48041CBE7F7
:1072200021F48051D0E72068816941F0040103E036
:107230002068816941F020018161207E6FF0FF02AA
:10724000D4E90773A68A1102400602EB0727A0F1D2
:107250000070384327685B1E184301EB0646304335
:10726000F861A068B0F5407F11D104F12800A68C28
:107270006FF00F0C89C801EB0641401E02EB0322A0
:10728000104322680CEB071318430843D060206EAC
:1072900030B12068626ED0F8C0101143C0F8C01041
:1072A000D4E917126846D14209D02168A36E51F87B
:1072B000C82F50F8233022F007021A430A60216CCD
:1072C00049B12168626C51F8BC3F50F8226023F04C
:1072D000070232430A60A16C51B12168E36C51F896
:1072E000BC2F50F8233022F0700242EA03120A60E9
:1072F000216D51B12168626D51F8BC3F50F82200F8
:1073000023F4E06242EA002008602068A84204D129
:107310006068816821F003018160C4F894800121D4
:10732000C4F89C8084F898102046FDF7EBFBF9E642
:107330006C49010800A000402DE9F047B4B0814637
:1073400014212EA8F9F7A9FAB8216846F9F7A5FA89
:10735000664C0026D9F800004FF08051644A0C3C7E
:10736000614F4FF00208614D9042DFF888A14FF065
:10737000090938D100201B914A13CDE90020684645
:1073800001F0DAFE08B1FDF789FB3868401C38606F
:10739000012807D1286840F480702860286800F42C
:1073A00080703390206840F008002060206803223D
:1073B0002E922EA900F00800CDE92F863196CDE956
:1073C0003290504600F0CEF800220521132000F044
:1073D0008FFA132000F07FFA00220521152000F01B
:1073E00087FA15203BE0444A90423DD100201B9192
:1073F0004FF40042CDE90020684601F09DFE08B13F
:10740000FDF74CFB3868401C3860012807D128681C
:1074100040F480702860286800F480703390206801
:1074200040F002002060206860222E922EA900F019
:107430000200CDE92F863196CDE932902F4800F039
:1074400091F800220521142000F052FA142000F0D7
:1074500042FA00220521162000F04AFA162000F018
:107460003AFA34B0BDE8F087254A9042F9D10020BD
:107470001B914FF40042CDE90020684601F05CFE0C
:1074800008B1FDF70BFB3868401C3860012807D1B4
:10749000286840F480702860286800F48070339079
:1074A000206840F00800206020684FF440512E9181
:1074B000052200F00800CDE92F862EA93196CDE9EE
:1074C0003220504600F04EF8002205219F2000F0A7
:1074D0000FFA9F2000F0FFF900220521A02000F004
:1074E00007FAA020BBE7000004000020EC4402588B
:1074F00000A00040000C025800A400400004025804
:1075000000D400407047704770477047704770471D
:10751000704770477047704770477047704700006A
:107520002DE9F041084F01250024064605FA04F034
:10753000304203D057F8240000B18047641CE4B205
:10754000102CF3D3BDE8F081409B00204FF0B041F8
:1075500010B5D1F88820024203D0C1F88800FFF7A7
:10756000DFFF10BD2DE9F84F03247A4D00234FF0C3
:1075700001094FF0B04B4FF00F0AE4E009FA03F6AF
:10758000324078D00F7907F00307012F01D0022F86
:107590001AD187684FEA430ED1F80CC004FA0EF8EE
:1075A00027EA08070CFA0EFC4CEA070CC0F808C0E2
:1075B000476891F804C0B743CCF3001C0CFA03FCF5
:1075C0004CEA070CC0F804C00E79F643B6070BD09E
:1075D000C6684FEA43088F6804FA08FC26EA0C06DE
:1075E00007FA08F73743C7600E7906F00306022E44
:1075F00012D1DE080F694FEA437C00EB8606B646DF
:10760000366A4FEADC6C0AFA0CF807FA0CF726EA3D
:1076100008063743CEF820700F7906684FEA430812
:1076200007F0030704FA08FC07FA08F726EA0C0635
:10763000374307604E6816F4403F1CD0464E37680B
:1076400047F00207376036689F0706F0020600968B
:1076500023F0030606F1B046B6463F0FD6F808649D
:10766000DFF8F8800AFA07FC404526EA0C0603D149
:107670004FF0000C3AE065E0DFF8E4C0604502D16D
:107680004FF0010C32E0DFF8DCC0604502D14FF072
:10769000020C2BE0DFF8D0C0604502D14FF0030CA4
:1076A00024E0DFF8C8C0604502D14FF0040C1DE0B3
:1076B000DFF8BCC0604502D14FF0050C16E0DFF8E2
:1076C000B4C0604502D14FF0060C0FE0DFF8A8C04F
:1076D000604502D14FF0070C08E0DFF8A0C060451C
:1076E00002D14FF0090C01E04FF00A0C0CFA07FC34
:1076F0004CEA060CCEF808C44F68DBF80060FF02C5
:1077000026EA020600D516435F46CBF80060D1F8A2
:1077100004C0DBF804605FEA8C2C26EA020600D580
:1077200016437E606E684F6826EA0206BF0300D5E6
:1077300016436E602E684F6826EA0206FF0300D5E6
:1077400016432E605B1C0A6832FA03F67FF416AF0C
:10775000BDE8F88F80000058F44402580000025839
:107760000004025800080258000C02580010025889
:107770000014025800180258001C02580024025835
:107780000069084000D0012070470AB1816170474C
:107790000904FBE701488068704700007C00002076
:1077A0000248816802781144816070477C000020A3
:1077B000032010B500F0BCF802F0FEFA0F4A1049A1
:1077C00014681368C4F3032203F00F038A5CC95CD6
:1077D00002F01F0201F01F01D0400A4A20FA01F115
:1077E0001160094908600F2000F010F808B101206D
:1077F00010BD00F04DF8002010BD000018440258E4
:10780000E04901088C0000208800002010B51028F5
:1078100004468AB02AD200220146A12000F068F86E
:10782000A12000F058F8154804601548016841F09F
:1078300080710160006808A900F0807009906846B6
:1078400002F046FA02F0A6FA0E49400000220E4C61
:10785000B0FBF1F10D4840F2E7330460C0E90332B8
:10786000491EC0E9011203F06BFD10B101200AB0FE
:1078700010BD064803F096FDF9E7000080000020E7
:10788000EC44025840420F0000E000408C11002000
:10789000074882B0016841F00201016000680022DF
:1078A0000F2100F002000090901E02B000F020B8FE
:1078B000F444025800280DDB410900F01F02890042
:1078C000012001F1E0219040C1F88001BFF34F8F0A
:1078D000BFF36F8F7047002809DB410900F01F02DA
:1078E0008900012001F1E0219040C1F800017047BA
:1078F0000E4BF0B41B680D46C3F30223C3F1070619
:10790000042E00D90426191D072901D2002300E006
:10791000DB1E012404FA06F19C40491E2940641E26
:10792000994014402143F0BC09F02BBC0CED00E061
:10793000064900F0070210B54FF6FF040868044B33
:10794000204040EA02201843086010BD0CED00E022
:107950000000FA052DE9F04F02688346FF484FF01A
:10796000000A8DB00C468242564602D10025012005
:1079700001E001250020E8460027814607EB47018A
:107980007F1C08EBC101F8B205F01CFF20B10820F4
:107990004FF0010ACBF85400FFB2022FEED3BAF138
:1079A000000F7CD1DFF8B4E3DEF80000C00707D099
:1079B000DEF8001046F0010621F00101CEF80010BB
:1079C000E7480068C00706D0E54846F002060168AF
:1079D00021F00101016005EB45030C93E1484246AB
:1079E00008EBC303DFF880B30121DC469F6800EB9E
:1079F0008707D7F8008428F48078C7F80084DBF87C
:107A00000070FF0732D0DCF80070B9F1010F27F0E9
:107A10000107CCF800705CD1069B00EB8303D3F820
:107A2000007447F00207C3F80074079B3BB100EBFA
:107A30008303D3F8007447F02007C3F80074099B50
:107A40004BB121EA030700EB8703D3F8047447F432
:107A50008027C3F804740A9BDBB321EA030700EB19
:107A60008703D3F8047447F0806730E00C9F52F826
:107A7000377077B300EB8707D7F800C42CF0010C00
:107A8000C7F800C45F683FB100EB8707D7F800C4B0
:107A90002CF0100CC7F800C4D3F80CC000E05AE179
:107AA000BCF1000F09D021EA0C0700EB8707D7F8DB
:107AB00004C42CF4803CC7F804C41B694BB121EA10
:107AC000030700EB8703D3F8047427F08077C3F82B
:107AD000047409EB4903D4F800C0CDF830C09146D6
:107AE00052F83370BC451BD009EBC302D4F808C070
:107AF000D2F80880C44513D0D4F804C0D2F804806A
:107B0000C44502D1BCF1000F0AD1D4F80CC0D2F8A0
:107B10000C80C44504D0D4F810C01269944551D1EA
:107B20000C9ABA4219D109EBC302D4F804C0D2F8B6
:107B30000480C44511D1D4F80CC0D2F80C80C445DF
:107B40000BD1D4F810C01269944506D1DBF800308F
:107B500043F00103CBF8003034E000EB870709EB7A
:107B6000C302D7F8003423F00103C7F80034536888
:107B70003BB100EB8303D3F8007427F01007C3F880
:107B80000074936800EB8303D3F8007427F48077C4
:107B9000C3F80074D3684BB121EA030700EB8703F5
:107BA000D3F8047427F48037C3F8047412694AB117
:107BB00021EA020300EB8302D2F8043423F080733D
:107BC000C2F80434A3685A4600EB8303D3F8007468
:107BD00027F4407747EA452747F48077C3F80074D5
:107BE000DBF800C063695F1ECCF3074C674508D91A
:107BF0005E4FD2F800C007EB03472CF47F033B43F2
:107C000013601268D207226800EB8202D2F80034B7
:107C10003FD023F003035B1CC2F8003462684AB112
:107C200000EB8202D2F8003423F0300343F010035B
:107C3000C2F80034E268D3030AD521EA020300EB5C
:107C40008302D2F8043423F4E02343F480330AE0BF
:107C50005AB121EA020300EB8302D2F8043423F084
:107C6000E06343F08073C2F804342269D30307D57C
:107C7000914300EB8100D0F8041421F4E0214AE0A4
:107C8000F2B3914300EB8100D0F8041421F0E061DD
:107C90004EE001EB450723F003033B43C2F80034F9
:107CA00062685AB100EB8202D2F8003423F030034C
:107CB00043EA451343F01003C2F80034E268D303EB
:107CC0000CD521EA020300EB8302D2F8043423F43A
:107CD000E02343EA854343F480330CE06AB121EAB0
:107CE000020300EB8302D2F8043423F0E06343EA9A
:107CF000856343F08073C2F804342269D30300E043
:107D00001AE00BD5914300EB8100D0F8041421F464
:107D1000E02141EA854141F440310BE062B19143F9
:107D200000EB8100D0F8041421F0E06141EA8561A4
:107D300041F04071C0F80414F00705D0DEF80010DF
:107D400041F00101CEF80010B00704D504480168E5
:107D500041F0010101600DB0504609E000500052B1
:107D600000A0005200B0005200B400520000FFFF1B
:107D7000BDE8F08FF8B500250446FFF70BFD064679
:107D800024B100206065206D10B170E001256EE027
:107D9000204600F073F841F28830A065258A6FF024
:107DA000FF012268D4F814C00F02636B07EB05458E
:107DB000E06801EB0C27D4F81CC0184393683D43DE
:107DC0002D4F28433B4040EA0C0018439060206848
:107DD000236AC26822F4E0221A43C2602368228E1A
:107DE000A06B40EA024018612268E06B5061D4E960
:107DF0000003026801EB032322F4F85119430160E8
:107E0000A06D0022202133460090204605F048FD59
:107E100005002CD12068626AC168521E21F0FF0162
:107E20001143C1602068A268016821F0400111433C
:107E300001602068D4E90A12D0F80831114323F018
:107E4000A0421143C0F808112068016841F0010107
:107E50000160A069022804D12068816841F0020114
:107E60008160E068B0F1806F03D002202065284671
:107E7000F8BD0120FAE70000F4F8E0F82DE9F0433E
:107E8000B5B0044614216846F8F707FDB82106A8E6
:107E9000F8F703FD4749206888427DD100201990FA
:107EA0004FF000710446CDE9061006A801F044F930
:107EB00008B1FCF7F3FD4048016841F4001101608E
:107EC000016801F400110591016841F4002101608D
:107ED000006800F40020059037480C30016841F03C
:107EE00001010160016801F001010591016841F0A3
:107EF00002010160016801F002010591016841F091
:107F000010010160016801F010010591016841F064
:107F100008010160006802250927009500F00800AB
:107F2000DFF89880032603966946CDE90470CDE911
:107F300001544046FFF716FB062102940820CDE9C4
:107F40000361CDE9000569464046FFF70BFB0121BF
:107F5000DFF86C9002AA4FF00408CDE900156946DD
:107F6000484682E85001FFF7FDFA02AA69464846F2
:107F700082E8D000CDE90085FFF7F4FA0B21114823
:107F80004FF40068CDF80080CDE90361CDE90154DC
:107F90006946FFF7E7FA00E008E002AA0A486946E6
:107FA00082E8D000CDE90085FFF7DCFA35B0BDE806
:107FB000F083000000A00052D44402580000025890
:107FC0000004025800100258000C025801680123F6
:107FD000C0F8D834002280F8CC248869044A40F0E4
:107FE00000608861486D10434865002070470000BC
:107FF0000300001070470068416200207047F0B530
:1080000003685D6A39B19F6A4C1E00204FF4827686
:1080100005EB17450BE045EA0240986210E0471C6B
:1080200006EB800053F800C0F8B205EB1C45A042F7
:10803000F5D34FF4807000EB810045EA02421A50FC
:108040000020F0BDD0F8E00407F0B5BF01EBC1029D
:1080500000EB8202D0F8E004126A07F008BF01EBDF
:10806000C10200EB8202D0F8E004D2F8602207F0EF
:108070005ABFD0F8E00407F0A0BF0A0601F00F01D4
:1080800001EBC10100EB810101D5143101E001F5E3
:108090001571006808F08EBE01F00F020B0670B576
:1080A00002EBC20104464FF001004FF0000504EB63
:1080B000810102D54875143103E081F8555201F56C
:1080C00015710A7094F89424012A08D084F8940455
:1080D000206808F08DFB002084F8945470BD0220C5
:1080E00070BD70B50279044601F00F00904201D9CD
:1080F000012070BD01F00F024FF000050B0602EBEE
:10810000C2014FF0010204EB810102D54A7514311E
:1081100003E081F8555201F515718D70087094F8DF
:108120009404012808D084F89424206808F0CAFC3C
:10813000002084F8945470BD022070BD01F00F013E
:1081400001EBC10100EB8100D0F8680270472DE916
:10815000F04101F00F0604460D064FF0010006EB5A
:10816000C6014FF0000504EB810102D548751431BA
:1081700003E081F8555201F51571C2F30A024F78F8
:108180000B718A600E7007B14E83022B00D14D71C6
:1081900094F89424012A09D084F89404206808F003
:1081A0006FFA284684F89454BDE8F0810220FBE77A
:1081B00070B501F00F05002405EBC50100EB81014E
:1081C00001F5187181E81C0001F80B4C01F80C5DF9
:1081D0008379012B00D1CA618279006808F0CAFC5A
:1081E000002070BD70B50D460179044605F00F0002
:1081F000884201D9012070BD29064FF000064FF0DA
:10820000010206D500EBC00104EB81014A7514316F
:1082100007E005EBC50104EB810181F8556201F52A
:1082200015718A70087094F89404012807D084F8B6
:108230009424206808F072FC280702D007E002208E
:1082400070BDA17904F29C42206808F00FFC002068
:1082500084F8946470BD70B501F00F04002504EB40
:10826000C401012600EB8101203181E82C0001F8D6
:108270000B6C01F80C4D8379012B00D1CA61827916
:10828000006808F077FC002070BD00002DE9FC5F5D
:1082900005680446284608F029FE00287ED120689B
:1082A00008F050FE002879D0D5F80808C0F30D205A
:1082B000C4F8D404206808F045FE800704D520687F
:1082C000416901F002014161206808F03BFEC106EE
:1082D00004F29C40009035D52068816921F010019E
:1082E00081612F6A07F00F01C7F3434001EBC10121
:1082F000022804EB810606F5157602D0062812D076
:108300001BE047F6F070074217D0C7F30A12F16876
:108310001746284608F01AFE7169F0683944716101
:108320003844F06009E000990822284608F00EFE63
:108330007069C7F30A11084470612068816941F0CF
:1083400010018161206808F0FDFD00034FF0080B6B
:108350004FF0000A4FF001097CD52068002608F094
:10836000D0FD074674E0F80770D02068F1B208F03D
:10837000E1FD8046C00707D005EB4611C1F8089B18
:108380003146204605F0B6FA5FEA087024D505EBC1
:108390004611C1F808BBFA49206800E03EE2026CD1
:1083A00000EB461001928A42D0F8081B05D9090457
:1083B00003D54FF40041C0F8081B204600F001FB34
:1083C000EF490198884207D9A079012804D1206893
:1083D0000121009A08F04AFB5FEAC86004D505EB6A
:1083E00046111020C1F8080B5FEA88701DD5686936
:1083F000000605D5D5F8040840F48061C5F80418D6
:1084000006EBC60004EB800090F8571200F51570DB
:10841000012905D180F803A02046F1B200F004FA4A
:1084200005EB46110220C1F8080B5FEA886004D50D
:1084300005EB46112020C1F8080B5FEA884005D5FE
:1084400005EB46114FF40050C1F8080B7F08761C6D
:10845000002F88D1206808F075FD40036ED5206894
:1084600008F048FD0026074666E0F80762D020685D
:10847000F1B208F04DFD8046C00723D0D5F834286E
:1084800006F00F0C05EB461309FA0CF08243C5F811
:108490003428C3F80899A07901280FD106EBC6004B
:1084A00004EB8000D0E907211144016236B9606A0B
:1084B00020B920680121009A08F0D8FA2046F1B2CC
:1084C000FFF7C4FD5FEA087003D505EB4611C1F85C
:1084D00008B95FEAC86004D505EB46111020C1F861
:1084E00008095FEA486004D505EB46114020C1F851
:1084F00008095FEA887016D53146284608F0CBFC9B
:1085000006EBC60004EB8000C17D1430012905D1C3
:1085100080F803A02046F1B200F082F905EB461185
:108520000220C1F808095FEA086003D531462046F9
:1085300005F046FA7F08761C002F96D1206808F0D7
:1085400001FD002811DAD5F8040820F00101C5F872
:10855000041894F8CC0401283BD0204600F016FA09
:108560002068416901F000414161206808F0EAFC9F
:1085700000050BD5D5F80808C00702D0204600F04A
:1085800049FA2068416901F400614161206808F0FE
:10859000D9FC00010AD52068416901F00061416100
:1085A00094F8CC04E0B1204600F034FA206808F0DA
:1085B000C9FCC00472D5D5F8040820F00100C5F844
:1085C00004082068102108F066FC00214FF67F3275
:1085D0002DE00021204684F8CCA4FFF70BFDBFE777
:1085E00084F8CC942068406D0121C0F38300C4F866
:1085F000D0042046FFF7FEFCD8E700BF05EB411092
:10860000C0F80829D0F8003923F40013C0F8003965
:10861000C0F8082BD0F8003B23F40013C0F8003B4F
:10862000D0F8003B43F00063C0F8003B491C2079C0
:108630008842E3D8D5F81C0840F00111C5F81C1891
:10864000E07B68B1D5F8840840F00B01C5F88418C8
:10865000D5F8440840F00B012846C5F844180DE051
:10866000D5F8140842F22B010843C5F81408D5F8D0
:10867000100840F00B012846C5F81018D0F8000883
:1086800020F4FE61C5F80018A1792068009A08F06E
:10869000EDF92068416901F480514161206808F0DA
:1086A00051FC800416D5206808F02AF8206808F0EC
:1086B00010FCE07101F03AFB23680146E2791846AC
:1086C00008F0A4FC204600F04BF92068416901F451
:1086D00000514161206808F035FC000707D52046AD
:1086E00000F058F92068416901F0080141612068F3
:1086F00008F028FC000615D5A869012620F08001A5
:10870000A9610CE006EBC60004EB800090F857026C
:10871000012803D12046F1B2FFF7AFFC761C207987
:10872000B042EFD8206808F00DFCC0021FD501262A
:108730004F4614E006EBC60005EB461304EB800140
:10874000D3F800090A7E012A08D1002806DAF0B21F
:10875000CF7540F080012046FFF78FFC761C207912
:10876000B042E7D82068416901F480114161206876
:1087700008F0E8FB800234D501204A4629E00000D9
:108780000A30544F00EBC00305EB401604EB8301A5
:10879000D6F8006B91F85832012B19D1002E17DA58
:1087A00094F8D434C6F3004603F00103B3420FD16A
:1087B00081F85722A96941F08003AB616969090614
:1087C00006D4D5F8040840F40070C5F8040803E0A6
:1087D000401C21798142D5D82068416901F40011FB
:1087E0004161206808F0AEFB400007D52046FFF746
:1087F00029FC2068416901F080414161206808F04E
:10880000A1FB40070AD520684568680702D52046C5
:10881000FFF72FFC2068416829434160BDE8FC9FB9
:10882000D0F8E00407F021BCD0F8E00407F031BC38
:10883000F8B5040004D094F89504002510B106E0C2
:108840000120F8BD204684F8945400F057F8032026
:1088500084F89504206808F003F9207C8DF8000066
:1088600094E80F0007F05AFF0226B0BB20680021F1
:1088700008F08CFB88BB002001270CE000EBC00156
:10888000421C04EB81014F750D76CD610D624D6286
:108890000875C885D0B221798142EFD8002011E057
:1088A00000EBC001421C04EB810181F8555281F8B4
:1088B0005852C1F85C52C1F86052C1F8645281F854
:1088C0005402D0B221798142EAD8207C8DF8000090
:1088D00094E80F0008F00EF810B184F89564AFE743
:1088E000207B657484F89574012802D12046FFF737
:1088F0006DFB206807F0F0FF0020F8BD10B5B0B0A8
:108900000446B8216846F7F7C8FF13492068884233
:1089100020D100204FF480214FF440122192CDE964
:108920000010684600F008FC08B1FCF7B7F800F04A
:10893000B3F80A48016841F0007101600068002244
:10894000052100F000702E904D20FEF7D1FF4D2044
:10895000FEF7C1FF30B010BD00000440D8440258FB
:1089600070B50446C079012570B1022801D0FCF72A
:1089700095F8D4F8E004294607F0FAFBD4F8E004AF
:10898000BDE8704007F0AEBB0025F2E7D0F8E00488
:1089900007F0D7BBD0F8E00407F0DDBB10B5044604
:1089A00090F8940401280AD00120617484F894049A
:1089B000206808F01AFB002084F8940410BD0220FF
:1089C00010BDD0F8E02400F29C41104607F0DCBB5B
:1089D00010B590F8941404460068012909D00121CB
:1089E00084F89414C168490609D5617B012902D035
:1089F00005E0022010BD816B41F480318163206865
:108A000008F027FA206807F059FF002084F8940442
:108A100010BD000010B50446D0F8E00407F0F6FBE6
:108A20002068D0F8001E41F00101C0F8001EE07A75
:108A3000002804D00248016841F00601016010BD21
:108A400010ED00E0134970B50A68D243520705D50E
:108A5000096801F00701814213D118E00A6822F089
:108A6000070202430A60FEF795FE0A4D4FF47A763C
:108A70000446083D07E000BFFEF78CFE001BB04235
:108A800001D9012070BD2868C0438004F4D40020BF
:108A900070BD00000C4802580248016841F0807126
:108AA000016070470C48025810B501F03FF90549C4
:108AB0000968054AC1F30211515C01F01F01C84069
:108AC00010BD000020440258E04901084A4930B571
:108AD000494C0B1D0A680C3409681D68246802F0B3
:108AE000030305F00102C1F30511C4F3CC0400290E
:108AF00014FB02F200EE102AF8EE400A76D0414A4A
:108B00009FED3E1ADFED3E1AB7EE000A23B1012BAE
:108B10005AD0022B18D15CE0374C283C23689B06C6
:108B200012D5394B246801EE901A1168C4F3C104C0
:108B3000F8EE612AE34001EE903AC1F30801F8EE45
:108B4000611A81EEA22A07E002EE101A1168F8EE0F
:108B5000422A81EEA22A45E001EE901A1168F8EE51
:108B6000611A40EE811A71EE800A62EE200AC1F3AA
:108B7000462101EE101AB8EE411A31EE001AC0EE8D
:108B8000811ABCEEE11A80ED001A1168C1F30641AA
:108B900001EE101AB8EE411A31EE001AC0EE811A39
:108BA000BCEEE11A80ED011A1168C1F3066101EE15
:108BB000101AB8EE411A31EE000A80EE801ABCEEAF
:108BC000C10A80ED020A30BD01EE901ADFED0F2AD6
:108BD00003E001EE901ADFED0E2A1168F8EE611A3B
:108BE00082EEA12AC1F30801B6E7FFE70021016088
:108BF0004160816030BD0000284402580000003907
:108C00000024744C304402580090D0030024744A6D
:108C1000001BB74B494930B5484C0B1D0A6814344A
:108C200009681D68246802F00303C5F30012C1F34C
:108C30000531C4F3CC04002914FB02F200EE102A23
:108C4000F8EE400A75D03F4A9FED3D1AB7EE000A94
:108C50006BB1DFED3D1A012B01D0022B64D002EE87
:108C6000101A1168F8EE422A81EEA22A21E0334C54
:108C7000283C23689B0612D5344B246801EE901AD9
:108C80001168C4F3C104F8EE612AE34001EE903AA2
:108C9000C1F30801F8EE611A81EEA22A0BE001EEA1
:108CA000901ADFED2B2A00BFF8EE611A116882EEF0
:108CB000A12AC1F3080101EE901A1168F8EE611AB9
:108CC00040EE811A71EE800A62EE200AC1F346215D
:108CD00001EE101AB8EE411A31EE001AC0EE811AF8
:108CE000BCEEE11A80ED001A1168C1F3064101EEF5
:108CF000101AB8EE411A31EE001AC0EE811ABCEE1D
:108D0000E11A80ED011A1168C1F3066101EE101A33
:108D1000B8EE411A31EE000A80EE801ABCEEC10AAC
:108D200080ED020A30BD04E001EE901ADFED092A61
:108D3000BAE70021016041608160F3E728440258EE
:108D400000000039384402580024744A0090D003CF
:108D50000024744C001BB74B494930B5484C0B1DDF
:108D60000A681C3409681D68246802F00303C5F30F
:108D70000022C1F30551C4F3CC04002914FB02F214
:108D800000EE102AF8EE400A75D03F4A9FED3D1ADA
:108D9000B7EE000A6BB1DFED3D1A012B01D0022BBB
:108DA00064D002EE101A1168F8EE422A81EEA22A6F
:108DB00021E0334C283C23689B0612D5344B2468B1
:108DC00001EE901A1168C4F3C104F8EE612AE34081
:108DD00001EE903AC1F30801F8EE611A81EEA22A81
:108DE0000BE001EE901ADFED2B2A00BFF8EE611ABE
:108DF000116882EEA12AC1F3080101EE901A1168F0
:108E0000F8EE611A40EE811A71EE800A62EE200AD5
:108E1000C1F3462101EE101AB8EE411A31EE001AE4
:108E2000C0EE811ABCEEE11A80ED001A1168C1F3A0
:108E3000064101EE101AB8EE411A31EE001AC0EEEA
:108E4000811ABCEEE11A80ED011A1168C1F30661C6
:108E500001EE101AB8EE411A31EE000A80EE801AC7
:108E6000BCEEC10A80ED020A30BD04E001EE901AAA
:108E7000DFED092ABAE70021016041608160F3E774
:108E80002844025800000039404402580024744A23
:108E90000090D0030024744C001BB74B2DE9F04F19
:108EA000A14A0546DFF87CA280F48070DFF880924A
:108EB00089B013119F4C08439C48AAF104064FF057
:108EC000805C4FF0005828D0DFF858B285F48067F6
:108ED0000F430BF1080B4FD085F400670F4360D0B0
:108EE00085F480570F4372D085F400570F434FF439
:108EF00080394FF4003E69D085F400270F4373D0CA
:108F000085F480370F4370D085F480460E436DD0D2
:108F100085F400420A436AD02AE0DAF8001001F032
:108F20000701052924D2DFE801F0F9AA6A259F008C
:108F300006A8FFF7CBFD079809B0BDE8F08F68469B
:108F4000FFF768FE0098F7E703A8FFF705FF03980F
:108F5000F2E72068C0F3C10022FA00F0ECE72268D3
:108F6000D2056ED561456CD11846E5E74145E3D0A1
:108F70000020E1E74846DFE7DBF8001001F460017C
:108F8000B1F5800F3BD005DC00294AD0B1F5001FB8
:108F9000EED174E0B1F5C00FECD0B1F5000FE7D120
:108FA00062E0DBF8001001F0E061B1F1007F26D053
:108FB00004DCB1B3B1F1807FDAD160E0B1F1407F80
:108FC000D8D0B1F1806FD3D14EE000E01BE0DAF8E9
:108FD000001001F4E041B1F5005F10D008DC01B3EE
:108FE000B1F5805FC4D14AE035E058E065E088E043
:108FF000B1F5405FBED0B1F5804FB9D134E0206803
:109000008000B5D5A0E7DAF8001001F4E021B1F551
:10901000403F6DD006DC61B149457BD07145A7D199
:1090200058E07BE0B1F5802F66D0B1F5A02F9FD13D
:109030000DE000F09DFE7FE76846FFF7EBFD01982D
:109040007AE728E003A8FFF787FE049874E7216811
:1090500089038AD48CE7DBF8001011F440310ED07C
:10906000494510D0714583D13168256801F04051E0
:109070006D077FF574AF00297FF471AF69E7206851
:109080000001E7D55BE720688000E3D503A8FFF780
:1090900063FE059850E722689203DBD566E73068E7
:1090A00010F480303AD04845D4D120680001D1D5A1
:1090B0006846FFF7AFFD02983EE7DBF8001001F0CD
:1090C000E041B1F1405F13D008DC71B1614521D0BE
:1090D0004145BFD120688000B4D449E7B1F1804F49
:1090E0000AD0B1F1A04FB2D042E7FFF7DDFC23E791
:1090F00020684007AED52CE72068C005AAD533E725
:1091000008E0DAF8001011F04051A0D0614505D018
:1091100041459FD1206800018ED429E72068800155
:1091200098D505E7504402580090D00300366E01F0
:109130000080BB00004402582DE9FE4F0546DFF8D1
:1091400000A450F8081B0024FD4FC943019005F10D
:10915000280026460AF1240A009008011DD4686EF2
:1091600050B1B0F5801F0CD0B0F5001F0ED0B0F597
:10917000401F1ED001240FE0386840F400303860F2
:1091800017E00198022104F0EDFD03E000980221B0
:1091900004F078FE04000CD026462888C043C005A1
:1091A00023D4A86D05281ED2DFE800F00C11161B91
:1091B0001B006A6EDAF8001021F440111143CAF85E
:1091C0000010EAE7386840F40030386009E00198A0
:1091D000002104F0C7FD03E00098002104F052FED6
:1091E0000446C4B100E0012426462888DFF85083F5
:1091F000C04308F12C0840052FD4D5F8A400B0F5E1
:10920000C00F28D010DCB8B1B0F5001F19D0B0F5F0
:10921000800F0FD11AE0AA6DDAF8001021F00701D3
:109220001143CAF80010E0E7B0F5000F13D0B0F515
:10923000200F10D001240FE0386840F4003038606F
:1092400009E00198002104F08DFD03E00098002161
:1092500004F018FE044694B126462888C043000551
:1092600030D4D5F8A800B0F1407F29D011DCC0B1CE
:10927000B0F1807F1AD0B0F1007F10D11BE0D5F89B
:10928000A420D8F8001021F460011143C8F80010A0
:10929000E3E7B0F1806F13D0B0F1A06F10D00124DC
:1092A0000FE0386840F40030386009E00198002190
:1092B00004F058FD03E00098002104F0E3FD0446AB
:1092C00094B126462868DFF878B2C0430BF1200B32
:1092D00080011FD4E86CD8B110280FD0202812D0FC
:1092E000302815D0012414E0D5F8A820D8F80010B3
:1092F00021F0E0611143C8F80010E3E7386840F45A
:109300000030386004E00198022104F02BFD04468F
:1093100074B126462888C043C0042BD4E86DB0F54C
:10932000005F20D00DDCA0B1B0F5805F0FD115E05B
:10933000EA6CDBF8001021F030011143CBF800108B
:10934000E8E7B0F5405F13D0B0F5804F10D00124AE
:109350000FE0386840F40030386009E001980021DF
:1093600004F000FD03E00098002104F08BFD0446AA
:109370008CB126462888C043800429D4286EB0F5D5
:10938000403F23D010DC08B3B0F5803F14D0B0F5D7
:10939000003F0FD115E0EA6DDAF8001021F4E0414A
:1093A0001143CAF80010E5E7B0F5802F0ED0B0F5F4
:1093B000A02F0BD001240AE00198012104F0D2FC77
:1093C00003E00098012104F05DFD044694B12646B7
:1093D0002888C04340042AD4D5F8AC00B0F1405FDF
:1093E00023D010DC08B3B0F1805F14D0B0F1005F7F
:1093F0000FD115E02A6EDAF8001021F4E0211143B4
:10940000CAF80010E4E7B0F1804F0ED0B0F1A04FE1
:109410000BD001240AE00198012104F0A3FC03E031
:109420000098012104F02EFD044674B126462888D8
:10943000C04300041FD4E86ED8B1B0F1805F0ED0F5
:10944000B0F1005F10D0012414E0D5F8AC20D8F8BA
:10945000001021F0E0411143C8F80010E7E7386838
:1094600040F40030386004E00198012104F07AFCF7
:10947000044674B126462868C043C0011ED4A86CB7
:10948000D0B101280ED0022811D0032814D0012415
:1094900013E0EA6EDAF8001021F040511143CAF8E7
:1094A0000010E8E7386840F40030386004E00198C4
:1094B000022104F057FC04466CB126462868C043DC
:1094C000400255D41F48016841F480710160FEF7E5
:1094D00061F981460EE0AA6CDBF8001021F003016F
:1094E0001143CBF80010E9E7FEF754F9A0EB0900AF
:1094F00064283BD813480068C005F5D5BCBBDFF82D
:109500004090B5F8B01009F14409D9F8000001F411
:10951000407100F44070884211D0D9F80010D9F899
:10952000002021F4407142F48032C9F80020D9F8BB
:10953000002022F48032C9F80020C9F8001003E0AE
:109540002C44025800480258D5F8B000B0F5807F8E
:1095500019D1FEF71FF9029011E000BFFEF71AF9CA
:109560000299411A41F28830814208D903242646E3
:109570002878DFF81494C043C00721D03CE0D9F824
:1095800000008007EAD5D5F8B010C1F30120032808
:10959000FE480DD0016821F47C510160B5F8B0207F
:1095A000D9F80010C2F30B021143C9F80010DFE72D
:1095B000F74A036802EA111223F47C511143ECE7E5
:1095C000A86F182816D005DCA0B1082808D01028EC
:1095D00004D10AE020280DD028280BD001240AE06D
:1095E0000198012104F0BEFB03E00098012104F082
:1095F00049FC044664B126462878C04380071ED43F
:10960000686F062819D2DFE800F0160C111616163E
:10961000AA6FD9F8001021F038011143C9F80010E1
:10962000EAE70198012104F09DFB03E00098012185
:1096300004F028FC04467CB100E00124264628788A
:10964000C04340071FD4D5F89000062819D2DFE8A0
:1096500000F0160C111616166A6FD9F8001021F0DA
:1096600007011143C9F80010E9E70198012104F04E
:1096700079FB03E00098012104F004FC0446A4B146
:1096800000E0012426462878C04380062BD4D5F874
:109690008C00B0F1405F24D011DC10B3B0F1805FDA
:1096A00015D0B0F1005F10D116E0D5F89020D8F8B1
:1096B000001021F007011143C8F80010E3E7B0F1F2
:1096C000804F0ED0B0F1A04F0BD001240AE00198DA
:1096D000002104F047FB03E00098022104F0D2FBD4
:1096E000044694B126462878C04340062BD4D5F8CA
:1096F0009800B0F5406F24D011DC10B3B0F5806F46
:1097000015D0B0F5006F10D116E0D5F88C20D9F83F
:10971000001021F0E0411143C9F80010E3E7B0F573
:10972000805F0ED0B0F5A05F0BD001240AE0019855
:10973000002104F017FB03E00098022104F0A2FBD3
:10974000044694B126462878C04300062BD4D5F8A9
:109750009C00B0F5C04F24D011DC10B3B0F5005F11
:1097600015D0B0F5804F10D116E0D5F89820D8F874
:10977000001021F4E0511143C8F80010E3E7B0F500
:10978000004F0ED0B0F5204F0BD001240AE0019815
:10979000002104F0E7FA03E00098022104F072FBD4
:1097A000044654B126462878C04300071ED4D5F895
:1097B0008000B0F5805F0AD00FE0D5F89C20D8F883
:1097C000001021F460411143C8F80010EBE7009845
:1097D000022104F057FB00B10126D5F88020D9F80A
:1097E000001021F440511143C9F800102878C043FB
:1097F000C00613D4D5F89400B0F5807F05D1009849
:10980000022104F03FFB00B10126D5F89420D8F8DE
:10981000001021F440711143C8F800102868C043BB
:10982000000316D4D5F8A00038B1B0F5803F09D0B8
:10983000B0F5003F0BD001240AE00198002104F0AC
:1098400091FA03E00098022104F01CFB04468CB15D
:1098500026462868C043400322D4D5F88400B0F5DA
:10986000801F11D0B0F5001F13D0B0F5401F15D0E8
:10987000012414E0D5F8A020D8F8001021F44031DC
:109880001143C8F80010E4E7386840F4003038604D
:1098900004E00098012104F0F5FA04465CB1264684
:1098A0002868C043C0031CD4286D70B1B0F5803F58
:1098B00010D0012414E0D5F88420D9F8001021F448
:1098C00040111143C9F80010EAE7386840F400304D
:1098D000386004E00198022104F044FA0446DCB147
:1098E00026462868C043800005D40098022104F071
:1098F000C9FA00B101262868C04380031BD4E86F71
:10990000B8B1B0F5807F10D0B0F5007F11D0B0F5C0
:10991000407F0ED001240DE02A6DDBF8001021F409
:1099200080311143CBF80010DBE7386840F4003099
:1099300038607CB326462868C043C00207D42A6F2B
:10994000DAF8001021F000411143CAF8001028682D
:10995000C043800207D4AA6EDAF8001021F08071AB
:109960001143CAF800102868C043400009D40748D2
:10997000016821F4004101600168D5F8B420114369
:1099800001602868C04306E054440258104402585D
:10999000CFFFFF001DE007D46A6DDBF8001021F057
:1099A00040511143CBF800102868C043000208D48E
:1099B000D5F88820D9F8001021F440011143C9F8E6
:1099C000001028790024C04300F00100204309D092
:1099D0000EE0EA6FD9F8001021F440711143C9F884
:1099E0000010A8E70198002104F0BCF900B1064678
:1099F0002879C04300F00200204305D101980121DD
:109A000004F0B0F900B106462879C04300F0040024
:109A1000204305D10198022104F0A4F900B10646C3
:109A20002879C04300F00800204305D100980021A8
:109A300004F028FA00B106462879C04300F010006F
:109A4000204305D10098012104F01CFA00B106461C
:109A50002879C04300F02000044304D1009802217B
:109A600004F010FA00B916B10120BDE8FE8F002005
:109A7000FBE700002DE9F05F04000F467ED0DFF821
:109A80003882D8F8000000F00F00B8420CD2D8F8A5
:109A9000001021F00F013943C8F80010D8F8000079
:109AA00000F00F00B84269D12078844D40070AD5F4
:109AB0002069296801F07001884204D9296821F0E1
:109AC00070010143296020787C4E361D00070AD5BD
:109AD0006069316801F07001884204D9316821F071
:109AE0007001014331602078C0060AD5A069316851
:109AF00001F4E061884204D9316821F4E061014356
:109B000031602078DFF8B4B180060BF1080B0CD57A
:109B1000E1695846DBF8002002F07002914204D956
:109B2000026822F070020A430260207880070AD59A
:109B3000E068296801F00F01884204D9296821F002
:109B40000F01014329602078C0073ED05B49A2681D
:109B50002868183920F47060104328606068022873
:109B600018D0032819D00968012819D049070029FD
:109B70004ADADFF848A1AAF1080A00E044E0DAF87E
:109B8000002022F007020243CAF80020FDF702FE7F
:109B9000814612E009688903E9E709688901E6E777
:109BA000C905E4E7FDF7F6FDA0EB090141F28830B5
:109BB000814202D90320BDE8F09F6168DAF8000015
:109BC00000F03800B0EBC10FECD1207880070AD547
:109BD000E068296801F00F01884204D2296821F069
:109BE0000F0101432960D8F80010404601F00F0131
:109BF000B9420BD9016821F00F01394301600068B7
:109C000000F00F00B84201D00120D4E720784007CF
:109C10000AD52069296801F07001884204D22968B8
:109C200021F0700101432960207800070AD560699E
:109C3000316801F07001884204D2316821F070016E
:109C4000014331602078C0060AD5A069316801F46B
:109C5000E061884204D2316821F4E061014331605F
:109C6000207880060CD5E1695846DBF8002002F028
:109C70007002914204D2026822F070020A4302602C
:109C800000F09AF80E492A682B68C2F3032203F009
:109C90000F038A5CC95C02F01F0201F01F01D04073
:109CA000084A20FA01F11160074908600748006876
:109CB000BDE8F05FFDF7AABD00200052184402582D
:109CC000E04901088C00002088000020800000206E
:109CD00070B5144C3F220260124A24680832131DEA
:109CE000114D04F00704446016681C1D06F47066EC
:109CF0008660166806F00F06C660126802F07002F1
:109D000002611A6802F0700242611A6802F4E062AD
:109D10008261226802F07002C261286800F00F00C0
:109D2000086070BD104402580020005230B500F0A9
:109D300043F80B4A0B490C4B15681468C5F3032212
:109D400004F00F048A5C095D02F01F0201F01F019C
:109D5000D040064A20FA01F119601060084630BD73
:109D600018440258E04901088C00002088000020B7
:109D700000B5FFF7DBFF05490968054AC1F3021189
:109D8000515C01F01F01C84000BD00001C44025896
:109D9000E049010800B5FFF7C9FF05490968054A10
:109DA000C1F30221515C01F01F01C84000BD000059
:109DB0001C440258E0490108454970B54548096806
:109DC000434B103B11F0380208D00111082A03D090
:109DD000102A0BD0182A0BD0084670BD19688906C6
:109DE000FBD51968C1F3C101C84070BD3A4870BDC8
:109DF0003749374D18310C1D24350A680968266823
:109E00002D6802F0030406F00102C1F30511C5F349
:109E1000CC0515FB02F200EE102AB8EE400AE9B3B9
:109E20002F4ADFED2E0AB7EE001A6CB1DFED2D1AC6
:109E3000012C01D0022C43D002EE101A1068F8EE6B
:109E4000422A81EEA22A1EE01C68A40611D51B68D6
:109E500001EE901A1168C3F3C103F8EE612AD840ED
:109E600001EE900AC1F30800F8EE611A81EEA22A11
:109E70000BE001EE901ADFED1C2A00BFF8EE611A2C
:109E8000106882EEA12AC0F3080001EE900AF8EEF5
:109E9000611A40EE201A31EE810A00E015E022EE50
:109EA000000A1068C0F34620401C00EE900AF8EE4D
:109EB000600A80EE201ABCEEC10A10EE100A70BDD6
:109EC00001EE901ADFED092AD8E7002070BD0000EE
:109ED000104402580090D00300366E010000003993
:109EE000304402580024744A0024744C001BB74BC1
:109EF000F0B50D461F49204C002887B016464FF09C
:109F000000004FF002020F684FF0030319D047F032
:109F100004070F60096801F0040105911102009126
:109F2000CDE90120CDE9033014486946FDF71AFB5D
:109F3000206845EAC61120F07E400843206007B043
:109F4000F0BD47F001070F60096801F001010591BC
:109F50004FF480710091CDE90120CDE9033008482C
:109F60006946FDF7FFFA2068354320F0FE7028436C
:109F7000E4E70000E0440258104402580008025888
:109F8000000002582DE9F05F04007DD0FF4F2078DB
:109F9000FE4D1837DFF8F483103DC00748D0D8F8DD
:109FA0000000396800F03800102815D0182803D1B7
:109FB00001F0030002280FD06068B0F5803F12D096
:109FC00010B1B0F5A02F18D0286820F48030286098
:109FD000286820F4802009E02868800328D560687C
:109FE0000028D2D024E0286840F4803028606068DF
:109FF00088B1FDF7CFFB064609E0286840F48020D1
:10A000002860F0E7FDF7C6FB801B64287ED828682F
:10A010008003F7D50CE0FDF7BDFB064605E000BF69
:10A02000FDF7B8FB801B6428F0D828688003F7D4BC
:10A030002078800756D5D8F80000DFF850933968AB
:10A0400010F03800A9F10C090ED0182801D18807AA
:10A050000AD0E068A8B3296821F0190101432960FA
:10A06000FDF798FB064628E02868400702D5E0681F
:10A0700000288AD0E168286820F019000843286089
:10A08000FDF788FB064606E0D2E000BFFDF782FB45
:10A09000801B0228BAD828684007F7D5217CD9F858
:10A0A000002022F0FE4242EA0161C9F8001019E0E6
:10A0B000FDF770FB801B0228A8D828684007F7D559
:10A0C000ECE7FFE7286820F001002860FDF762FB5D
:10A0D000064604E0FDF75EFB801B022896D8286840
:10A0E0004007F7D42078C00646D5D8F80000DFF83E
:10A0F0009C92396800F03800A9F10409082812D0B0
:10A10000182805D101F00300012800E0CEE00AD0B4
:10A11000E0690028286820D040F080002860FDF722
:10A1200039FB064615E02868C00502D5E06980289D
:10A130007ED194F82010D9F8002022F07C5242EA17
:10A140000161C9F8001017E0FDF724FB801B02280D
:10A15000A0D82868C005F7D5EBE720F0800028607C
:10A16000FDF718FB064604E0FDF714FB801B0228F0
:10A1700090D82868C005F7D42078000729D58348EF
:10A180006169643000298146016811D041F0010104
:10A190000160FDF7FFFA064605E000BFFDF7FAFA99
:10A1A000801B022888D8D9F800008007F6D510E077
:10A1B00021F001010160FDF7EDFA064605E000BF60
:10A1C000FDF7E8FA801B022870D8D9F80000800754
:10A1D000F6D42078800623D5A0690028286810D0FE
:10A1E00040F480502860FDF7D5FA064605E000BF30
:10A1F000FDF7D0FA801B022858D828688004F7D5CC
:10A200000EE020F480502860FDF7C4FA064604E012
:10A21000FDF7C0FA801B022848D828688004F7D4CC
:10A220002078400751D5DFF86891D9F8001000E098
:10A2300015E141F48071C9F80010FDF7ABFA06464C
:10A2400005E000BFFDF7A6FA801B64282ED8D9F8D8
:10A250000000C005F6D54D4EA068603601280AD032
:10A2600008B1052813D0306820F001003060306854
:10A2700020F0040002E0306840F001003060A06887
:10A2800041F2883A98B1FDF785FA81460AE03068D4
:10A2900040F004003060EEE7FDF77CFAA0EB090126
:10A2A000514503D830688007F6D50EE072E0FDF71F
:10A2B00071FA814606E000BFFDF76CFAA0EB0901D8
:10A2C000514567D830688007F6D4606A00287CD092
:10A2D000DFF8B8A0D8F800100AF1200A4FF6F87B92
:10A2E0000AF10408C1F3C2010329AAF104096DD0DF
:10A2F0000228286820F08070286003D0FDF74AFA11
:10A30000044681E0FDF746FA064604E0FDF742FA0E
:10A31000801B022875D828688001F7D4E26A40F2D1
:10A32000F331386854F8283F884340EA0210184354
:10A330003860217B4FF4FE0C22894FF0FE47208AC3
:10A340004902267D521E401EA1F5007189B2C2F35A
:10A3500008021143761E0CEA00400143484607EA12
:10A3600006621143CAF80010D9F8001021F001016B
:10A37000C9F80010D8F80030266A23EA0B0343EA34
:10A38000C601C8F80010D9F8001004E010440258C3
:10A390000048025835E0A26921F00C011143C9F8C8
:10A3A00000100168E26921F00201114301600168B7
:10A3B00041F480310160016841F4003101600168BD
:10A3C00041F480210160016801E06CE020E041F08F
:10A3D00001010160286840F080702860FDF7DAF91B
:10A3E000044604E0FDF7D6F9001B022809D82868C6
:10A3F0008001F7D557E000BFFDF7CCF9001B02281C
:10A4000002D90320BDE8F09F28688001F4D44AE017
:10A4100039680128DAF8000021D0A26A01F00303AC
:10A4200093421CD1E26AC1F305118A4217D1216B14
:10A43000C0F30802491E8A4211D1616BC0F3462263
:10A44000491E91420BD1A16BC0F30642491E9142B5
:10A4500005D1E16BC0F30660491E814201D00120A5
:10A46000D0E7A16C4646D8F80000C0F3CC0081428A
:10A4700019D0D9F800004D4620F00100C9F80000BD
:10A48000FDF788F94FEA0007FDF784F9B842FBD0E1
:10A49000A26C306820EA0B0040EAC20030602868F5
:10A4A00040F0010028600020ACE700002DE9F041F9
:10A4B00004001D4616460F4603D0D4F8880018B194
:10A4C00008E00120BDE8F081002084F884002046E7
:10A4D00001F042FD2420C4F888002068016821F0C2
:10A4E00001010160A06A10B1204604F031FC204651
:10A4F00004F0D0FD0128E5D0206871050D4A41EA3D
:10A500000541836843F4804383602068836823F4B3
:10A5100000433B4383602068036813400B430360A0
:10A520002068016841F0010101602046BDE8F0416A
:10A5300004F072BCFFFF00FC70B5044603F0D2FDCE
:10A54000022811D0204603F0CDFD084D05EB401048
:10A550008069002808D0204603F0C4FD05EB4010B8
:10A560008069BDE87040004770BD0000809B0020FE
:10A570002DE9F047044600680021036942698768B5
:10A5800094F8816000F130095FEA025C03EA020599
:10A590000AD51A0708D5816941F400618161204616
:10A5A00000F0C6FCBDE8F08715F0600F08D1680721
:10A5B00006D5616F20468847216F204688470121D4
:10A5C00005F04100012805D1680703D4216F20461A
:10A5D0008847012105F02200022806D1680704D42B
:10A5E000616F2046BDE8F04708470029DAD1280707
:10A5F0004FF001085BD52068816941F00801816155
:10A600002068816941F0100181612068816941F40D
:10A61000006181612068016921F008010161206801
:10A62000806810F4404F20D023E0E0680F2806D95E
:10A630002068616E006B0860606E001D0FE00728E7
:10A6400006D9B9F80000616E0880606E801C06E0D3
:10A650002068616E90F830000870606E401C606683
:10A66000B4F86A00401EA4F86A00B4F86A00002832
:10A67000DBD1204603F09CFC84F88180D4F8840070
:10A6800018B12046FFF758FF8CE7052E07D0042E9F
:10A6900009D0032E86D1204600F06CFD82E72046CB
:10A6A00000F07AFD7EE7204600F00AFC7AE715F418
:10A6B000587FE9D068060AD5D4F8840040F0040039
:10A6C000C4F884002068816941F040018161A805D7
:10A6D0000AD5D4F8840040F00100C4F88400206852
:10A6E000816941F400718161E8050AD5D4F88400DC
:10A6F00040F00800C4F884002068816941F480714A
:10A700008161A8060AD5D4F8840040F08000C4F81E
:10A7100084002068816941F020018161D4F88400BF
:10A720000028B1D0206840F26B32C7F38131036852
:10A73000032923F0010101602068016921EA020177
:10A74000016102D084F881809BE72068104D816808
:10A7500021F440418160E06F50B10565E06FFBF787
:10A760003FFB28B1D4F8840040F04000C4F88400D6
:10A77000A06F002888D00565A06FFBF731FB00288B
:10A780008CD0D4F8840040F04000C4F8840009E77D
:10A790006DE000082DE9F047040029D0594A4FF038
:10A7A00000092068584B594D9042C4F8289006D0B3
:10A7B000984204D0A84202D0E1680F2918D8E16875
:10A7C0004FF0010AE76B0831C9080AEB57167143CD
:10A7D000904205D0984203D0A84201D0082907D85A
:10A7E000904203D0984201D0A84204D1102902D946
:10A7F0000120BDE8F08794F8810020B9204684F854
:10A80000809000F085F8022084F8810020680168BB
:10A8100021F0010101602068A1698268B1F1806FB7
:10A8200002F4F81110D16268B2F5800F01D01AB1AC
:10A830000AE0A26B22B107E0A26BB2F1805F03D104
:10A84000026842F4805202606068400209D5E06804
:10A85000072806D32068236D026822F480721A4309
:10A8600003E02068026822F480720260A66AE06950
:10A87000E26B25683043E3680A4310431843A8603D
:10A88000D4E90D02D4E90581636A25691843D4F837
:10A8900020C00A43266810432843A56DD4E90172FD
:10A8A000D4E9123140EA080040EA0C00384308437A
:10A8B000104318432843F060606868B920688168D5
:10A8C00021F4C05141F4006181602068816821F465
:10A8D000C06141F4806181602068016D21F0010157
:10A8E00001656068400206D52068626DC16821F08C
:10A8F00000411143C160C4F8849084F881A0002015
:10A9000077E700000030014000380040003C004084
:10A910002DE9F047B4B0074614212EA8F5F7BDFF86
:10A92000B8216846F5F7B9FF614902263868002466
:10A930005D4D4FF00308DFF874A188424FF0050920
:10A940003DD1811417940020CDE900106846FEF730
:10A95000F3FB08B1FAF7A2F853481030016841F44C
:10A9600080510160006800F480503390286840F006
:10A9700008002860286800F008003390286840F03C
:10A9800002002860286830AA45464F4600F00200C1
:10A9900033908020CDE92E0682E8B00045482EA9EC
:10A9A000FCF7E0FD082030AACDE92E062EA950467E
:10A9B00082E8B000FCF7D6FD34B0BDE8F0873E4930
:10A9C0008842F9D1811417940020CDE9001068461F
:10A9D000FEF7B2FB08B1FAF761F8334808300168B6
:10A9E00041F480410160006800F4804033902868A1
:10A9F00040F004002860286800F0040033902868C4
:10AA000040F002002860286806214546C84600F04C
:10AA10000200CDE92E16CDE93045CDE93290274828
:10AA20002EA9FCF79FFD4FF40051504630AACDE906
:10AA30002E162EA982E83001FCF794FD204E272324
:10AA4000204A4FF480684FF44039304686E81C00B5
:10AA5000C6E903487461B461C6E907497462FBF74B
:10AA600077FE08B1FAF71AF8154D28221549402348
:10AA70007835FE671831B763284685E81E016C619A
:10AA8000AC61C5E907496C62FBF762FE08B1FAF7F1
:10AA900005F8BD6700220521AF632420FCF728FFDD
:10AAA0002420FCF718FF87E7E0440258000402580E
:10AAB00000300140000C02580038004000080258E5
:10AAC000BC070020400002402DE9F84F8946C16BC9
:10AAD000044600689A4616464909491C1FFA81F83F
:10AAE00030300090FCF756FE834694F88100012830
:10AAF00038D1B9F1000F6FD0002EFCD094F880004F
:10AB000001282FD0A1680025012784F88070042037
:10AB100084F88100C4F88450C4F86490E565A4F812
:10AB20006050256765672C34B1F5C02FA687E6878E
:10AB3000E58654F82C0D18D0C16821F4C02141F4E9
:10AB40008021C160206841686FF30F01314341608B
:10AB50002068016841F0010101606068B0F5800F74
:10AB600008D00CE00220BDE8F88F016821F40061F4
:10AB70000160E7E72068016841F400710160E06866
:10AB80000F2824D829E0206841694269D20705D1FD
:10AB9000B4F86A3043450DD209040BD5006B616EE1
:10ABA0000860606E001D6066B4F86A00401EA4F87C
:10ABB0006A000CE0FCF7EEFDA0EB0B01514503D35E
:10ABC000BAF1FF3F03D0AAE0BAF1000F40D0B4F8C9
:10ABD0006A000028D7D194E09FE007283CD88CE099
:10ABE000216848694969C9070AD000980088616EE0
:10ABF0000880606E801C6066B4F86A00401E15E034
:10AC0000B4F86A20424514D2010412D50098008895
:10AC1000616E0880606E801C606600990988018002
:10AC2000606E801C6066B4F86A00801EA4F86A003A
:10AC300012E0B4F86A10012901D18004D5D4FCF7E0
:10AC4000A9FDA0EB0B01514503D3BAF1FF3F03D09F
:10AC500065E0BAF1000F62D0B4F86A000028BFD1F5
:10AC60004FE0206841694269D2070AD090F830006D
:10AC7000616E0870606E401C6066B4F86A00401E29
:10AC800024E0B4F86A30434523D20A0421D590F871
:10AC90003000616E0870606E401C6066216891F83B
:10ACA00030100170606E401C6066216891F83010B1
:10ACB0000170606E401C6066216891F83010017070
:10ACC000606E401C6066B4F86A00001FA4F86A0059
:10ACD00013E0B4F86A20042A02D211F4C04FC5D19F
:10ACE000FCF758FDA0EB0B01514503D3BAF1FF3F30
:10ACF00003D014E0BAF1000F11D0B4F86A000028B4
:10AD0000AFD1204603F054F984F88170D4F8840060
:10AD100084F8805000283FF426AF012023E7204626
:10AD200003F046F9D4F8840084F8805040F4807031
:10AD3000C4F8840084F88170032014E72DE9F04101
:10AD4000044690F8810016460025012802D084F8B8
:10AD500080502FE059B356B394F88000012829D0D1
:10AD6000A268012784F88070042084F88100C4F868
:10AD70008450256765676166A4F860502C34B2F58D
:10AD8000C02FA687E687E58654F82C0D15D0C1683C
:10AD900021F4C02141F48021C0F80C10E0684FF488
:10ADA00080410F280ED9E26F92698A420AD084F856
:10ADB000805055E00220BDE8F081016821F4006177
:10ADC0000160EBE707284FF4005205D9E06F806976
:10ADD000904201D08842EAD12068836823F48043FE
:10ADE0008360E068072811D8E06F8369934205D13A
:10ADF000B4F86A20521C5208A4F86A20806988427C
:10AE000010D1B4F86A00C01C800809E00F2809D8E6
:10AE1000E06F8069884205D1B4F86A00401C4008A0
:10AE2000A4F86A00E06F23490164E16F2248C86317
:10AE3000E16F2248C864E06F0565B4F86A302168A4
:10AE4000626EE06F3031FBF761FE58B1D4F88400D8
:10AE500084F8805040F01000C4F8840084F88170B9
:10AE60000120A8E7E06FC069B0F5807F20684168E5
:10AE70006FF30F0100D0314341602068816841F4D5
:10AE8000804181602068016941F45071016120684E
:10AE9000016841F0010101606068B0F5800F04D1E4
:10AEA0002068016841F400710160002084F880503E
:10AEB00081E70000B3E00008BDE0000887E000087B
:10AEC00070B5044603F00EF9022811D0204603F0B5
:10AED00009F9084D05EB40104068002808D02046CD
:10AEE00003F000F905EB40104068BDE870400047F2
:10AEF00070BD0000809B002070B5044603F0F2F89E
:10AF0000022811D0204603F0EDF8084D05EB401063
:10AF10000069002808D0204603F0E4F805EB401053
:10AF20000069BDE87040004770BD0000809B0020B4
:10AF300070472DE9F84F044600689946174600F11E
:10AF4000200B8A46FCF726FC064694F8810001286F
:10AF500039D1BAF1000F7ED0002FFCD094F88000D8
:10AF6000012830D0A26800254FF0010884F88080C5
:10AF7000032184F88110C4F88450C4F85CA065668D
:10AF8000A4F86850656725672C34B2F5C02FA786F2
:10AF9000E786E58754F82C0D18D0C16821F4C0214C
:10AFA00041F40031C160206841686FF30F013943FB
:10AFB00041602068016841F0010101606068B0F5FE
:10AFC000800F08D00CE00220BDE8F88F016841F442
:10AFD00000610160E7E72068016841F400710160E9
:10AFE000E0680F281CD820E02068416989070BD54C
:10AFF000E16D09680162E06D001DE065B4F8620072
:10B00000401EA4F862000BE0FCF7C4FB811B49451D
:10B0100003D3B9F1FF3F03D09DE0B9F1000F32D067
:10B02000B4F862000028DFD179E007282FD872E059
:10B030002068416989071ED5B4F8621001290DD92D
:10B04000E16B59B1E16D09680162E06D001DE065D9
:10B05000B4F8620000E07CE0801E09E0E06D018849
:10B06000ABF80010E06D801CE065B4F86200401E93
:10B07000A4F862000BE0FCF78DFB811B494503D36C
:10B08000B9F1FF3F03D066E0B9F1000F63D0B4F827
:10B0900062000028CCD142E02068416989072ED5A2
:10B0A000B4F8621003290CD9E16B402909D9E16D8C
:10B0B00009680162E06D001DE065B4F86200001FE0
:10B0C0001AE0B4F8621001290CD9E16B51B1E06DBE
:10B0D0000188ABF80010E06D801CE065B4F86200F8
:10B0E000801E09E0E16D097880F82010E06D401CB9
:10B0F000E065B4F86200401EA4F862000BE0FCF7C3
:10B1000049FB811B494503D3B9F1FF3F03D022E03E
:10B11000B9F1000F1FD0B4F862000028BCD10022A2
:10B120004B4608212046009602F0E6FF28B1D4F8ED
:10B13000840040F02000C4F88400204602F038FF6C
:10B1400084F88180D4F8840084F8805000283FF48B
:10B150003BAF012038E7204602F02AFFD4F88410E4
:10B1600084F8805041F48071C4F8841084F88180A0
:10B17000032029E710B502F0B5FF022808D00549E1
:10B1800001EB40100068002802D0BDE810400047E5
:10B1900010BD0000809B002070B5044602F0A2FFA5
:10B1A000022811D0204602F09DFF084D05EB40100B
:10B1B0008068002808D0204602F094FF05EB40107C
:10B1C0008068BDE87040004770BD0000809B002093
:10B1D000024A136883430B4313607047040400580A
:10B1E0007047704770470000F0B590F83C20012A86
:10B1F00043D0012280F83C20D1E90242204ECD69A3
:10B2000022F440722243D1E9004322F480621A43BF
:10B2100022F400622243D1E9043422F480521A431A
:10B220000B6B22F4005222430C8B22F480421A430F
:10B23000036822F4702242EA0442002422F0805281
:10B24000B34242EA050202D00E4DAB4210D10F8D3F
:10B2500022F4700CD1E90862CD6A4CEA075121F062
:10B260008071314321F00071114321F000522A43D3
:10B270005A6480F83C400020F0BD0220F0BD000080
:10B280000000014000040140F0B590F83C20012A84
:10B2900041D0224E012480F83C40022280F83D201B
:10B2A00002681F4D5368B242D2F808C001D0AA42CA
:10B2B00003D14F6823F470033B430F6823F07003FE
:10B2C0001F4357600268B24219D0B2F1804F16D0C6
:10B2D000144B9A4213D0144B9A4210D0134B9A42FB
:10B2E0000DD0AA420BD0124B9A4208D0114B9A4271
:10B2F00005D0114B9A4202D0104B9A4204D1896872
:10B300002CF0800319439160002180F83D4080F8C3
:10B310003C100846F0BD0220F0BD000000000140D6
:10B32000000401400004004000080040000C004000
:10B33000001800400040014000E0004000E40040F0
:10B3400010B5040003D094F83D0010B107E00120CF
:10B3500010BD002084F83C00204600F022F80220B6
:10B3600084F83D002068211D02F0CAFF012084F806
:10B37000480084F83E0084F83F0084F8400084F8D8
:10B38000410084F8420084F8430084F8440084F8C3
:10B39000450084F8460084F8470084F83D0000200A
:10B3A00010BD704790F83D10012901D00120704771
:10B3B0001A4A022180F83D100168CB6843F001036E
:10B3C000CB60006890421AD0B0F1804F17D014497A
:10B3D000884214D01349884211D0134988420ED0B4
:10B3E000124988420BD01249884208D0114988423C
:10B3F00005D01149884202D01049884207D181689E
:10B400000F4A1140062906D0B1F5803F03D00168EC
:10B4100041F0010101600020704700000000014080
:10B420000004004000080040000C004000040140FF
:10B43000001800400040014000E0004000E40040EF
:10B440000700010070472DE9F0410446006800271D
:10B45000C6680569A90713D5B10711D5FA1E02619F
:10B4600001212177206880698007204602D0FFF7FC
:10B47000E9FF04E000F0F8F8204600F0EDF9277746
:10B48000680716D5700714D5226802206FF00401F2
:10B49000116120772068806910F4407F204602D037
:10B4A000FFF7D0FF04E000F0DFF8204600F0D4F909
:10B4B0002777280715D5300713D5226804206FF0A9
:10B4C0000801116120772068C0698007204602D0FA
:10B4D000FFF7B8FF04E000F0C7F8204600F0BCF921
:10B4E0002777E80616D5F00614D5226808206FF0F5
:10B4F0001001116120772068C06910F4407F204658
:10B5000002D0FFF79FFF04E000F0AEF8204600F005
:10B51000A3F92777E80708D0F00706D021686FF075
:10B5200001000861204600F083FA280601D4A8042F
:10B5300008D5300606D521686FF402500861204610
:10B54000FFF74FFEE80508D5300606D521686FF4F1
:10B55000807008612046FFF743FE680608D5700634
:10B5600006D521686FF040000861204600F06AFAB5
:10B57000A8060AD5B00608D521686FF0200008613A
:10B580002046BDE8F041FFF72DBEBDE8F081000088
:10B5900030B587B0044614216846F5F77EF9246873
:10B5A00000222B4D022329490120AC4211D10C6805
:10B5B00044F010040C60096801F0100105914FF48B
:10B5C00008510091CDE90132CDE9032021486946B7
:10B5D00025E0B4F1804F12D01F4D2048AC4222D15B
:10B5E0000C6844F002040C600968009301F0020149
:10B5F000CDE901320392CDE9043169460FE00C68D0
:10B6000044F001040C60096801F001010591052175
:10B610000091CDE90132CDE9032011486946FBF7DD
:10B62000A1FF07B030BD0F4DAC42FAD10C6844F019
:10B6300002040C60096801F002010591E913009110
:10B64000CDE90132CDE903236946E8E7E044025839
:10B65000000001400010025800040040000402589D
:10B660000000025800180040704770B5044690F87A
:10B670003C0000260D4601280BD0012084F83C0038
:10B680000C2A4AD007DC82B1042A20D0082A06D12D
:10B6900031E0022070BD102A53D0142A63D0012655
:10B6A000002084F83C00304670BD206802F0A6FE01
:10B6B0002068816941F0080181612068816921F079
:10B6C0000401816120682A698169114311E02068C1
:10B6D00002F0E6FE2068816941F400618161206822
:10B6E000816921F48061816120682969826942EA67
:10B6F00001218161D4E7206802F01EFF2068C16942
:10B7000041F00801C1612068C16921F00401C161F3
:10B7100020682A69C169114311E0206802F058FFCE
:10B720002068C16941F40061C1612068C16921F4E8
:10B730008061C16120682969C26942EA0121C16151
:10B74000AEE7206802F080FF2068416D41F00801FB
:10B7500041652068416D21F00401416520682A6936
:10B76000416D114311E0206802F0A8FF2068416D8F
:10B7700041F4006141652068416D21F480614165BB
:10B7800020682969426D42EA0121416588E710B5C8
:10B79000040003D094F83D0010B107E0012010BD73
:10B7A000002084F83C00204600F022F8022084F8B3
:10B7B0003D002068211D02F0A3FD012084F848000F
:10B7C00084F83E0084F83F0084F8400084F841008B
:10B7D00084F8420084F8430084F8440084F845006B
:10B7E00084F8460084F8470084F83D00002010BD2E
:10B7F00008B501681348814201D113480FE013488E
:10B80000B1F1804F0BD0124A914210D1016841F042
:10B8100002010160006800F00200009008BD0168AC
:10B8200041F001010160006800F00100F5E7094AFC
:10B830009142F3D1016841F040010160006800F0DD
:10B840004000EAE700000140F0440258E844025892
:10B8500000040040001800407047000030B5044666
:10B860004FF0020269B1042912D0082917D00C291F
:10B870001CD0102921D094F84300012824D00120A5
:10B8800030BD94F83E000128F9D184F83E201DE037
:10B8900094F83F000128F2D184F83F2016E094F894
:10B8A00040000128EBD184F840200FE094F84100DB
:10B8B0000128E4D184F8412008E094F842000128EE
:10B8C000DDD184F8422001E084F843200122206881
:10B8D00002F086FD1E4920681E4A1F4B884209D08F
:10B8E000904207D0984205D01C4DA84202D01C4D72
:10B8F000A84203D1456C45F4004545642068884260
:10B9000018D0B0F1804F15D01649884212D0164990
:10B9100088420FD0154988420CD090420AD0144971
:10B92000884207D0984205D01249884202D0124975
:10B93000884207D18168114A1140062906D0B1F525
:10B94000803F03D0016841F001010160002030BD5B
:10B95000000001400004014000400140004401405B
:10B96000004801400004004000080040000C004076
:10B970000018004000E0004000E400400700010023
:10B9800030B50022044600680D4602F029FD41F260
:10B990001111224B20688A1098420BD0204B9842FC
:10B9A00008D0204B984205D01F4B984202D01F4B25
:10B9B000984209D1036A0B4206D1036A134203D1AC
:10B9C000436C23F4004343642068036A0B4206D1AE
:10B9D000016A114203D1016821F0010101604FF0B9
:10B9E00001005DB1042D0CD0082D0DD00C2D0ED012
:10B9F000102D0FD084F84300002030BD84F83E00A5
:10BA0000FAE784F83F00F7E784F84000F4E784F8A9
:10BA10004100F1E784F84200EEE700000000014039
:10BA20000004014000400140004401400048014042
:10BA300000680349884201D1FBF7B2BE704700009D
:10BA400000E00040704730B590F88410012918D00C
:10BA5000012280F884202421C0F8881000222024AC
:10BA600001680B680D6823F0005325F001050D6097
:10BA7000426601680B60C0F8884080F88420104658
:10BA800030BD022030BD7047704770B5044690F855
:10BA9000840001281DD0012284F884202420C4F8C9
:10BAA000880020680568026822F0010202602068B0
:10BAB000826822F060620A438260204603F026F921
:10BAC0002268202100201560C4F8881084F88400C2
:10BAD00070BD022070BD70B5044690F88400012846
:10BAE0001DD0012284F884202420C4F88800206816
:10BAF0000568026822F0010202602068826822F074
:10BB000060420A438260204603F000F92268202147
:10BB100000201560C4F8881084F8840070BD0220ED
:10BB200070BD70477047000010B503F08DFA06280D
:10BB30000AD000EBC001054800EB81000069002835
:10BB400002D0BDE81040004710BD00008C9A0020D4
:10BB50002DE9F04107680025044640F60F03022650
:10BB6000F8693968BA6818420AD183067ED501F0AF
:10BB7000200302F0805C53EA0C0377D0616F7EE112
:10BB8000D44BDFF854C3134001EA0C0C53EA0C0CFD
:10BB90006CD05FEAC07C0CD05FEAC15C09D54FF085
:10BBA000010CC7F820C0D4F8907047F00107C4F822
:10BBB0009070870709D5D70707D027683E62D4F869
:10BBC000906046F00406C4F8906046070AD5D60790
:10BBD00008D0276804263E62D4F8906046F002063A
:10BBE000C4F8906006070CD501F020061E4308D06B
:10BBF000266808233362D4F8903043F00803C4F871
:10BC0000903003050BD54B0109D526684FF400632E
:10BC10003362D4F8903043F02003C4F89030D4F865
:10BC20009030002B3DD0800609D501F0200002F0B5
:10BC30008051084303D0616F09B1204688472168CD
:10BC4000D4F890008968490602D410F0280F2AD051
:10BC5000204603F0B7F92068806840061ED52068AA
:10BC6000083050E8001F21F0400100E021E040E8EA
:10BC70000012002AF3D1D4F8800078B19749016509
:10BC8000D4F88000FAF7ACF800280AD0D4F8800085
:10BC9000016D00E02046BDE8F04108472046FFF76F
:10BCA00043FFBDE8F0812046FFF73EFFC4F8905007
:10BCB000F7E7D4F86CC02023BCF1010F7ED15FEA16
:10BCC000C06C7BD55FEAC16C78D5102038622068E3
:10BCD0008068400673D5D4F8802081491068884276
:10BCE00034D07F491831884230D07D493031884284
:10BCF0002CD07B494831884228D07949603188422C
:10BD000024D077497831884220D0754990318842D3
:10BD10001CD07349A831884218D07249884215D086
:10BD200070491831884211D06E49303188420DD0A7
:10BD30006C494831884209D06A496031884205D04F
:10BD400068497831884201D06649903140684FF4A3
:10BD500080770004000C40D0B4F85C1081423CD9DC
:10BD6000A4F85E00D069B8422FD0216851E8000FD6
:10BD700020F4807041E80002002AF6D120680830E3
:10BD800050E8001F21F0010140E80012002AF5D11F
:10BD90002068083050E8001F21F0400140E8001200
:10BDA000002AF5D1C4F88C30E566206850E8001F01
:10BDB00021F0100140E80012002A01E04AE019E0F9
:10BDC000F3D1D4F88000F9F75BFE2667B4F85C0085
:10BDD000B4F85E10401A81B208E0B4F85C108142F9
:10BDE0007FF466AFD069B842FAD126672046FFF7E4
:10BDF0004AFE56E7B4F85C00B4F85E10B4F85E2072
:10BE0000401A81B2002AF4D00029F2D0226852E808
:10BE1000000F20F4907042E80007002FF6D1324F57
:10BE2000206800F1080050E8002F02EA070240E80D
:10BE3000002CBCF1000FF3D1C4F88C30E5666567C7
:10BE4000226852E8000F20F0100042E80003002BA7
:10BE5000F6D1CAE7C60209D5560207D54FF48010BD
:10BE600038622046BDE8F041FFF75CBE06060AD501
:10BE700001F0800602F40002164304D0A16F0029ED
:10BE80007FF408AF0DE7420611D54A060FD52046CC
:10BE9000016851E8002F22F0400241E80024002C04
:10BEA000F6D1C0F88830856700F00EFCF9E6020292
:10BEB00006D54A0004D52046BDE8F041FFF731BE63
:10BEC000C00196D5002994DA2046BDE8F041FFF77D
:10BED000DBBD00000100001020010004C3EE0008DB
:10BEE0001000024010040240FEFFFFEF10B50400F6
:10BEF00003D0D4F8880010B107E0012010BD002065
:10BF000084F88400204600F027F82420C4F8880034
:10BF10002068016821F001010160A06A10B120468B
:10BF200002F016FF204603F0B5F80128E6D020689D
:10BF3000416821F4904141602068816821F02A0124
:10BF400081602068016841F0010101602046BDE880
:10BF5000104002F061BF00002DE9F04FB5B004467B
:10BF600014212EA8F4F799FCB8216846F4F795FC43
:10BF7000FA4D0226FA494FF000082068083DDFF824
:10BF8000DC93770288425DD1002168460222CDF819
:10BF90007480CDE90021FDF7CFF808B1F8F77EFDF8
:10BFA000D9F8001041F48011C9F80010D9F8000048
:10BFB00000F480103390286840F00400286028685E
:10BFC00000F004003390286840F0080028602868DA
:10BFD0000825B146464669022E9100F00800CDE9D9
:10BFE0002F982EA9CDF8C480CDE93250DD48FBF75B
:10BFF000B9FA04212E91CDE92F96DB482EA9CDE97F
:10C000003165FBF7AFFAD94D4121D94828604FF48B
:10C010004030C5E90116C5E903676E61AE61C5E947
:10C02000076028466E62FAF793FB08B1F8F736FD11
:10C03000C4F8805000220521AC633520FBF758FC82
:10C0400035206CE0CB494FF0070A4FF0400B884297
:10C050006AD1002168460222CDF87480CDE9002122
:10C06000FDF76AF808B1F8F719FDD9F8001041F0AA
:10C070008041C9F80010D9F8000000F080403390EA
:10C08000286840F01000286028684FF4C0712E9195
:10C090002EA900F010004546CDE92F68CDF8C480E8
:10C0A000CDE932A0B448FBF75DFADFF8C0824F2338
:10C0B000B24A4FF4803908F17808404688E82C00ED
:10C0C000C0E90357C8F81450C8F81850C8E9075910
:10C0D000C8F82450FAF73CFB08B1F8F7DFFCA34E90
:10C0E0005022C4F88080F036C8F83840A349304662
:10C0F000C6E9035775611831B561C6E9075975621C
:10C1000086E80608FAF724FB08B1F8F7C7FCE667EB
:10C1100000220521B4635220FBF7EAFB5220FBF713
:10C12000DAFB35B0BDE8F08F9549884230D1002068
:10C13000CDF878800121CDE900106846FCF7FCFFBE
:10C1400008B1F8F7ABFC85480830016841F01001F0
:10C150000160006800F010003390286840F0010092
:10C16000286028682EAA4FF4C06100F0010082E820
:10C170004201CDE932A083482EA9CDF8C480FBF757
:10C18000F1F9002205212520FBF7B2FB2520C6E7A7
:10C190007D49884266D1002168460222CDF874802C
:10C1A000CDE90021FCF7C8FF08B1F8F777FCD9F812
:10C1B000001041F40031C9F80010D9F8000000F473
:10C1C00000303390286840F008002860286870210B
:10C1D0002E912EA900F008004546CDE92F68CDF834
:10C1E000C480CDE932A06048FBF7BCF9674E2B2232
:10C1F0005F494FF400383046783186E82600C6E9BA
:10C2000003577561B561C6E907587562FAF7A0FA78
:10C2100008B1F8F743FCDFF874912C23C4F8806070
:10C2200009F17809B4634846514A9032C0E903578E
:10C23000C9F81450C9F8185089E80C08C9E907581A
:10C24000C9F82450FAF784FA08B1F8F727FCC4F8C3
:10C250007C9000220521C9F838402620FBF748FBD6
:10C2600026205CE74A49884276D1002168460222AE
:10C27000CDF87480CDE90021FCF75EFF08B1F8F736
:10C280000DFCD9F8001041F48021C9F80010D9F84C
:10C29000000000F480203390286840F002002860FD
:10C2A000286800F002003390286840F008002860F9
:10C2B00028684FF480412E912EA900F008004546D1
:10C2C000CDE92F68CDF8C480CDE932A03148FBF725
:10C2D00049F94FF440712E91CDE92F6522482EA9DE
:10C2E000CDE9315AFBF73EF9284E2D2220494FF473
:10C2F0000039F0364831304686E82600C6E9035753
:10C300007561B561C6E907597562FAF721FA08B196
:10C31000F8F7C4FB204D2E23C4F88060B463284690
:10C32000134AC5E90387C5F814806032C5F8188040
:10C33000C5E90789C5F8248085E80C08FAF708FAEA
:10C3400008B1F8F7ABFBE56700220521AC632720B5
:10C35000FBF7CEFA2720E2E620E00000E84402588E
:10C360000050004000080258000C0258540D0020F4
:10C3700028000240007800400010025828040240C3
:10C38000001001400000025800440040BC0E002094
:10C390000048004000040258241000203949884217
:10C3A0007FF4BFAE0021CDF8788001226846CDE948
:10C3B0000021FCF7C1FE08B1F8F770FB32480168B4
:10C3C00041F080010160006800F08000339028682F
:10C3D00040F010002860286845462EA900F01000A3
:10C3E000339004202E90CDE92F68DFF8A080CDE9AE
:10C3F00031504046FBF7B6F80B2108202E90CDE9CE
:10C400002F65CDE931512EA94046FBF7ABF8DFF897
:10C41000809077261F4B4FF440384846C0E90357B9
:10C42000C9F81450C9F8185089E84808C9E90758EC
:10C43000C9F82450FAF78CF908B1F8F72FFB144E1D
:10C44000762114487836C4F87C904830C9F83840D2
:10C4500086E82300C6E9035775613046B561C6E931
:10C4600007587562FAF774F908B1F8F717FBC4F8C2
:10C47000806000220521B4639C20FBF739FA9C20E0
:10C480004DE60000001C0140F04402580010025824
:10C490009C100020100402402DE9F84F0446D0F80B
:10C4A0008C009B4616460D46202802D00220BDE88F
:10C4B000F88FC5B1BEB10027C4F890702220C4F82F
:10C4C0008C00E7662034FBF765F9824654F8180CB7
:10C4D000A6874FF48053E687FF21203C984207D17E
:10C4E000226912B119E00120E1E740F2FF1114E0E6
:10C4F0004FF07F0278B1B0F1805F11D0A4F8607086
:10C500009842B4F860704FF0200801D1206970B1F2
:10C510002E4600250CE0266936B9A4F86010EFE736
:10C52000216909B13F21F8E7A4F86020E8E7002677
:10C5300007F0FF09B4F85E00F0B100225346202155
:10C540002046CDF800B002F0E7FF18B1C4F88C80A7
:10C550000320ACE72068406A56B100EA090006F8FB
:10C56000010B00BFB4F85E00401EA4F85E00E1E7D6
:10C57000384025F8020BF5E7C4F88C80002096E7D8
:10C5800030B4D0F88C30202B02D0022030BC704761
:10C59000A9B1A2B10B4D00240368C466AB420BD015
:10C5A0005B681B0208D5046854E8003F43F08063D1
:10C5B00044E80035002DF6D130BC02F059BF01200F
:10C5C000E4E70000000C005810B502F03DFD06281D
:10C5D0000AD000EBC001054800EB8100C0680028CC
:10C5E00002D0BDE81040004710BD00008C9A00202A
:10C5F00010B502F029FD06280AD000EBC00105485D
:10C6000000EB81008068002802D0BDE810400047A0
:10C6100010BD00008C9A00202DE9F8430446D0F8A4
:10C620008800984616460D46202802D00220BDE814
:10C63000F883A5B19EB10021C4F890102120C4F860
:10C6400088001834FBF7A6F8814654F8100CA6872A
:10C65000E6872027183CB0F5805F02D003E0012078
:10C66000E5E7206910B12E46002510E000260EE017
:10C670008021204602F050FFC0B9DEB116F8010B50
:10C6800021688862B4F85600401EA4F85600B4F839
:10C6900056004B464FF00002CDF800800028E7D14D
:10C6A0004FF04001204602F037FF48B1C4F88870CF
:10C6B0000320BCE735F8020B2168C0F30800E0E76F
:10C6C000C4F888700020B2E710B502F0BDFC06285F
:10C6D0000AD000EBC001054800EB8100406800284B
:10C6E00002D0BDE81040004710BD00008C9A002029
:10C6F000FEE70000F0B500230A251C463026372748
:10C7000011E000BFB5EB107F02D906EB107C01E011
:10C7100007EB107C01F813C001EB430C00015B1C1C
:10C720008CF80140DBB29342ECD3F0BD10EE100A5E
:10C730000C49B6EE001AF7EE080A20EE011AA1EB3A
:10C74000600000EE100AF0EE601A21EE002A42EEC0
:10C75000401A21EE800A21EE001A41EE400A20EE36
:10C76000800A7047DF59375F70B51C4615462DEDBE
:10C77000088B93ED011A93ED000AD0ED010A90EDBC
:10C7800000BAB4EE410AF1EE10FAB1EE608A01D0BF
:10C79000B0EE608AD1ED00AAD0ED028A91ED011AC7
:10C7A0002AEE809A2BEE0B0AD1ED020AB1EE41AAD5
:10C7B00008EE080AF1EE609A08EEA80A05F04CFBB4
:10C7C00020EE000A0AEEEA0A05F046FBF0EE40AA67
:10C7D0004FF0FF30F4EE6AAAF1EE10FA49D1B0EE54
:10C7E000CA0AF0EEE90A30EE200AB4EEEA0AF1EEE7
:10C7F00010FA3ED328EE080A08EEA80A09EE490A04
:10C8000005F02AFB28EE891A68EE090A08EE001ADC
:10C8100048EEC00AB0EE410A04F0D6FFB0EE409AEE
:10C82000B0EE6A1AF0EE690AB0EE4A0A06F0ACFD04
:10C83000F0EE40AAB0EE693AF0EE4A2AB0EE682A6D
:10C84000F0EE481AB0EE4B1AF0EE6A0AB0EE490A62
:10C8500006F064FD85ED009AD4ED010A002020EE7B
:10C86000800A85ED010A94ED020A20EE2A0A85ED80
:10C87000020ABDEC088B70BD91ED021A71EE600AE0
:10C8800080EE801A80ED021AD1ED000A60EE800A77
:10C89000C0ED000AD1ED010A80EE801A80ED011A88
:10C8A0000020704790ED021A41EE000AC1ED020A25
:10C8B000D0ED000A80EE801A81ED001AD0ED010A59
:10C8C00020EE800A81ED010A90ED030A81ED030A52
:10C8D00090ED040A002081ED040A704700EB81000E
:10C8E000006E00F0F84070478068C0F3C0007047E9
:10C8F0008068C0F3800070478068C0F38000704794
:10C9000000EB8101034B51F8600F20F00040104311
:10C910000860704700600258D0ED002A32EEC03A3D
:10C92000B0EEC33AB4EEE03AF1EE10FA02DC90ED6C
:10C93000000A0BE0F4EEC02AF1EE10FA02DD30EE50
:10C94000200A01E030EE600A80ED000AB4EEC10A70
:10C95000F1EE10FA02DD80ED001A06E0B4EEE10A15
:10C96000F1EE10FA01D2C0ED001A91ED000AF0EEDE
:10C97000C00AF4EEC20AF1EE10FA0BDDB5EEC00A01
:10C98000F1EE10FA02DD81ED002A03E0B1EE420A79
:10C9900081ED000A0020704738B390ED061AD0ED03
:10C9A000012AF0EE400AD0ED071A41EE620A90ED3E
:10C9B000022A4FF07F4241EEC20A10EE901AB2EB0B
:10C9C000410F01D1F0EE400A90ED040AD0ED032AA8
:10C9D00090ED052A21EE000A80ED071AC0ED060A47
:10C9E00000EEA20A01EE820A70479FED010A70472D
:10C9F0000000000010B504002DED068B18D0F5EEF8
:10CA0000C00A9FED2C1AC4ED000AF1EE10FA84ED75
:10CA1000061AF7EE008A84ED071A0CD8C4ED038AD3
:10CA200084ED041A84ED051A84ED011A80ED021AD2
:10CA3000BDEC068B10BD80EE201ADFED1F0A80EEE4
:10CA4000810A05F027FA9FED1DAAB0EE408AB0EEEC
:10CA50004A0A05F013F8F0EE009AB0EE689A20EE5C
:10CA6000291AB0EE680A68EE080A18EE080A01EE04
:10CA7000089A20EE291A08EE089A80EE890AC1EE7B
:10CA8000090A84ED030A20EE291A84ED050AB0EEA6
:10CA90004A0AC4ED010A84ED041A04F0EFFF20EE07
:10CAA000290A40EE488A48EE088A88EE890A84ED11
:10CAB000020ABDE700000000DB0F4940DB0F493FE1
:10CAC000B8B190ED031AD0ED041AD0ED050A31EE9D
:10CAD000211A31EE201AC0EE010A10EE901A6FEA08
:10CAE000D15111F0FF0F07D0C0ED060AC0ED070AC3
:10CAF00006E09FED040A704780ED060A80ED070A04
:10CB0000FFF74ABF0000000030B58DB00024684632
:10CB1000242109940A940B94F3F7BFFE24480425BA
:10CB2000224B4FF41012012103600223C0E90124BB
:10CB3000C0E90415047603224176C36180F82040E1
:10CB40008462C0E90B42C463046480F84440816499
:10CB5000F8F7C8FD08B1F7F7A1FF154809A909942E
:10CB6000F8F712FA08B1F7F799FF1248062140F2D8
:10CB7000FF7203928DE823000D486946CDE9045405
:10CB80008DF82140F8F794FA08B1F7F787FF0C21E8
:10CB90000948CDE9000106486946F8F789FA0028F6
:10CBA00001D0F7F77BFF0DB030BD00000020024040
:10CBB000880300201000C0100000B84F394808B5A5
:10CBC000016841F001010160016801F0010100917B
:10CBD000016841F00201016000680022052100F0B7
:10CBE000020000900B20FAF783FE0B20FAF773FE89
:10CBF000002205210C20FAF77BFE0C20FAF76BFED1
:10CC0000002205210D20FAF773FE0D20FAF763FECE
:10CC1000002205210E20FAF76BFE0E20FAF75BFECC
:10CC2000002205210F20FAF763FE0F20FAF753FECA
:10CC3000002205211020FAF75BFE1020FAF74BFEC8
:10CC4000002205211120FAF753FE1120FAF743FEC6
:10CC5000002205212F20FAF74BFE2F20FAF73BFE8A
:10CC6000002205213820FAF743FE3820FAF733FE78
:10CC7000002205213920FAF73BFE3920FAF72BFE76
:10CC8000002205213A20FAF733FE3A20FAF723FE74
:10CC9000002205213B20FAF72BFEBDE808403B208F
:10CCA000FAF719BED84402581748002170B5154D3F
:10CCB00001228160182605600225C16020240174CC
:10CCC0000423417481744661C0E906250262426210
:10CCD0008262C262C0E90C210464C0E90E21C0E98D
:10CCE0001131C0E91331C0E91531C0E91714C0E9A9
:10CCF0001913FAF7FFF9002803D0BDE87040F7F7E1
:10CD0000CDBE70BD00A00040700400201848002176
:10CD100070B5164D01220560182581602024C16080
:10CD20000423017441748174C0E90552C26140F268
:10CD30000645026242628262C262C0E90C25046456
:10CD4000C0E90E21C0E91131C0E91331C0E9153144
:10CD5000C0E91714C0E91913FAF7CCF9002803D079
:10CD6000BDE87040F7F79ABE70BD000000A4004017
:10CD7000100500201848002170B5164D01220560ED
:10CD8000182581602024C1600423017441748174DA
:10CD9000C0E90552C26140F6120502624262826237
:10CDA000C262C0E90C250464C0E90E21C0E911315A
:10CDB000C0E91331C0E91531C0E91714C0E91913EE
:10CDC000FAF798F9002803D0BDE87040F7F766BE7F
:10CDD00070BD000000D40040B0050020074A0021CB
:10CDE000074810B505F0D0FD0649074A0860002144
:10CDF000BDE81040054805F0C7BD000030490108F6
:10CE000049E1000800000020504B010831E700080C
:10CE10002DE9F04F87B014216846F3F73EFD5E48D8
:10CE2000016841F010010160016801F010010591F5
:10CE3000016841F004010160016801F004010591FD
:10CE4000016841F080010160016801F080010591F5
:10CE5000016841F001010160016801F001010591E3
:10CE6000016841F002010160016801F002010591D1
:10CE7000016841F00801016000684FF46044DFF888
:10CE80001C81002200F00800214605904046FAF778
:10CE90007CFC012240462921FAF777FC4FF400463A
:10CEA0003F4800223146FAF770FC4FF440693D4894
:10CEB00000224946FAF769FC4FF4805A39480122AA
:10CEC0005146FAF762FC4FF4806B3748002259460E
:10CED000FAF75BFC012569464046CDE90045002490
:10CEE00002940394FAF73EFB032769462920CDE913
:10CEF0000005CDE902474046FAF734FB4FF48818A5
:10CF000069464FF4A0500294CDE900082448FAF78E
:10CF100029FB00966946CDE9015421480394FAF7AC
:10CF200021FBCDF800906946CDE901541D480394DA
:10CF3000FAF718FB1B486946CDE900A5CDE9025771
:10CF4000FAF710FBCDF800B06946CDE90154164858
:10CF50000394FAF707FB2802144D02218DE8130011
:10CF60006946284603940494FAF7FCFA0096694649
:10CF7000CDE901842846FAF7F5FA0021A802FEF768
:10CF800027F9002205212820FAF7B2FC2820FAF719
:10CF9000A2FC07B0BDE8F08FE04402580008025838
:10CFA0000010025800040258000C025800000258F9
:10CFB00070B586B018216846F3F76FFC1848082250
:10CFC000164D0021012417238160D606E0E80352A4
:10CFD000032580E81A0000F11403C0E9031483E874
:10CFE00062000162C0E90912C16201630C48FAF7EC
:10CFF000C1FE08B1F7F752FD4FF0011041F288323F
:10D0000069460094CDE902400548FAF7A3FC0028E0
:10D0100001D0F7F743FD06B070BD000000A000523C
:10D02000500600202DE9F0414FF480051448134AC2
:10D0300007276E114FF0007C2C0180E8E4100021DE
:10D04000A300C0E90514C0E9073141629A0081627A
:10D05000C162C0E90D21C163016441648164C1649E
:10D06000016541658165FDF795FB002803D0BDE8AA
:10D07000F041F7F713BDBDE8F0810000003001403A
:10D08000AC0600202DE9F04117484FF48007DFF887
:10D0900054C00021FA000726C0F800C01301C0E9FF
:10D0A0000362C0E90171C0E90731416255105400C3
:10D0B00081625201C162C0E90D21C1630164416412
:10D0C0008164C164016541658165C0E90554FDF76E
:10D0D00061FB002803D0BDE8F041F7F7DFBCBDE8F5
:10D0E000F0810000003800403407002010B58AB0FD
:10D0F000002468461C21079408940994F3F7CDFB9B
:10D10000164840F2CF711722134BC0E90241046167
:10D110008461C0E90032FEF73AFB08B1F7F7BEFCC4
:10D120000E4807A907940994FEF7AEF808B1F7F77F
:10D13000B5FC60206946CDE9000408480422029449
:10D140000494FEF792FA08B1F7F7A8FC0348FEF73B
:10D150001FFA0AB010BD000000180040900900201E
:10D1600010B598B000241C210DA8149415941694A1
:10D17000F3F793FB34216846F3F78FFB2748182217
:10D18000254942F2107380E81600C0E90334446177
:10D190008461FEF7FCFA08B1F7F780FC1F4814A978
:10D1A000149415941694FEF76FF808B1F7F776FC0F
:10D1B0000DAA41F28831602082E81300174800224E
:10D1C0000DA91094119412941394FEF74EFA08B11D
:10D1D000F7F764FC114808220DA9FEF746FA08B1DA
:10D1E000F7F75CFC4FF400500094039401030194A2
:10D1F000CDE904400294CDE9084108486946069407
:10D200000A940C94FDF7F0FF08B1F7F747FC0348C8
:10D21000FEF7BEF918B010BD00000140AC080020B8
:10D2200010B58AB0002468461C210794089409941C
:10D23000F3F733FB1A4842F2107118224FF0804383
:10D24000C0E9024104618461C0E90032FEF79FFA3F
:10D2500008B1F7F723FC124807A907940994FEF7D1
:10D2600013F808B1F7F71AFC602041F288318DE815
:10D2700013000B48002269460494FEF7F6F908B142
:10D28000F7F70CFC064808226946FEF7EEF908B1EC
:10D29000F7F704FC0248FEF77BF90AB010BD000066
:10D2A000F808002030B58BB0002468461C21079494
:10D2B00008940994F3F7F1FA164842F20F72172313
:10D2C000134D8021C0E9024204618161C0E900532D
:10D2D000FEF75DFA08B1F7F7E1FB0E4807A90794DE
:10D2E0000994FDF7D1FF08B1F7F7D8FB6020694634
:10D2F000CDE9000407480C2202940494FEF7B5F926
:10D3000008B1F7F7CBFB0348FEF742F90BB030BD8D
:10D31000000400404409002070B518480021164C54
:10D32000042300F10C0C164D22158CE80E008161CF
:10D33000A614C16101624162816280E87000FEF75B
:10D34000D5FD08B1F7F7AAFB0C480021FEF7C3FB97
:10D3500008B1F7F7A3FB09480021FEF796FB08B1D7
:10D36000F7F79CFB0548FEF76EFB002803D0BDE8ED
:10D370007040F7F793BB70BD00500040DC090020FF
:10D38000A08601001848002110B5164C0C224FF45D
:10D3900061230460C0E90131C160C0E90412816108
:10D3A000C161016241628162FEF7A0FD08B1F7F739
:10D3B00075FB0D480021FEF78EFB08B1F7F76EFBF9
:10D3C00009480021FEF761FB08B1F7F767FB064843
:10D3D000FEF739FB002803D0BDE81040F7F75EBB2D
:10D3E00010BD000000780040700A0020184800219D
:10D3F00010B5164C0C224FF461230460C0E90131D2
:10D40000C160C0E904128161C1610162416281624F
:10D41000FEF76CFD08B1F7F741FB0D480021FEF760
:10D420005AFB08B1F7F73AFB09480021FEF72DFB3C
:10D4300008B1F7F733FB0648FEF705FB002803D0D9
:10D44000BDE81040F7F72ABB10BD0000001C0140EA
:10D45000C00C00201848002110B5164C0C224FF4C7
:10D4600061230460C0E90131C160C0E90412816137
:10D47000C161016241628162FEF738FD08B1F7F7D0
:10D480000DFB0D480021FEF726FB08B1F7F706FB60
:10D4900009480021FEF7F9FA08B1F7F7FFFA064844
:10D4A000FEF7D1FA002803D0BDE81040F7F7F6BA2E
:10D4B00010BD000000100140040B0020184800219E
:10D4C00010B5164C0C22174B0460C0E90131C16045
:10D4D0000B46C0E9041281610A46C16101624162E2
:10D4E0008162FCF7E3FF08B1F7F7D8FA0C48002196
:10D4F000FEF7F1FA08B1F7F7D1FA09480021FEF773
:10D50000C4FA08B1F7F7CAFA0548FEF79CFA0028F2
:10D5100003D0BDE81040F7F7C1BA10BD0044004089
:10D52000980B002000093D001848002110B5164C4A
:10D530000C22174B0460C0E90131C1600B46C0E901
:10D54000041281610A46C161016241628162FCF795
:10D55000ADFF08B1F7F7A2FA0C480021FEF7BBFABD
:10D5600008B1F7F79BFA09480021FEF78EFA08B1D7
:10D57000F7F794FA0548FEF766FA002803D0BDE8ED
:10D580001040F7F78BBA10BD004800402C0C00206B
:10D5900000093D0010490122104810B502F042FC7C
:10D5A00008B1F7F77BFA0E490C4802F05AFE08B1B1
:10D5B000F7F774FA0B49094802F0DAF908B1F7F7FE
:10D5C0006DFA064802F0D2FE08B1F7F767FABDE837
:10D5D0001040FBF761BA000008000020D8110020BD
:10D5E000E800002068000020FEE770B505000C464A
:10D5F00031D0002C2FD020781022287204F11F0186
:10D6000060786872A078A872E078E8722079287350
:10D61000B4F805002882D4F807006861D4F80B003C
:10D62000A861D4F80F00E861D4F81300A862D4F818
:10D6300017006862D4F81B00286205F12C00F3F78C
:10D640008BF8D4F82F002864D4F83300686494F879
:10D65000370085F8480070BD00F07AB810B520B1E9
:10D660007821F3F71AF9002010BD6FF0010010BD0A
:10D6700010B50D4C207810B16FF0020010BD05F010
:10D6800081F9A06068B10321084A0846F5F732FE27
:10D69000074A04210320F5F72DFE01202070002009
:10D6A00010BD6FF0010010BDD401002079D7000833
:10D6B00059D6000870B504000D4604D02248017800
:10D6C000FC2907D102E06FF0010070BD90F837002F
:10D6D000FD2806D01D484168491C41604FF0FF30CD
:10D6E00070BD19492046FFF780FF04F1200004F1C6
:10D6F0005C0304F1680607C883E8070004F114001E
:10D700000C3B07C883E8070004F12C000FC886E82B
:10D710000F0094ED190AD5ED000A002030EE200A22
:10D7200084ED190A94ED180AD5ED010A30EE200AAD
:10D7300084ED180AD5ED020A94ED170A30EE200A9E
:10D7400084ED170A70BD000025000024D4010020DC
:10D75000032010B5F5F78EFD0068016821F0010186
:10D7600001600320F5F786FD0068016841F00101C2
:10D770000160002010BD000002481021806805F003
:10D780007BB80000D4010020032010B5F5F772FD2E
:10D7900004493822FEF7F4FE002801D04FF0FF3094
:10D7A00010BD000025000024C8220121102010B562
:10D7B00005F09CF8102801D0002010BD012010BDFC
:10D7C000FEE70000F0B503004FF0000004460BD068
:10D7D000022B09D841B100220A604A60022B8A60FC
:10D7E000CA600A6102D007E00120F0BD294A126830
:10D7F000D20734D04FF40074274D002205EB82038A
:10D80000D3F80434DE0707D003F0020604F0020761
:10D81000BE4201D1561C0E60DE0607D503F020067D
:10D8200004F02007BE4201D1561C4E60DE0507D52C
:10D8300003F4007604F40077BE4201D1561C8E60DA
:10D84000DE0311D503F4802604F48027BE420BD1F9
:10D850009E0302F1010604D446F4803603E00F4C27
:10D86000CAE746F08076CE60DE010FD503F0806611
:10D8700004F08067BE4209D19B0102F1010302D48A
:10D8800043F4803301E043F080730B61521C022AA1
:10D89000B4D3F0BD00B4005200B000522202040420
:10D8A0002DE9F041984616460F460446069D08E0CD
:10D8B000681C06D0F9F76EFFA0EB0800A8420AD852
:10D8C0004DB12068006A384000D00120B042EFD14D
:10D8D0000020BDE8F0814FF400702065606D40F0DD
:10D8E000010060650120F4E70148FAF7CFBC0000B1
:10D8F000D42800202DE9F041044680790D462027E8
:10D90000236801284FF4004604F29C4203EB4511C2
:10D91000D3F840C0D1F8080B09D0DFF89CE0F445FB
:10D920003AD1020433D500BFC1F8086B40E0234B65
:10D930005FEA007E04D59C453AD90004F4D437E070
:10D940005FEA806E02D5C1F8087B31E010F0280F45
:10D950002ED19C4501D90004E6D4D1F8101B05EB6B
:10D96000C50004EB8000C1F31201D0F87432A3EBC0
:10D970000101C0F8681200F51570ADB903691BB15B
:10D98000C2681144C1600FE0206801210AE08006EE
:10D990000AD5C1F8087B07E035B9D4F8640218B994
:10D9A0000021184603F062F82046E9B2FAF757FB67
:10D9B0000020BDE8F08100000A31544F0A30544F76
:10D9C0002DE9F84F0E460568814601EBC60100EBD4
:10D9D0008104D4E909201434904202D90120BDE821
:10D9E000F88FA168101A814200D20846C01C05EBCE
:10D9F000461887081BE000BFA268A0EB010A524549
:10DA000000D2924699F806100AF1030000911FFA1D
:10DA10008AF3E16887082846F2B203F06BFBE168FD
:10DA200001EB0A00E060616901EB0A006061D8F86F
:10DA3000180980B2B84205D3D4E90401814201D269
:10DA40000028D9D1D4E90401884208D8D5F834187F
:10DA5000012006F00F0290408143C5F834180020E1
:10DA6000BDE7000010B504462DED068BF0EE409AA0
:10DA7000F0EE618AB0EE418AB0EE609A19EE900A3B
:10DA800003F078FB002850D019EE100A03F072FB67
:10DA900000284AD0B0EE480A10EE100A03F06AFBE4
:10DAA000002842D018EE900A03F064FBE8B36068E7
:10DAB000F0EE490AB0EE690A90ED071AF6F731FC6C
:10DAC0006068F0EE409AD0ED000A04F11C0020EEF0
:10DAD000891A20EEA99AB0EE410AFEF75DFF207880
:10DAE000DFED38AAB0EE40AA70B101280ED1D4ED16
:10DAF000020AB0EE680A04F069F8D4ED050A7AEE7D
:10DB0000600A80EE808A01E0B0EE6A8A18EE100AA0
:10DB1000C4ED049A84ED05AA6FEAD05010F0FF0F0F
:10DB200001D1B0EE6A8A606800E047E0D4ED030AF4
:10DB300090ED010AD0ED031A49EE280A20EE090AF9
:10DB400090ED021A204A11EE101A08EE610A21EE39
:10DB5000201A91421CDD10EE901A6FEAD15111F09B
:10DB6000FF0F15D070EE011A90ED052AF0EEE11AC4
:10DB7000F4EEC21AF1EE10FA0AD890ED042AF0EE93
:10DB8000E01AF4EEC21AF1EE10FA01D8C4ED030A5D
:10DB900030EE010A10EE101A6FEAD15111F0FF0FAA
:10DBA0000CD0D0ED050A10EE900A904201DDF4F79A
:10DBB000C7FF84ED060ABDEC068B10BD94ED060A86
:10DBC000F9E7000000000000BD37863570B504009D
:10DBD0000D464FF0FF3137D050686FEAD05010F04B
:10DBE000FF0F31D090686FEAD05010F0FF0F2BD0AC
:10DBF000D0686FEAD05010F0FF0F25D010696FEA9F
:10DC0000D05010F0FF0F1FD050696FEAD05010F0C5
:10DC1000FF0F19D0B7EE001A6260C1EE000A10EED5
:10DC2000900A6FEAD05010F0FF0F0DD0C4ED020A39
:10DC3000D2ED060A04F11C00FEF7DCFE204625703A
:10DC400000F004F8002070BD084670BD10B570B13A
:10DC50009FED080A80ED030A80ED040A80ED050AB5
:10DC600080ED060A1C30FEF72BFF002010BD4FF0A0
:10DC7000FF3010BD00000000F7EE000AB0EE081AF9
:10DC800070EEC00A60EE004A10B590ED002A60EE1A
:10DC9000811A20EEA04A24EE801AD1ED003A61EEFE
:10DCA000A04A64EE200A21EE804AD2ED002A64EEFA
:10DCB000801A20EE822A24EE000A93ED003A029C9C
:10DCC00001EEA32A00EE222A01EE032A84ED002AA7
:10DCD00090ED012AD1ED013A92ED013A20EE822A2F
:10DCE000D3ED012A01EEA32A00EE032A01EE222A37
:10DCF00084ED012AD0ED023A91ED023AD2ED022AEA
:10DD000060EEA30A93ED022A41EE830A40EE220A56
:10DD100041EE020AC4ED020A10BD70EEC00A00EE28
:10DD2000810A704791ED001AD0ED000A31EE601AB9
:10DD300041EE000AC2ED000A91ED011AD0ED010A90
:10DD400031EE601A41EE000AC2ED010A91ED021AAD
:10DD5000D0ED020A31EE601A41EE000AC2ED020A6D
:10DD6000704700002DE9F047454D044689464FF0C5
:10DD7000000A2868C04380070AD0414E283E306818
:10DD800020F080603060F9F705FD0746B04608E0F6
:10DD90000120BDE8F08700BFF9F7FCFCC01B02289A
:10DDA00067D8D8F800000001F6D4206829684FF43D
:10DDB000FE0721F47C313E0241EA00302860207ADF
:10DDC000A389B4F804C040022D4D2D495B1E227C6E
:10DDD000ACF1010C1035091DA0F5007080B2521E87
:10DDE000CCF3080C07EA034340EA0C00184306EAA8
:10DDF0000262104328600868626920F0C000104386
:10DE000008600A68A06922F0200202430A60281D07
:10DE10000A6822F010020A6002684FF6F873E4699B
:10DE20009A4342EAC40202600868B9F1000F40F068
:10DE300010020A6011D00868B9F1010F11D040F446
:10DE400000100860D8F80000444640F08060C8F830
:10DE50000000F9F79FFC05460DE0086840F400203B
:10DE6000EFE740F48010ECE7F9F794FC401B022840
:10DE700001D903208DE720680001F5D5504688E7D9
:10DE8000284402582DE9F047454D044689464FF095
:10DE9000000A2868C04380070AD0414E283E3068F7
:10DEA00020F080503060F9F775FC0746B04608E076
:10DEB0000120BDE8F08700BFF9F76CFCC01B022809
:10DEC00067D8D8F800008000F6D4208829684FF47D
:10DED000FE0721F07C713E0241EA00502860207A62
:10DEE000A389B4F804C040022D4D2D495B1E227C4D
:10DEF000ACF1010C1835091DA0F5007080B2521E5E
:10DF0000CCF3080C07EA034340EA0C00184306EA86
:10DF10000262104328600868626920F44060104380
:10DF200008600A68A06922F4007202430A60281D92
:10DF30000A6822F480720A6002684FF6F873E46996
:10DF40009A4342EAC40202600868B9F1000F40F443
:10DF500080720A6011D00868B9F1010F11D040F049
:10DF600080700860D8F80000444640F08050C8F83F
:10DF70000000F9F70FFC05460DE0086840F480004A
:10DF8000EFE740F40000ECE7F9F704FC401B02283F
:10DF900001D903208DE720688000F5D5504688E739
:10DFA000284402580148FCF7E3BA00003407002077
:10DFB00010B5026840F26F335169946944F0080467
:10DFC00094610268946944F01004946102681468D2
:10DFD00024F001041460026814699C43146102680F
:10DFE000936823F44043936090F88120042A0CD076
:10DFF0008A060AD5D0F8842042F08002C0F8842036
:10E000000268936943F02003936190F88120032A0A
:10E010000CD04A060AD5D0F8842042F00402C0F899
:10E0200084200268936943F0400393618A050AD50E
:10E03000D0F8842042F00102C0F88420026893697D
:10E0400043F400739361C9050AD5D0F8841041F0F8
:10E050000801C0F8841001688A6942F480728A61FC
:10E060000021A0F86210A0F86A1010BD10B5806BF6
:10E0700000210122A0F86A10A0F8621080F8812027
:10E08000FCF75AFA10BD10B5846BF7F7EBFF0228C6
:10E090000ED02046FFF78CFFD4F88410012041F009
:10E0A0001001C4F8841084F881002046FCF744FA7B
:10E0B00010BD10B5806BFCF71FFF10BD10B5806B55
:10E0C00090F88110072909D0C16FC969B1F5807F27
:10E0D00005D00068016941F00801016110BDFCF73D
:10E0E000EFFE10BD00680349884201D1002070474F
:10E0F00002207047003800402DE9F0411C461646CA
:10E100000D460746DDF818800AE000BFF9F742FB2C
:10E11000A0EB0800A04202D3601C01D00BE054B178
:10E120003868406935EA000007D00020B042EDD0E1
:10E130000020BDE8F0810320FBE70120F6E701782D
:10E14000407841EA0020704710B5FFF723FA04F049
:10E1500019FCBDE8104004F05FBC4FF0E02010B5A2
:10E16000006906F0B9F8012803D0BDE8104005F0B9
:10E1700077BC10BD70B59CB04C216846F2F78DFBA2
:10E18000202113A8F2F789FB0220FAF75BFC224852
:10E19000016821F4404101600168002401F440411C
:10E1A0001B9101688904FCD502204025C30323226A
:10E1B0000121CDE90023CDE903152822099006911C
:10E1C00004230D910C260A90CDE90B02CDE90E3007
:10E1D000CDE9106468461294FBF7D4FE08B172B61C
:10E1E000FEE708221A95CDE91625D30113AA3F2090
:10E1F0000321CDE9185382E8130013A8FBF73AFC7A
:10E2000008B172B6FEE700214FF480220846FBF702
:10E210006FFE1CB070BD0000184802582D48F0B5C4
:10E220002D4A016841F470010160106800F00F0090
:10E23000072804D2106820F00F00C01D1060274985
:10E240000020264C10340B68254D43F001030B6071
:10E2500020600B682B400B60136803F00F03072B43
:10E2600004D9136823F00F03DB1D13601B4C1D4AF8
:10E2700018341D4B261D371D2060184C1B4D2834AB
:10E280003060261D3860371D23603B1D35601C1D26
:10E290003A60251D2E1D1860331D226028603260F3
:10E2A00018600B680D4A0D4C23F48023D4320B60A8
:10E2B000603420601068C0040BD4136843F2D200AD
:10E2C0000B4943F4805313600860106820F48050B9
:10E2D0001060F0BD88ED00E00020005200440258BC
:10E2E0007FEDF6EA80020101000202020000FF0158
:10E2F000004000520148FDF7A6B800008C11002034
:10E300002DE9F0472C4B4FF0804A2C4D0268984283
:10E310002B4E2C4F2C4C09D0504507D0A84205D08D
:10E32000B04203D0B84201D0A04205D1D1F804C018
:10E3300022F070024CEA0202DFF890C0DFF8908011
:10E340009842DFF8909015D0504513D0A84211D0D4
:10E35000B0420FD0B8420DD0A0420BD0604509D0DA
:10E36000404507D0484505D01B4DA84202D01B4D63
:10E37000A84203D1CD6822F440722A438E684D69C9
:10E3800022F08002C6620E682A439842866207D055
:10E39000A04205D0604503D0404501D0484501D199
:10E3A000096901630368012143F0040303604161CB
:10E3B0000260BDE8F087000000000140000400405A
:10E3C00000080040000C00400004014000400140F3
:10E3D000004401400048014000E0004000E40040EB
:10E3E00010B5046A012301F01F018B409C430462B5
:10E3F0008A40016A1143016210BD00002DE9F04F0F
:10E40000DFF88480214EDFF88890DFF888B0026A58
:10E41000036AB042DFF880A022F0020C1F4F23F005
:10E4200001020262426885698B680C6805EA08058A
:10E4300025F0030543EA0C0344EA050407D04845E8
:10E4400005D0584503D0504501D0B84205D1CD681C
:10E4500023F008031D4325F00403B04207D04845CC
:10E4600005D0584503D0504501D0B84205D122F41B
:10E470004076D1E9055235432A43426084614968B8
:10E4800041630362BDE8F08F8FFFFEFF0000014093
:10E4900000040140004001400044014000480140A8
:10E4A000F0B5DFF87CE01F4C1F4D026A036AA04202
:10E4B00022F0200623F01003036242688369D1F83A
:10E4C00008C00F6803EA0E0323F4407E46EA0C13EB
:10E4D0004EEA072601D0A84206D1CF6823F0800378
:10E4E00043EA071323F04003A0420AD0A84208D011
:10E4F0000E4CA04205D00E4CA04202D00D4CA042C2
:10E5000007D1D1E9054522F4406242EA840242EA99
:10E51000850242608661496881630362F0BD000044
:10E52000FF8FFFFE00000140000401400040014059
:10E530000044014000480140F0B5DFF87CE01F4D89
:10E540001F4E026A036AA84222F4007723F4807304
:10E5500003624368C269D1F808C002EA0E020C687F
:10E5600022F0030E47EA0C2244EA0E0401D0B04226
:10E5700006D1CF6822F4006242EA072222F48062C8
:10E58000A8420AD0B04208D00E4DA84205D00E4D88
:10E59000A84202D00D4DA84207D1D1E9055623F477
:10E5A000405343EA051343EA06134360C4614968D4
:10E5B000C1630262F0BD00008FFFFEFF000001405A
:10E5C0000004014000400140004401400048014077
:10E5D000F0B5046A026A22F4805202624268C3699A
:10E5E00024F40054DFF848C08E680D6803EA0C0379
:10E5F000104F23F4407344EA0634B84243EA05233B
:10E600000BD00D4DA84208D00C4DA84205D00C4DA2
:10E61000A84202D00B4DA84204D14D6922F4804299
:10E6200042EA85124260C361496801640462F0BD38
:10E63000FF8FFFFE00000140000401400040014048
:10E640000044014000480140F0B5164F164B026AE5
:10E65000046A984222F4003524F48033036242684D
:10E66000436D0E890C6803EA070344EA030445EA94
:10E6700006430BD00D4DA84208D00D4DA84205D041
:10E680000C4DA84202D00C4DA84204D14D6922F491
:10E69000803242EA0522426044654968816503622E
:10E6A000F0BD00008FFFFEFF0000014000040140AC
:10E6B000004001400044014000480140F0B5164FC1
:10E6C000164B026A046A984224F48013036222F40F
:10E6D00000144268436D0E890D6803EA070344EA9B
:10E6E000065443EA05230BD00D4DA84208D00D4D2A
:10E6F000A84205D00C4DA84202D00C4DA84204D12E
:10E700004D6922F4802242EA8522426043654968CD
:10E71000C1650462F0BD0000FF8FFFFE00000140F4
:10E720000004014000400140004401400048014015
:10E73000314810B5F5F712FE03F0AAFF2F4A002169
:10E740002F4804F021F92C4C00212E4A483C20602F
:10E750002D4804F019F9606000212C4A2C4804F07F
:10E7600013F9A06000212B4A2B4804F00DF9E0605A
:10E7700000212A4A2A4804F007F920610021294A89
:10E78000294804F001F960610021284A284804F072
:10E79000FBF8A0610021274A274804F0F5F8002281
:10E7A000E0611821022003F0F5FF002260622021C1
:10E7B000022003F0EFFF0022E0629021022003F02C
:10E7C000E9FF00222063F021022003F0E3FF002292
:10E7D00060630C21022003F0DDFF002220620C2187
:10E7E000022003F0D7FFA06303F084FF04F0CAF80F
:10E7F000BDE8104004F010B998A20020744B010845
:10E8000011EC0008984B01083DE80008BC4B0108DA
:10E8100091EC0008E04B010849E90008044C0108AC
:10E82000F1EB0008284C010849EA00084C4C0108AB
:10E8300075EB0008704C0108C1EA0008002003F0E5
:10E84000D5FE3E4C94F8AC0110B1012817D10EE072
:10E850003B4901F11800F4F7BFF939481830F4F7D3
:10E860009BF937483749B030F3F77EFD07E034486D
:10E870003830FEF7FDFE01210220F4F7C3FC94F8C6
:10E88000AC0198B10128FAD12D483830FEF77CFF51
:10E89000FEF78AFFC0B303F0FBFE29490C3101F1FA
:10E8A0002C00FEF707FF03F025FF32E0F4F7FAFA39
:10E8B000F4F760F9F4F76AF9F4F77CF9F4F786F9FC
:10E8C00003F0E6FE1E481830F4F71EFA1C48183014
:10E8D000F4F76AFA1A4A1B4B2432A2F10C0101F137
:10E8E0009800F3F7D1FD1649B03101F11400F3F7A8
:10E8F000D3FC03F0FFFE206A03F0ACFF10490023B5
:10E90000206A1A46C43116E0FFE70D483830FEF79A
:10E91000A5FE206A03F09EFF09490023206A1A46DB
:10E9200094310D4603F062FFA06B03F093FF0023C8
:10E93000A06B1A46294603F059FFA0E750A2002019
:10E9400048A4002078030020002003F04FFE274851
:10E95000F6F728FA26A0F4F7DDFC33A0F4F7DAFC8A
:10E96000334F0026334C00BFF4F7F8FC0500FBD012
:10E97000014631A0F4F7CEFC0D2D10D00A2D0ED09B
:10E980007F2D2AD0082D28D020887F28ECD2202D5A
:10E99000EAD37E2DE8D83D54411C2180E4E727A02E
:10E9A000F4F7B8FC20883E5480B1F6F78FF94FF4A5
:10E9B000007980461E484A464146F6F78BF90546DF
:10E9C00041461FA0F4F7A6FC002DF3D11848802182
:10E9D0002680F1F740FF14A005E020880028C3D06E
:10E9E000401E208017A0F4F795FCBDE7944C010869
:10E9F0000D0AE6ACA2E8BF8EE4BDBFE794A8E5919E
:10EA0000BDE4BBA4E8A18CEFBC8CE8BE93E585A572
:10EA10002068656C7020E69FA5E79C8BE591BDE4BE
:10EA2000BBA40D0A000000006D723E200000000033
:10EA300018A5002084030020256300000D0A0000B3
:10EA400025730000082008002DED028B03F00BFE5B
:10EA50004FF4FA71B0FBF1F6002003F0C7FD154842
:10EA6000F4F7CCFC03F0F8FD124F0546134C9FED74
:10EA7000128A354403F00CFE0E490023606A1A46E0
:10EA8000303103F055FE30B90A49B0EE480A01F1C1
:10EA90003000F4F7B9FC03F02DFEE06A03F0DAFE73
:10EAA0000023E06A391D1A4603F0A0FE284603F051
:10EAB000ABFDDEE798A500206F12033B50A20020BB
:10EAC00003F0D1FD4FF4FA71B0FBF1F6C82003F06A
:10EAD0008DFD244924489FED220AF5F721FB03F020
:10EAE000BBFD204C05464C3C2049002335441A46CA
:10EAF000206B03F01DFE18B91C491B48F5F7DCFB21
:10EB00001A490023A06B1A460C3903F011FE20B9F4
:10EB1000164915480C39F5F7F1FB00231449E06A52
:10EB20001A4603F005FE03F0B3FD11492A460E48CC
:10EB3000F4F7BAFC0D490C489031F5F7CBFA03F025
:10EB4000D9FD606B03F086FE08490023606B1A460E
:10EB5000903103F04BFE284603F056FDC4E7000059
:10EB60000000FA439CA2002060A700206CAA0020AD
:10EB7000ECAB002003F077FD4FF44871B0FBF1F6E9
:10EB8000C82003F033FD17491748F6F733F903F0AF
:10EB900063FD144D0446483D1449002334441A468D
:10EBA000686B03F0C5FD18B910490F48F6F79EF9D8
:10EBB00003F06EFD0C48F6F73DF903F09BFD0B49A1
:10EBC00009489039F6F7BEF9286B03F043FE074970
:10EBD0000023286B1A46903903F008FE204603F004
:10EBE00013FDD9E798A200206000002470A6002041
:10EBF00003F039FD6421B0FBF1F5002003F0F6FCD1
:10EC000003F02AFD04462C44204603F0FDFCFAE7FD
:10EC1000002003F0EBFC1A48F5F71AFEDFED190AA5
:10EC20009FED190AF4F7DEF9184C1548F5F7D0FEF8
:10EC30001420F5F7DDFE0028114807D0F5F72CFE6B
:10EC400001210020F4F7DEFA012106E0F5F7F6FDD8
:10EC500000210846F4F7D6FA00210120F4F7D2FA91
:10EC6000074907481831F5F741FE606A03F0F2FDE5
:10EC700003490023606A1A46183103F0B7FDD4E750
:10EC800020A20020CDCC4C3E0000964350A2002094
:10EC900003F0E9FC3221B0FBF1F5002003F0A6FC03
:10ECA000F4F72EFAB6EE000A40F20510F4F7E0F998
:10ECB000B6EE000A40F24910F4F7DAF9B6EE000AAF
:10ECC0004FF4C470F4F7D4F9F4F726FA03F0C4FC57
:10ECD00004462C44204603F097FCFAE7044810B59C
:10ECE000FCF736FFBDE810400148F4F7E1BA000038
:10ECF000DC090020044810B5FCF72AFFBDE81040ED
:10ED00000148F4F7D5BA0000700A002030B5416E12
:10ED1000B9B101680D4B03F108048A688968C2F330
:10ED20004262490F5D5C615C2D01B5FBF1F1A0F819
:10ED30006A10995CA25C0901B1FBF2F1A0F86810BD
:10ED400030BD0121A0F86A10F8E70000D0490108A1
:10ED500090F82810090706D50168836B4A6822F4E9
:10ED600000421A434A6090F82810C90706D001688B
:10ED7000C36A4A6822F400321A434A6090F82810A5
:10ED8000890706D50168036B4A6822F480321A436A
:10ED90004A6090F82810490706D50168436B4A6815
:10EDA00022F480221A434A6090F82810C90606D53A
:10EDB0000168C36B8A6822F480521A438A6090F813
:10EDC0002810890606D50168036C8A6822F400526F
:10EDD0001A438A6090F82810490611D50168436CDF
:10EDE0004A6822F480121A434A60416CB1F5801FD0
:10EDF00006D10168836C4A6822F4C0021A434A6053
:10EE000090F82810090606D50168C26C486820F4FD
:10EE100000201043486070472DE9F8430025044660
:10EE2000C0F89050F8F7B6FC8046206820266FF0B6
:10EE30007E470068000713D5002243463104204670
:10EE4000009700F069FB58B1216851E8000F20F0ED
:10EE5000800041E80002002AF6D1C4F8886021E071
:10EE600020680068400722D5002243464FF4800105
:10EE70002046009700F050FBC8B1206850E8001F02
:10EE800021F4907140E80012002AF6D12068083081
:10EE900050E8001F21F0010140E80012002AF5D1DE
:10EEA000C4F88C60032084F88450BDE8F883C4F86B
:10EEB0008860C4F88C60E5662567002084F884507B
:10EEC000F3E710B5806B0021A0F85E10FCF72CFE74
:10EED00010BD70B5846B00252168D4F88800D4F883
:10EEE0008C608968090606D5212804D1A4F85650FB
:10EEF000204600F091F820688068400606D5222E52
:10EF000004D1A4F85E50204600F05CF8D4F89000DC
:10EF100040F01000C4F890002046FCF705FE70BDDC
:10EF200010B5C1690022806BB1F5807F2DD0A0F8AB
:10EF30005E20036853E8001F21F4807143E8001449
:10EF4000002CF6D10168083151E8003F23F001039D
:10EF500041E80034002CF5D10168083151E8003F48
:10EF600023F0400341E80034002CF5D12021C0F803
:10EF70008C10C16E012908D1016851E8003F23F0CF
:10EF8000100341E80034002CF6D10267C16E01295C
:10EF900002D0FDF719FB10BDB0F85C10FCF773FD53
:10EFA00010BD10B5806B01210167C16E012902D02F
:10EFB000FDF71EFB10BDB0F85C104908FCF763FDBF
:10EFC00010BD000010B5026852E8001F21F49071D6
:10EFD00042E80013002BF6D10E4B0268083252E8CB
:10EFE000001F194042E80014002CF6D1C16E01291F
:10EFF00008D1026852E8001F21F0100142E8001316
:10F00000002BF6D100212022C0F88C20C166416778
:10F0100010BD0000FEFFFFEF026852E8001F21F064
:10F02000C00142E80013002BF6D10168083151E815
:10F03000002F22F4000241E80023002BF5D120210B
:10F04000C0F888107047000000680D49884201D15F
:10F05000002070470B49884201D1012070470A49BE
:10F06000884201D1022070470849884201D103201B
:10F0700070470749884201D1042070470620704735
:10F08000005000400044004000480040001C014087
:10F09000007800402DE9F04304468068E24E87B0D6
:10F0A000E24B2168D4E90427D4F81CC010430A6855
:10F0B000002547EA0C073843324002430A602068C3
:10F0C000E268416821F44051114341602268A1691E
:10F0D0009A4201D0206A01439668DFF854C3D54FA5
:10F0E000D54806EA0C060E4396602168666ACA6A2D
:10F0F00022F00F023243CA622268BA420ED100687F
:10F1000000F0380018286FD07ADCB8B308286CD02B
:10F1100010286BD18BE0282868D18EE0C7498A423D
:10F1200009D1006800F0070006285FD2DFE800F090
:10F13000507D7F818385C2498A4209D1006800F0F1
:10F14000070006287BD2DFE800F0437072747678FF
:10F15000BC498A4209D1006800F0070006286ED237
:10F16000DFE800F036636567696BB7498A420BD107
:10F17000006800F00700062861D200E043E0DFE805
:10F1800000F0275456585A5CB0498A4206D10068AC
:10F1900000F0380018284CD0B7DD31E0AC498A4285
:10F1A00009D1006800F00700062848D2DFE800F027
:10F1B000103D3F414345A7498A420BD1006800F00A
:10F1C000070006283BD2DFE800F00330323436383F
:10F1D000002035E0A0498A4209D1006800F03800DB
:10F1E000182826D091DD0BE023E01EE027E09B49A4
:10F1F0008A420AD1006800F03800182819D084DD4E
:10F20000202888D11CE001201AE09A4217D18A48B0
:10F21000001D006800F00700062810D2DFE800F0AB
:10F22000030507090B0D02200AE0042008E008206E
:10F2300006E0102004E0202002E0402000E08020D2
:10F240008749DFF820829A42874A4FF400434FEA09
:10F2500021174FF000064ED110281AD006DC0228E4
:10F2600009D004280BD008287ED10DE020283ED0FC
:10F27000402879D13DE0F9F717FC014610E06846D7
:10F28000F9F7C8FC01990BE003A8F9F765FD0499AB
:10F2900006E01068800605D51068C0F3C100C140C3
:10F2A000002970D0606A676838F8102007EB4703C0
:10F2B000B1FBF2F0834257D8B0EB073F54D800239C
:10F2C00008461946F1F74CF902467808130E120267
:10F2D00043EA012110183A4671410023F1F740F941
:10F2E000624AA0F5407191423ED821688FE03946CC
:10F2F000D8E71946D6E7D4F81CC04FF6EF799C45FD
:10F3000046D1082819D005DC58B101280CD00428B2
:10F3100075D10DE0102815D0202835D040286ED1A9
:10F3200034E0FAF725FD01E0FAF734FD014610E07C
:10F330006846F9F76FFC01990BE003A8F9F70CFD9B
:10F34000049906E01068800604D51068C0F3C10077
:10F35000C140C1B1636A606838F81330B1FBF3F1A2
:10F36000490001EB500100E049E0B1FBF0F0A0F1F1
:10F370001001494543D84FF6F0732168C0F34202AB
:10F380001840104343E043E03946E3E71946E1E71C
:10F39000082819D005DC58B101280CD004282ED13A
:10F3A0000DE0102815D020282BD0402827D12AE0A6
:10F3B000FAF7DEFC01E0FAF7EDFC014610E06846E2
:10F3C000F9F728FC01990BE003A8F9F7C5FC0499AB
:10F3D00006E01068800604D51068C0F3C100C14083
:10F3E000B1B1636A606838F81330B1FBF3F101EB37
:10F3F0005001B1FBF0F0A0F11001494505D90125FC
:10F4000006E03946EDE71946EBE7216880B2C860AF
:10F410000120A4F86A00A4F8680028466667A66779
:10F4200007B0BDE8F0830000F369FFCF000C00587F
:10F43000FFF4FF1100100140544402580044004002
:10F4400000480040004C00400050004000140140C3
:10F4500000780040007C004000180140001C014082
:10F460000090D003B849010800440258FFFC0F0087
:10F4700070B50446D0F8800000232225A165A4F8C9
:10F480005C20C4F89030C4F88C50F0B11F49C163BF
:10F49000D4F880101E480864D4F880101D48C86451
:10F4A000D4F8800003651346A56D2168D4F8800068
:10F4B0002A462431F7F72AFB38B11021C4F89010FE
:10F4C0002020C4F88C00012070BD206940B1216863
:10F4D00051E8000F40F4807041E80002002AF6D1A4
:10F4E0002068083050E8001F41F0010140E8001298
:10F4F000002AF5D12068083050E8001F41F0400193
:10F5000040E80012002AF5D1002070BD21EF00086C
:10F51000A3EF0008D3EE00082DE9F04799461746FF
:10F520000D460446089E4FF0000833E0701C31D0B1
:10F53000F8F730F9A0EB0900B04218D8BEB1206846
:10F540000168490726D5802D24D0402D22D0C169DD
:10F55000C94309070DD4082505622046FFF732FD8F
:10F56000C4F89050012084F88480BDE8F08703201F
:10F57000FBE7C069C04300050CD421684FF400606C
:10F5800008622046FFF71EFD2021C4F8901084F881
:10F590008480ECE72068C06935EA000004D00020D0
:10F5A000B842C3D00020E0E70120F9E7044810B5D5
:10F5B000FCF7CEFABDE810400148F3F779BE000031
:10F5C000C00C0020044810B5FCF7C2FABDE810409A
:10F5D0000148F3F76DBE0000040B0020044810B58D
:10F5E000FCF7B6FABDE810400148F3F761BE000031
:10F5F000980B0020044810B5FCF7AAFABDE81040AB
:10F600000148F3F755BE00002C0C00202DE9F04115
:10F610000C46D0F8D412D0F8C83200EB8101D1F8F2
:10F62000C01229B304F00F02002702EB820500EBA1
:10F630008506B5694DB102EBC20203EB8202D269C5
:10F64000B5FBF2F302FB1352A2B1C1F81472D0F869
:10F65000D42200EB8200D0F8C40203692BB1D1F8A8
:10F66000080201F50471224698470020BDE8F081A8
:10F670000320FBE7002321461A46B76100F0D3FDC3
:10F68000F3E770B50546D0F8D40205EB8000D0F85A
:10F69000C04294B1284600F0A0FCC4F80C02D5F892
:10F6A000D40205EB8000D0F8C412D4F80402CA6872
:10F6B00004F503719047002070BD032070BD000069
:10F6C00070B5224D0446297800F0C8FB2878002642
:10F6D00000F00F0000EB800004EB800086842046E1
:10F6E000697800F0BBFB687800F00F0000EB800049
:10F6F00004EB8000A0F864612046A97800F0AEFB1E
:10F70000A87800F00F0000EB800004EB80008684F6
:10F71000C684D4F8D40204EB8000D0F8C01299B1AA
:10F72000D0F8C40240688047D4F8D40204EB8000CB
:10F73000D0F8C00200F09FFFD4F8D40204EB8000A0
:10F74000C0F8C062C4F8BC62002070BD9400002004
:10F7500010B5D0F8D41200EB8100D0F8C04284B1CB
:10F76000D0F8C41259B194F80002FF2807D08B6872
:10F77000214694F801229847FF2084F800020020D7
:10F7800010BD032010BD00000A2101800048704711
:10F790009800002070B5822106460D4800F076FAE8
:10F7A000012105460A4800F071FA81210446084803
:10F7B00000F06CFA0DB11021A9714FF0400104B1B5
:10F7C000A18000B1818043203080014870BD0000DD
:10F7D000A400002070B5822106460D4800F056FABC
:10F7E000012105460A4800F051FA812104460848E3
:10F7F00000F04CFA0DB11021A9714FF4007104B161
:10F80000A18000B1818043203080014870BD00009C
:10F81000A400002070B5822106460D4800F036FA9B
:10F82000012105460A4800F031FA812104460848C2
:10F8300000F02CFA0DB11021A9714FF0400104B174
:10F84000A18000B1818043203080014870BD00005C
:10F85000A40000202DE9F0474FF407750446284620
:10F8600000F00AFF06004FF0000965D02946F1F7C5
:10F8700014F8D4F8D40201273C4D4FF4007A4FF02D
:10F88000100804EB8000C0F8C062C4F8BC62207CA1
:10F89000F0B3297840230222204600F00EFC28789D
:10F8A000402300F00F0000EB800004EB8000878411
:10F8B00002226978204600F000FC697808230322C0
:10F8C000204601F00F0101EB810104EB8101A1F859
:10F8D0006471A97801F00F0101EB810104EB810152
:10F8E000A1F82680A97800F0E8FBA978C84601F0C5
:10F8F0000F0101EB810104EB81018F84C6F80492B2
:10F90000D4F8D40204EB8000D0F8C402006800E010
:10F910001AE006F501768047C6F81080C6F8148014
:10F9200032687AB1207CF8B140236978204600F033
:10F93000D0FB0020BDE8F087D4F8D41204EB81019D
:10F94000C1F8C0920220F5E72978022253462046EA
:10F9500000F0B3FB2878534600F00F0000EB800066
:10F9600004EB80008784A3E75346DEE79400002081
:10F9700039B1D0F8D42200EB8200C0F8C4120020C4
:10F98000704703207047D0F8D42200EB8200D0F8F3
:10F99000C00218B1C0F8041200207047032070475D
:10F9A000D0F8D43200EB8300D0F8C00228B1C0F800
:10F9B0001022C0F8081200207047032070472DE97C
:10F9C000FC410646D0F8D4020C46002106EB80002C
:10F9D0000D46D0F8C0728DF80010ADF8041037B1A4
:10F9E000217811F060022CD0202A48D102E00320B7
:10F9F000BDE8FC81E288E2B109060BD5D0F8C4026B
:10FA00003946836860789847E288072A00D9072238
:10FA100039462CE0607887F80002E088402800D35F
:10FA200040203946C2B2304687F8012200F07FF804
:10FA30002AE0D0F8C4020022214683686078984703
:10FA400022E0607830B101281ED00A2809D00B28A6
:10FA500015D110E096F89C02032810D1022201A9CA
:10FA600005E096F89C02032809D101226946304638
:10FA700000F077F808E096F89C02032804D02146AD
:10FA8000304600F049F803252846B1E710B5D0F814
:10FA9000D41200EB81020121D2F8C0221AB1D2F8AF
:10FAA000143213B116E0032010BD0B490123C2F834
:10FAB0001432D2F81032097801F00F0404EB8404F8
:10FAC00000EB8404A361D2F81032D2F8082200F0CF
:10FAD000AAFB0021084610BD9400002010B5D0F804
:10FAE000B82200245268904700B10324204610BD7C
:10FAF000002070470020704713460A46002110B5C9
:10FB000000F0E7FA002010BD13460A46002110B5A8
:10FB100000F089FB002010BD10B58021044600F0E4
:10FB200063FB2046BDE81040002100F05DBB10B52E
:10FB3000C0F858210323C0F89432C0F85C21134662
:10FB40000A46002100F0C5FA002010BD10B50521BD
:10FB5000C0F8941200231A46194600F0BAFA0020A1
:10FB600010BD10B582610223C0F89432C261134601
:10FB70000A46002100F057FB002010BD10B50421FB
:10FB8000C0F8941200231A46194600F04CFB0020DE
:10FB900010BDF8B504460D460020ADF800004888B9
:10FBA000010A062947D006DC01290FD0022912D00C
:10FBB000032962D11DE0072946D00F295DD1D4F871
:10FBC000B402C26920E0694690473BE0D4F8B41221
:10FBD000207C0A68F7E7207C02260028D4F8B802C7
:10FBE00005D0C16A684688470146467036E0816A9A
:10FBF000F8E7C0B2062840D2DFE800F003090D1193
:10FC00001519D4F8B4024268B2B3207CDBE7D4F80B
:10FC1000B4028268F8E7D4F8B402C268F4E7D4F812
:10FC2000B4020269F0E7D4F8B4024269ECE7D4F810
:10FC3000B4028269E8E7207CF0B9D4F8B802416BDD
:10FC400068468847014609E0207CA8B9D4F8B80284
:10FC5000016B68468847014607204870EA888AB1E8
:10FC6000BDF8000040B1824200D902462046ADF8FE
:10FC70000020FFF776FFF8BDFFE729462046FFF793
:10FC80004BFFF8E72046FFF779FFF4E778B54288A5
:10FC90000D460178002604468A4212D9ADF80010BC
:10FCA0000AE0694600F019F84178052904D1817805
:10FCB0000646A94205D000266188BDF80020914281
:10FCC000EFD8304678BD002102E0491C401CC9B283
:10FCD0000278002AF9D1084670470A8803781A4446
:10FCE0000A8001780844704770B5002816460D4612
:10FCF00020D00446FFF7E7FF02220146100202EB84
:10FD00004101814204D82046FFF7DDFF4000801CFE
:10FD100030803378032102202B700022697006E0C6
:10FD2000431C2954D8B2411C641C2A54C8B22178FF
:10FD30000029F5D170BD01004FF0000004D0012969
:10FD400001D0022901D00320704701207047000034
:10FD500004A00A46024910B5FFF7C6FF004810BDCF
:10FD6000B414002043444320436F6E66696700006B
:10FD700012200880004870472C00002004A00A468A
:10FD8000024910B5FFF7B0FF004810BDB4140020C1
:10FD900043444320496E74657266616365000000E8
:10FDA00004200880004870472800002004A00A466C
:10FDB000024910B5FFF798FF004810BDB4140020A9
:10FDC0004D526F626F74000004A00A46024910B5DC
:10FDD000FFF78AFF004810BDB41400204D726F6217
:10FDE0006F7420436C69000010B51A2008800B481E
:10FDF0000A490830021F096800681468081809D009
:10FE000007490822FCF776FC0549042220461031F8
:10FE1000FCF770FC0248801E10BD000000E8F11FD6
:10FE20004E00002078B10023C0F8B832C0F8C432C8
:10FE3000C0F8D03209B1C0F8B4120121027080F8C4
:10FE40009C1200F0CFB80320704710B5D0F8C8025C
:10FE5000F8F747F9BDE81040FFF76DBF10B5D0F8CF
:10FE6000C802F8F719F9BDE81040FFF764BF2DE9A3
:10FE7000F041174604464FF0000521B194F89C026A
:10FE8000032842D04CE0D4F8941204F11400022963
:10FE900035D1D0E902639E4206D9F21A3946826012
:10FEA0002046FFF731FE0FE0B34214D1406898427C
:10FEB00011D3D4F8981288420DD200222046114660
:10FEC000FFF722FEC4F8985200231A46194620462E
:10FED00000F0FFF813E094F89C02032808D1D4F84E
:10FEE000B802C16821B1C4F8D452C168204688471D
:10FEF0008021204600F078F92046FFF727FE94F88D
:10FF0000A00268B184F8A0520AE0D4F8B8024269AD
:10FF100032B1C4F8D452426920469047002800D13B
:10FF20000020BDE8F08170B5134604464FF0000292
:10FF300021B194F89C02032830D03AE0D4F894120E
:10FF400004F5AA70032934D1D0E902518D420AD9AF
:10FF50006A1A82600846824200D302461946204649
:10FF6000FFF7CAFD25E094F8AA0210F01F0003D0A5
:10FF7000012802D0022800D0002294F89C02032815
:10FF800008D1D4F8B802016921B1C4F8D4220169BA
:10FF9000204688472046FFF7F1FD0AE0D4F8B80272
:10FFA000836933B1C4F8D42282692046904700287F
:10FFB00000D1002070BD0020704710B5D0F8B812F5
:10FFC000012280F89C22002429B103794A68D9B221
:10FFD000904700B10324204610BDD0F8C802F8F7BE
:10FFE000ADB8000070B50178012929D1154909255E
:10FFF000154C02230022C1F8E004C0F8C8120846DC
:020000040801F1
:100000000C600D71CB718A714B728A72CA720A735D
:100010008A73CA730A74F8F70BFC08B1F4F73EFD53
:1000200008484FF40071F7F7E6FF064880220021E8
:10003000F7F7E5FF034801214FF4BA72F7F7DFFF46
:10004000002070BDD428002000000440D0F8C82251
:1000500001F07F000B0600EBC00002EB800001D531
:10006000807D704790F85602704710B5D0F8D422C2
:1000700000EB8202D2F8B82222B190F89C32032B16
:1000800002D004E0032010BD126A02B190470020A4
:1000900010BD10B5D0F8D42200EB8202D2F8B822FD
:1000A00022B190F89C32032B02D004E0032010BD53
:1000B000526A02B19047002010BD10B51C46D0F81E
:1000C000C80213462246F8F742F8BDE81040FFF791
:1000D00032BE10B5D0F8C802F8F76AF8BDE8104093
:1000E000FFF729BE2DE9F041044601250020D4F890
:1000F000B812064684F89C52C4F894026060C4F8B2
:10010000A40284F8A00231B14A6822B1002120463D
:10011000904700B103262046002240231146FFF7F6
:10012000CCFF4027A4F8645100223B4680212046A2
:10013000C4F86071FFF7C1FFA58430462762BDE8AF
:10014000F08190F89C12042903D190F89D1280F858
:100150009C120020704710B590F89C12032905D11D
:10016000D0F8B81211B1C96901B18847002010BD9B
:1001700001740020704710B5D0F8C802F8F70EFCE3
:10018000BDE81040FFF7D7BD70B5044600F2AA20C5
:10019000054600F051F894F8AA020123B4F8B01211
:1001A00010F01F02C4F89432C4F898120AD0012A41
:1001B0000ED0022A12D000F080012046BDE8704027
:1001C00000F012B829462046BDE8704000F0D0B8D3
:1001D00029462046BDE8704000F013BA2946204663
:1001E000BDE8704000F05BB910B5D0F8C802F7F771
:1001F000F9FFBDE81040FFF79EBD10B5D0F8C8026A
:10020000F8F7E6FBBDE81040FFF795BD90F89C12AB
:10021000042903D090F89C1280F89D12042180F8E4
:100220009C120020704710B5D0F8C802F8F713F8F8
:10023000BDE81040FFF77FBD70B5054608788C1CFF
:100240002870487868702046FDF779FFA41C688004
:100250002046FDF774FFA880A01CFDF770FFE88022
:1002600070BD38B504460020ADF80000A1B1C4F857
:10027000B812D4F8D40204EB8000D0F8B802C16AF6
:1002800019B168468847C4F8D002D4F8D802401C97
:10029000C4F8D802002038BD032038BDD0F8B832E9
:1002A00002460020002B02D01B68104618477047FA
:1002B0002DE9F0412C4E0446887800258846C1B2CD
:1002C0000129317006D941462046FFF725FC03205D
:1002D000BDE8F08194F89C02022702280CD0032884
:1002E0001DD041462046FFF717FC31782046FFF726
:1002F000F5FB03252846EBE789B320466160FFF74D
:10030000CDFF050004D041462046FFF705FC1DE067
:100310002046FFF733FC032084F89C02EAE7C1B1D2
:10032000606888421BD0C1B22046FFF7D7FB317806
:1003300020466160FFF7B2FF050010D0414620461D
:10034000FFF7EAFB21792046FFF7C8FB84F89C728F
:10035000D0E7616084F89C722046FFF7BFFB20461F
:10036000FFF70CFCC6E7000090000020FFF745BF38
:100370002DE9F0410A784FF0000512F060020CD030
:10038000202A01D0402A7DD1D0F8D42200EB82026D
:10039000D2F8B8229268904731E04B7800220126CB
:1003A0000A2B6FD2DFE803F041666E586E08056EC7
:1003B0002D29FFF7EEFB67E004468888D8B9C88886
:1003C000C8B94888802816D294F89C2200F07F078C
:1003D000032A10D03946204684F89E72FFF7CBFEE0
:1003E0002046FFF7CBFB1FB1022084F89C024BE0B4
:1003F00084F89C6248E0204644E0FFF759FF054638
:1004000042E0CB88012B3DD190F89C32012B04D0E7
:10041000022B02D0032B35D104E000F108018260E9
:10042000012216E00122011D13E090F89C22012A0E
:1004300003D0022A01D0032A24D1CA88022A21D15A
:10044000D0F8A412C66009B10321C160022200F1F4
:100450000C01FFF786FB17E04A88012A02D0022A26
:1004600003D00FE0C0F8A46216E08988090A80F87A
:10047000A01211E090F89C32012B08D0022B06D07C
:10048000032B04D0FFF748FB2846BDE8F0814988DC
:100490000129F9D1C0F8A422FFF770FBF4E72DE998
:1004A000F0410A780E460979054612F060004FF0D7
:1004B0000008CCB20BD0202801D040286AD12146B8
:1004C0002846FFF715FBFF2800D0D8B396E07078D8
:1004D000C8B3012824D003285CD195F89C020228D7
:1004E00002D0032856D10CE0002C53D0802C51D0E0
:1004F00021462846FFF778FE80212846FFF774FE44
:100500007CE0708840B93CB1802C05D0F08818B9E7
:1005100021462846FFF768FE2846FFF72FFB6DE0CF
:1005200095F89C020228DFD0032863D1708880BB35
:10053000600603D021462846FFF787FC2846FFF7D0
:100540001DFBBCE700E00AE0C5F8D402D5F8B8020C
:100550008268F2B131462846904780464EE095F8D1
:100560009C020027022802D0032843D113E00CB1DB
:10057000802C3FD1200604F07F0000EB800005EBCB
:10058000800101D5143101E001F5AA7102220F604A
:100590002CE033E02EE0200604F00F0000EB80009A
:1005A00005EB800009D5808C20B304F07F0000EBC0
:1005B000800005EB800614360AE0B0F86401C8B18B
:1005C00004F07F0000EB800005EB800606F5AA76BC
:1005D0004CB1802C07D021462846FFF737FD10B1DB
:1005E0000120306000E03760022231462846FFF7E4
:1005F000B8FA03E031462846FFF78EFA4046BDE8D8
:10060000F08170B5054608780E464FF0000410F0F2
:10061000600003D0202801D0402827D195F89C0203
:10062000012803D0022801D003281FD1B088C1B20D
:1006300001291AD8C1B22846FFF75CFAFF280CD06E
:1006400058B9D5F8B8128A683AB1C5F8D402284624
:100650008A6831469047044600E00324F08820432E
:1006600007D12846FFF78AFA03E031462846FFF70C
:1006700053FA204670BD704700487047B4260020EA
:1006800070B54D7801230A78012D1C4C02F00F053E
:1006900003FA05F3D0F81C5817D000EB421245EAD4
:1006A0000343C0F81C38D2F8000B00040BD40B89AC
:1006B0000979D2F8000BC3F30A03184344EA8141D5
:1006C0000843C2F8000B002070BD9EB23543C0F84D
:1006D0001C5800EB4213D3F800090004F3D40D8931
:1006E0000979D3F80009C5F30A058904284341EACA
:1006F000825108432043C3F80009E4E7008000105A
:10070000D0F800196FF30A01C0F80019D0F80418E6
:1007100041F48071C0F804180020704770B50D4690
:100720000446C2F307211E460498012922D0E0683E
:1007300040F04000E060204600F03CF8C6F307219E
:100740000029A16B2ED021F48031A163C5F30741AC
:1007500001290ED1E16D154A89B2E165E16D1143C0
:10076000E165A16841F00601A160A16841F02001A6
:10077000A16070BDA26BC3B20D49012B22F4803081
:10078000A063E06800EA0100E060E06820F4401047
:10079000E06003D1E06840F48010E060204600F0A3
:1007A00009F8D3E741F48031CFE700000000EE0301
:1007B000BFFFBDFF08B500214FF070620091009BA4
:1007C0005B1C009393420CD80369002BF7DA00916D
:1007D000016941F0010101610099491C00919142B8
:1007E00001D9032008BD0169C907F5D1002008BD62
:1007F00070B50A7801234C78012C00EB42122CD002
:10080000D2F8004B002C0BDAD2F8004B44F0006415
:10081000C2F8004BD2F8004B44F08044C2F8004BC1
:100820000C78D0F83C5804F00F0403FA04F425EADD
:100830000444C0F83C480978D0F81C4801F00F0186
:100840008B401C4924EA0343C0F81C38D2F8000B43
:100850000840C2F8000B002070BDD2F80049002CFF
:100860000BDAD2F8004944F00064C2F80049D2F82B
:10087000004944F08044C2F800490D78D0F83C4863
:1008800005F00F050C4E03FA05F5ADB2AC43C0F808
:100890003C48D0F81C48097801F00F018B4099B210
:1008A0008C43C0F81C48D2F800093040C2F8000957
:1008B000D1E700000078F3EF007833ECD0F8001EA9
:1008C00021F00301C0F8001ED0F8041821F0020145
:1008D000C0F8041800207047D0F8001E21F0030172
:1008E000C0F8001ED0F8041841F00201C0F8041846
:1008F000002070472DE9F04F00250F469046044632
:100900002E46284604EB8001C1F80451401C0F28F4
:10091000F8D3C3F307405FEA0009204610D0806B8C
:1009200040F40011C4F83810C8F30720C4F8005E82
:100930000128204617D0D0F8001841F0030119E033
:10094000D0F8040840F00201C4F80418A06B20F4A9
:100950000011A163206840F040012160206840F050
:1009600080012160E0E7D4F80018380E204601D05D
:1009700041F00101C0F80018102100F08CFA00B11C
:100980000126204600F06BFA00B101264FF67F3AAF
:100990004FF0006CC4F810584FF0904BC4F8145846
:1009A000C4F81C580020FAB214E000BF04EB401158
:1009B000D1F80039002B06DA10B1C1F800B904E013
:1009C000C4F800C901E0C1F80059C1F81059C1F8D4
:1009D00008A9401C8242E9D8002013E004EB401132
:1009E000D1F8003B002B06DA10B1C1F800BB04E0DF
:1009F000C4F800CB01E0C1F8005BC1F8105BC1F89E
:100A000008AB401C8242E9D8D4F81008C7F307426B
:100A1000002A6FF0804120F48072C4F81028A5618C
:100A2000616103D1A06940F01000A061A069C8F322
:100A30000741094A1043A06119B1A06940F00800BC
:100A4000A061B9F1010F03D1A06904490843A06175
:100A50003046BDE8F08F000000383C8004000040C4
:100A6000816821F0010181600020704710B5144CAD
:100A7000036CA34203D9D0F8003B002B1EDB0023FC
:100A8000C0F8103B0129D0F8101B41F40021C0F838
:100A9000101BD0F8101B41F01801C0F8101BD0F843
:100AA000101B41F0C041C0F8101B07D1C0F8142B37
:100AB000D0F8001B41F08021C0F8001B002010BDC1
:100AC0000A30544F0B784A78012A00EB43100BD0C0
:100AD000D0F8002B22F40012C0F8002B097903296A
:100AE00014D0022912D017E0D0F8002922F4001205
:100AF000C0F800290979032901D002290CD1D0F8C6
:100B0000001941F08051C0F8001905E0D0F8001B31
:100B100041F08051C0F8001B002070470A784B78E4
:100B2000D1B2012B00EB421012D0D0F8002B002ADA
:100B300006DB29B1D0F8001B21F08041C0F8001B72
:100B4000D0F8001B41F40011C0F8001B00207047D2
:100B5000D0F80029002A06DB29B1D0F8001921F0CD
:100B60008041C0F80019D0F8001941F40011C0F814
:100B70000019EBE7F8B50B786FF060464F788C4DB5
:100B8000DCB2012F00EB43132BD0D3F8107B002CE9
:100B900007EAC544C3F8104BD3F8104B04EA050428
:100BA000C3F8104B7ED00D69002D7CD08C68254495
:100BB0006D1EB5FBF4F5ADB26C430C6206EAC5459B
:100BC000D3F8104B2C43C3F8104BD3F8104B0D6ADD
:100BD000C5F3120554EA0504C3F8104B012A73D07B
:100BE000CEE00F6907B3D3F810796FF31207C3F89B
:100BF0001079D3F8107907EA0507C3F810791CB308
:100C0000D1F810C08D68D3F81079AC44ACF1010C68
:100C1000BCFBF5F5ADB206EAC5463743C3F810791B
:100C20000E79012E1CD02AE0D3F810692E40C3F8AB
:100C30001069D3F8105945F40025C3F81059D3F8BA
:100C400010596FF3120520E00E698D68AE4200D98D
:100C50000D61D0F8106946F40026C0F810690EE066
:100C6000D3F810694FF0C04707EA457726F0C04631
:100C7000C3F81069D3F810593D43C3F810590E69F1
:100C8000D3F81059C6F312063543C3F81059012A98
:100C90001BD000EB4413D3F8004944F00444C3F8DC
:100CA000004901E047E05AE00C79012C2ED00A6996
:100CB0005AB30B78D0F83418012203F00F039A408E
:100CC0001143C0F8341871E056E0CA691AB100EB5C
:100CD0004413C3F81429097901290ED1D0F8081852
:100CE000C90500EB4411D1F8002902D442F00052AA
:100CF00001E042F08052C1F8002900EB4410D0F826
:100D0000001941F00441C0F800194FE0D0F808483C
:100D1000E405D3F8004902D444F0005401E044F063
:100D20008054C3F8004900920B8A0A78C9689BB2C4
:100D300000F0E0F93AE00C690CB18C680C618C6849
:100D40000C62C4F31205D0F8104B2C43C0F8104BC2
:100D5000D0F8104B44F40024C0F8104B3EE78D68E7
:100D6000D3F8104BC5F312052C43C3F8104BD3F83E
:100D7000104B44F400242FE7CA680AB1C3F8142BBF
:100D8000097901290CD1D0F80808C005D3F8000B67
:100D900002D440F0005001E040F08050C3F8000B56
:100DA000D3F8000B40F00440C3F8000B0020F8BD5E
:100DB000FFFF07E038B5002242F2107400230092D2
:100DC0000A784D78012D00EB421219D0D2F8005B61
:100DD000002D3CDAD2F8005B45F00065C2F8005BFC
:100DE0000A7800EB4212D2F8005B45F08045C2F869
:100DF000005B009A521C0092A24221D9012326E0F6
:100E0000D2F80059002D22DAD2F8005945F00065D9
:100E1000C2F800590A7800EB4212D2F8005945F0A6
:100E20008045C2F80059009A521C0092A242E5D8AF
:100E30000A7800EB4212D2F80029002AF3DB06E020
:100E40000A7800EB4212D2F8002B002AD1DB1846B8
:100E500038BD816841F0010181600020704708B50C
:100E600000214FF070620091009B5B1C0093934245
:100E70000AD80369002BF7DA009110230361009967
:100E8000491C0091914201D9032008BD0169C9069E
:100E9000F5D4002008BD18B500224FF07063009211
:100EA000009C641C00949C420CD80469002CF7DA66
:100EB0002024009244EA811101610099491C0091AB
:100EC000994201D9032018BD01698906F5D4002093
:100ED00018BDD0F8080810F0060004D0022803D08E
:100EE000062801D00F20704702207047406900F0AB
:100EF00001007047D0F81818D0F81C08084080B2DC
:100F00007047D0F81818D0F81C080840000C70473B
:100F100010B5D0F8102801F00F0300EB4114D0F801
:100F20003418D4F80809D94001F0010142EAC1118E
:100F3000084010BD00EB4111D1F8081BD0F814088F
:100F40000840704741698069084070470346084679
:100F500030B5940802F00301002203F5805303E04A
:100F60001D68521C40F8045BA242F9D300290CD042
:100F70001C680023491EDD00090403F10103090C6C
:100F800024FA05F200F8012BF4D130BD70B5044607
:100F9000C06801294FF0000520F0C040E06001D09A
:100FA00079B120E0E06840F00050E0600A20F5F7F9
:100FB000FBFE60690A3510F0010F10D1C82DF5D382
:100FC0000DE0E06840F08040E0600A20F5F7ECFEBC
:100FD00060690A3510F0010F01D0C82DF5D3C82D76
:100FE00001D0002070BD012070BDD0F800284FF462
:100FF000FE6303EA011322F4FE62C0F80028D0F871
:1010000000181943C0F8001800207047022A3ED18A
:10101000264A274B0A449A4201D20F2138E0254A3A
:10102000254B0A449A4201D20E2131E0234A244B37
:101030000A449A4201D20D212AE0224A224B0A4454
:101040009A4201D20C2123E0204B214A0B449342C7
:1010500001D20B211CE01F4B1F4A0B44934201D2CB
:101060000A2115E01D4B1E4A0B4493420FD31D4B22
:101070001D4A0B44934201D2082109E01B4B1C4A34
:101080001944914201D2072102E0062100E0092122
:10109000C2684FF4705322F47052C26003EA812395
:1010A000C1681943C160002070470000405327FF0A
:1010B00000350C00401E1BFF40420F0000DC0BFF00
:1010C000804F1200808CF9FE20D6130060B6E5FE3A
:1010D00060E3160000D3CEFE40771B00C05BB3FE7A
:1010E000C091210000CA91FE20753800E05459FEDD
:1010F000E09C410010B5029C74B900EB0232DB1C8D
:1011000000209B0802F5805204E000BF51F8044B18
:101110001460401C9842F9D3002010BDFEE703B4D0
:1011200001984100009850EAC12018BF04204A0DE0
:1011300018BF40F0010040F2FF72B2EB515F08BFF0
:1011400040F00200012808BF052002B070474100AE
:10115000080218BF04200A0E18BF40F001004FF02B
:101160007F4232EA010108BF40F00200012808BFB7
:10117000052070476FEAD05010F0FF0000D001202A
:101180007047090700284FEA116104DB00F1E020F5
:1011900080F80014704700F00F0000F1E02080F8A4
:1011A000141D704710B510EE104A4FF01A402DED87
:1011B000028B00EB4400B0F1C85F4AD84FF0FC400E
:1011C000B0EB440F22D2B0EEC00ADFED310A30EEB0
:1011D000C00ADFED300A20EE208A18EE100A02F075
:1011E000FDF800EE100A14F0004F1DBF9FED2A1A03
:1011F000DFED2A0AB1EE400A9FED291A08BFF0EE92
:10120000410ADFED281A20EE210A05E020EE008ACF
:101210009FED251ADFED250ADFED251A9FED252A22
:1012200070EEC00A20EE080A08EE212ADFED221A2D
:1012300048EE021A9FED212A08EE212ADFED201A3E
:1012400048EE021ABDEC028B40EE610A30EE810AD4
:1012500010BD4FF0CC40B0EB440F82BF9FED190A98
:10126000BDEC028B10BD4FF07F40B0EB440F05D2B8
:10127000BDEC028BBDE8104000F016BF0120EFF777
:1012800066FBBDEC028BBDE8104000F013BF000010
:101290000000803F0000003F0000494022AA7D3A44
:1012A00000000000000000C00000C93F22AAFD3974
:1012B00024FE1C3DC78AD83C1E67383D1B93993DD0
:1012C000AFAA2A3EDB0FC93F10B54FF00E402DEDFF
:1012D000028BB0EE408A18EE104A00EB4400B0F1E9
:1012E000506F4AD84FF0FC40B0EB440F22D2B0EE22
:1012F000C80ADFED360A30EEC00ADFED350A60EECF
:10130000208A18EE900A02F069F801EE100A14F033
:10131000004F1DBFDFED2F0A9FED2F0AB1EE411ADE
:10132000DFED2E0A08BF9FED2E0ADFED2E1A21EE0B
:10133000218A05E0DFED2C0A68EE088AB0EE600A2B
:101340009FED2A1ADFED2A1A30EE080A48EE811ABC
:101350009FED281A08EEA11ADFED271A48EE811A30
:101360009FED261A08EEA11A68EE281ABDEC028B32
:1013700001EE810A30EE200A10BD4FF0E440B0EBE0
:10138000440F0CD918EE100AFFF7E1FE042808BF3D
:1013900000F098FEB0EE480ABDEC028B10BD4FF095
:1013A0007F40B0EB440F07D2B0EE480ABDEC028B91
:1013B000BDE8104000F078BE0120EFF7C8FABDECA0
:1013C000028BBDE8104000F075BE00000000803FB9
:1013D0000000003F0000C9BF22AAFDB90000C93FBC
:1013E00022AAFD39000000C00000000024FE1C3DC0
:1013F000C78AD83C1E67383D1B93993DAFAA2A3E49
:1014000070B565482DED020B2DED048B059D25F083
:101410000044A04218DC6148844202DC0AD10498EE
:1014200040B19DED040BBDEC048B02B0BDE87040F3
:1014300000F028BE002DCCBF9FED590B9FED5A0B3D
:10144000BDEC048B02B070BD5948A04215DD59486F
:10145000A042D8BF4FF0FF3455DD9DED040B51EC99
:10146000100BFFF75CFE042808BF00F011FE9DED95
:10147000040BBDEC048B02B070BD9DED040B51EC70
:10148000100B00F095FFCDE904014B489FED4C0B8C
:10149000A0421CDD4C48A0420BDD9DED042B002436
:1014A0009FED4B1B12EE010B32EE011B80EE012B68
:1014B00027E09DED041B9DED042B012431EE401B24
:1014C00032EE000B81EE002B8DED042B1BE0424829
:1014D000A0420FDD9DED042B02249FED411B9DEDED
:1014E000043B32EE412B03EE010B82EE001B8DED2F
:1014F000041B08E09DED040B9FED3B1B032481EED4
:10150000002B8DED042B9DED040B3948062120EEB8
:10151000009B29EE098BB0EE480B784400F07AFD71
:1015200020EE099B3348B0EE480B0521784400F0CB
:1015300071FD20EE080B002C0BDA9DED042B39EE2B
:10154000001B9DED040BBDEC048B02B002EE410BC1
:1015500070BD2948784439EE000B00EBC4009DEDC6
:10156000042B90ED001B254812EE001B9DED040B93
:1015700031EE400B784400EBC400002D90ED001BD1
:1015800031EE400BB8BFB1EE400BBDEC048B02B0A6
:1015900070BD000000000000000010440000F07F5B
:1015A000182D4454FB21F93F182D4454FB21F9BF59
:1015B0000000DC3F0000203E0000F33F0000000080
:1015C000000000000000F03F0000E63F00000000C7
:1015D0000000000000000040008003400000000008
:1015E000000000000000F83F000000000000F0BF15
:1015F000323A0000F8390000B039000070390000BC
:1016000070B5614E2DED040B2DED048B82B0DDF82D
:1016100024C0DDE907235C422CF000411C4341EA71
:10162000D474069D22F00040B44205D86C422C438D
:1016300040EAD474B4420BD99DED081B9DED060B16
:1016400002B0BDEC048B04B0BDE8704000F01DBDDD
:10165000ACF14054A4F17F641C430BD0022404EA93
:10166000AC7444EAD27405439FED498B9FED4A2B3D
:101670000DD016E09DED060B51EC100B00F0DBFDDC
:1016800041EC100B02B0BDEC048B04B070BD002C1B
:1016900014BF012C9DED060BF4D0022C2ED0032C90
:1016A0002FD00B439FED3E1B9FED3F0B0AD0B14265
:1016B0001DD1B04209D121F0804120F08040099134
:1016C000079014E0002ADDDA15E0394B7B44002C4A
:1016D00008BF93ED000BD5D0012C04BF93ED000B98
:1016E000B1EE400BCED0022C08D0032C09D0B04272
:1016F0000AD1002AC6DAB0EE410BC3E7B0EE480BC0
:10170000C0E7B0EE420BBDE7401A00159FED2A9BE3
:101710003C28C8BF8DED000B15DCBCF1000FBCBF31
:1017200010F13C0F8DED009B0DDB9DED061B9DED3B
:10173000082B81EE020B51EC100B00F039FE00F08B
:101740007AFDCDE9000194B1012C0CD09DED001B78
:101750009FED1B0B022C31EE400B0CBF38EE400B03
:1017600030EE480B8EE7019880F0004001909DED2F
:10177000000BB4EE490BF1EE10FA04BF0220EFF7B4
:10178000E6F89DED000B7DE70000F07F0000000013
:10179000182D4454FB210940182D4454FB2109C045
:1017A000182D4454FB21F9BF182D4454FB21F93F57
:1017B000B038000000000000000000000000000041
:1017C000075C143326A6A13C70B54FF068422DED9E
:1017D000048BF0EE408A18EE900AB0EE608A18EEA4
:1017E000101A02EB4003B3F1654F3CBF02EB41021C
:1017F000B2F1654F7DD200BFC0F3C753C1F3C752EA
:101800009A1A1B2A09DD10F0004F14BF9FED830ABE
:101810009FED830ABDEC048B70BD12F11A0F36DA0E
:1018200011F0004F09D010F0004F0CBF9FED7D0A62
:101830009FED7D0ABDEC048B70BD88EE889A19EE91
:10184000100AFFF784FC042808BF00F03BFC18EEE8
:10185000900AFFF77CFC054618EE100AFFF777FCAC
:10186000044619EE100AFFF772FC042D18BF052D6F
:1018700008D1042C18BF052C04D1002804BF022075
:10188000EFF765F8B0EE490ABDEC048B70BD42007D
:10189000B2EB410F3AD910F0004F19BFDFED630AE8
:1018A0009FED630ADFED630A9FED630AB0EE481A0D
:1018B0000A46B1EE688A80F00041F0EE418A104697
:1018C0000A1A5200B2F1807F34D2484010F0004F23
:1018D000DFED5A1A9FED5A2A1DBF9FED5A1A70EE7E
:1018E000E10A30EE420A9FED581A08BF70EEA10AD5
:1018F00000E040E008BF30EE020AB0EE682A01EED8
:10190000482A08EE818AC2EE081A15E011F0004F4D
:1019100004BF9FED4E0AF0EE400AD1D010F0004F08
:1019200019BFDFED4B0A9FED4B0ADFED4B0A9FED30
:101930004B0AC5E7C8EE881A21EEA11A9FED482A86
:10194000DFED482A41EE022A9FED472A01EE222AC6
:10195000DFED462A41EE022A9FED452ABDEC048BBD
:1019600001EE222A21EE811A01EE020A30EE210A4E
:1019700030EE200A70BD4FF07F42B2EB400F28BF1F
:10198000B2EB410F09D2F0EE480AB0EE680ABDECA6
:10199000048BBDE8704000F08ABB40EA01035B00A5
:1019A00008BF41F0FF410BD0B2EB400F08BFB2EBD4
:1019B000410F08D120F0804008EE900A21F08041CC
:1019C00008EE101A18E7B2EB400F12BF5FEA4103AE
:1019D00040F0FF4001F000413FF40EAFB2EB410F89
:1019E00012BF5FEA400200F0004041F0FF413FF4C7
:1019F00003AF4A0092EA40033FF5FEAE002AACBFB7
:101A00009FED1C0A9FED1C0A68EE808A28EE008A72
:101A100018EE900A18EE101AEEE60000DB0FC9BFB0
:101A2000DB0FC93FDB0F4940DB0F49C00000C9BFD6
:101A300022AAFDB90000C93F22AAFD390060ED3E8F
:101A4000C30ACE37000000BF0000003F00000000C6
:101A5000000049C022AA7DBA0000494022AA7D3A6E
:101A60002DAD65BD8FB8D53D0FB511BE61C84C3EDB
:101A7000A8AAAABE0000804F0000802F10EE101A06
:101A800008B5434A6846B2EB410F26D94FF0E6400D
:101A9000B0EB410F94BF00204FF0FF300090009852
:101AA000DFED3C0A002860DB10F0010F46D060EE4D
:101AB000000ADFED391A9FED391A10F0020F00EE1F
:101AC000E11ADFED371A40EE811A21EEA01AF0EE8E
:101AD000400A40EE010A2ED041E0324B21F0004294
:101AE00093423FD911F0004FDFED2F0A20EE201A6C
:101AF000DFED2E0A19BF31EE601A71EE200A31EEC9
:101B0000201A71EE600ABDEEE01A11EE100A9FED88
:101B1000281A00F0030000EEC10A9FED261A00907B
:101B200000EEC10A9FED241A00EEC10A9FED231AB0
:101B300000EEC10AB3E7F1EE600A10E020EE000A01
:101B40009FED1F1ADFED1F1A10F0020F40EE011A71
:101B50009FED1D1A00EE211A40EE010AEBD1B0EE06
:101B6000600A08BD00F0B6FA99E710EE100A4000CE
:101B7000B0F17F4FF3D307D14FF00100EEF7E7FE4E
:101B8000BDE8084000F096BABDE8084000F08CBA05
:101B9000B61F927E0000803F336D4C39DA82083CDC
:101BA000A0AA2ABE490E494683F9223F0000004BF5
:101BB0000000C93F00A0FD390020A2331A61342C77
:101BC000B93AB2BACA9F2A3DDDFFFFBE10B52DED6E
:101BD000028BB0EE608AF0EE408A18EE101A18EE12
:101BE000900A02F0B3FD00F07040B0F1005F0CD03D
:101BF00018EE100A20F00040C0F1FF40C00F02BFF5
